:020000040800F2
:100000000080002051E90008D1F50008A92E000861
:10001000D3F50008D5F50008D7F50008000000006A
:10002000000000000000000000000000411F000868
:10003000D9F5000800000000D11F000815200008B5
:10004000DBF50008DDF50008DFF50008E1F5000844
:10005000E3F50008E5F5000865F500086BF5000814
:1000600071F5000877F500087DF50008E7F5000850
:10007000E9F50008EBF50008EDF50008EFF50008DC
:10008000F1F50008F3F50008F5F50008F7F50008AC
:10009000F9F50008FBF50008FDF5000883F50008F8
:1000A000FFF5000801F6000803F6000805F6000851
:1000B00007F6000809F600080BF600080DF6000820
:1000C0000FF6000811F6000813F6000815F60008F0
:1000D00017F60008B1FC00084101010819F60008F4
:1000E000A7F5000851F600081BF600081DF60008E9
:1000F0001FF60008000000000000000000000000E3
:1001000000000000000000005FF808F110B5054C89
:10011000237833B9044B13B10448AFF300800123B3
:10012000237010BD780400200000000038F9010899
:1001300008B5034B1BB103490348AFF3008008BD6A
:10014000000000007C04002038F9010808B50348CD
:1001500009F0C6FBBDE8084010F022B8809B0108FA
:1001600010F01EB870B5AEB007F088F8014604462E
:1001700012A807F073FB04F0D7FA054612A90AF09B
:10018000AFFA032204F111036B63002321342C63C3
:10019000254E099208AC254A254920468DF8203085
:1001A0000A96CDE90B23CDE90D33CDE90F33119339
:1001B00003F058FA38B931461E4809F091FB202166
:1001C0001D4802F0F3FD1A4A0FA9204603F014FA65
:1001D0002846214604F04EFB0F9810B1012108F08B
:1001E000ABFC0C9810B1012108F0A6FC2846134B7B
:1001F000134A144904F006FA00220721124B0B920D
:1002000008930792114B124A0993CDE90512114B3D
:100210000A9305AB93E807008DE8070094E80F0008
:1002200004F020FD2EB070BD749A0108809A010878
:10023000DB9A0108EA9A0108159B01086101000890
:10024000569B01087A9B0108D1EE000859EE000880
:10025000000008084D0100080E4B2DE90048D3E9C5
:100260000001B1F1004F08BF002810D00A4BD3E9BC
:100270000023121A63EB01039C46002107489042B9
:1002800071EB0C03B4BF01200020BDE80088012001
:10029000FBE700BF1000002008000020075101000C
:1002A00008B506F0EBFF036E60301B689847034B00
:1002B000C3E90001024B187808BD00BF0800002008
:1002C0002848002008B500F043FE044B1968411A85
:1002D000034809F005FB034B187808BDA004002073
:1002E000FF9B01082848002010B50020002106F0DF
:1002F000ADF9044678B1417980290FD1094B0279D3
:100300000168186803F0A6FD204606F037FD0821B5
:10031000204608F011FC044B187810BD034809F082
:10032000DFFAF1E73407002028480020B89C0108D4
:1003300010B506F0A3FF044607F00AF9034B188036
:10034000204607F011F9024B188010BDC4040020AC
:100350001800002008B50A4809F0C2FA00F0F8FDBC
:10036000084B186006F08AFF036E60301B689847E0
:10037000054BC3E90001FFF7DBFF044B187808BD0C
:100380008F9C0108A00400200800002028480020BD
:1003900008B506F073FFBDE8084006F0A9BF0000ED
:1003A00010B506F06BFF044606F068FF04F1580133
:1003B00000F16002034808F01BF80122024B1A60AA
:1003C00010BD00BFD80500209C04002010B51A4CB9
:1003D0002368DA0708D404F0C1F9802201461748DF
:1003E00003F09AFA0123236000F0B2FD144B134A84
:1003F0001860144B1A60FFF79BFF134809F070FA5E
:10040000124B1B68DB0701D4FFF7CAFF1621104807
:1004100007F078FF18B1B6210E4802F0C7FC0021A2
:100420000B4807F09FFF18B1B7210A4802F0BEFC45
:10043000094B187810BD00BF94040020A4050020CB
:10044000A004002034070020209C01089C04002008
:10045000D80500203F9C010828480020094B10B512
:100460001B685B6863B9FFF7F7FE044630B9064BBB
:1004700093F8203023B1054809F032FA204610BD28
:100480000124FBE734070020200000209F9C010886
:10049000F0B5444E85B0336804465D680F4685B1BB
:1004A000414D424809F01CFA6B463A4629463068ED
:1004B00003F082FA9DF8003025606371207105B069
:1004C000F0BDFFF7C9FE80B3394809F009FA0A22E6
:1004D0003849684608F093FA2946684608F0BAFA9F
:1004E0002946684608F0B6FA0121684608F0B2FAD3
:1004F000314B6846B3F9001008F0BBFA2F4B684641
:10050000198808F0CEFA684608F0AFFA0546684642
:1005100008F0ADFA01236371294B2071D3E9000182
:10052000284B2560C3E90001C9E7274D95F8203025
:10053000002BC4D1254809F0D3F925490F2268467C
:1005400008F05DFAD5E90023684608F09EFA297A9A
:10055000684608F07FFA6423A9690A26B1FBF3F123
:10056000684689B208F09DFAB5F91010684691FB0B
:10057000F6F108F07EFA69696846B1FBF6F189B2D6
:1005800008F08FFA684608F070FA0646684608F0E8
:100590006EFA0223637101232660207185F82030F2
:1005A0008DE700BF34070020C60400209E9B010891
:1005B000C49B0108C305002018000020C4040020CB
:1005C000080000201000002020000020E19B01080E
:1005D000B40500200A4B70B51B680546DB0701D443
:1005E000FFF7DEFE0524074E2946304607F0E6FEFB
:1005F00018B1013CF8D1204670BD0120FCE700BFD6
:100600009C040020D805002010B50D4C0D4B04F1C2
:100610000C00D3E90023C4E90023FFF7DBFF00232C
:1006200080F00100207284F82030B4F91010D4E971
:100630000532054809F054F9044B187810BD00BF85
:1006400020000020080000208D9D0108284800207F
:100650007FB51422002101A816F0DDFC01A8FFF7E8
:10066000B9FFDDE90332BDF90810044809F038F993
:10067000034B187807B05DF804FB00BF8D9D01089F
:10068000284800201FB56123CDE9013101A903925B
:1006900004F00EFE05B05DF804FB07B58DF80410FC
:1006A00001A98DF805208DF8063004F0C1FE03B0D5
:1006B0005DF804FB2DE9F04F87B006F0DFFDFFF792
:1006C00051FDFA2000F096FD04F048F8054603F0CD
:1006D0003DFC284606F088F8002306AC79492846F8
:1006E00044F80C3D03F0EBFE7749224641F8040B39
:1006F00008F0DCFE039951B1744809F0F1F8744830
:1007000009F0EEF840F24311724802F04FFB7248D4
:1007100009F0E6F806F0B2FD704D06462B68704C05
:1007200013F0010F04D104F0A9FD012320602B6018
:1007300006F16001206804F073FC2068694904F048
:1007400071FC614B25681A68674903A804F052FCE4
:1007500003A9284604F0A8FC644D654A2870654941
:100760002068FFF78FFF644A8DF805006349206811
:10077000FFF788FF8DF80600206805F0BDFC604A91
:100780008DF807005F492068FFF77CFF5E4A8046CE
:100790005E492068FFF776FF5D4A82465D49206822
:1007A000FFF770FF5C4B81465C4A5D49206806F0AC
:1007B000EFF95C4A06465C492068FFF763FF5B4A35
:1007C00083465B492068FFF75DFF2A788DF80400B7
:1007D0005849206805F0D2FD0746574D20689DF81E
:1007E00005302A7880F828309DF805109DF80630ED
:1007F000FFF753FF9DF807302A789DF80610206810
:10080000FFF74BFF4D4A43469DF8071020681278CA
:10081000FFF743FF53462A7841462068FFF73DFF24
:10082000DFF8248133462A7851462068FFF735FFE8
:1008300033462A7859462068FFF72FFF5B4698F821
:10084000002031462068FFF728FF9DF804302A7801
:1008500031462068FFF721FF394A4B469DF80410C6
:1008600020681278FFF719FF3B462A789DF804109C
:100870002068FFF712FF5B4698F800203946206891
:10088000FFF70BFF194A4B46394620681278FFF7ED
:1008900004FF53462A7849462068FFF7FEFE206889
:1008A00004F07CFF274809F01BF801224FF4AF71D8
:1008B000206804F00DFF002000F016FA07B0BDE834
:1008C000F08F00BF749A0108A4040020DE9C010888
:1008D000FE9C01083F9C0108119D0108980400201E
:1008E000D0050020910300082E9D0108300700204C
:1008F000CD03000810B1010851060008339D01081E
:10090000A10200083E9D0108090600084A9D010851
:1009100055030008559D0108910400085D04000876
:100920005C9D0108E90200089EAF0108C5020008AD
:10093000699D0108E5B00108284800202C480020E6
:100940002B480020739D0108E148002013B506F0F4
:1009500095FC044603689B689847204606F0A0FC77
:10096000002401234FF496720B49CDE900340B4863
:10097000234600F0CBF80A4808F0B2FF094808F017
:10098000AFFF00F09DFA40F26D11074802F00EFA39
:10099000204602B010BD00BFCC9D0108B50600087E
:1009A000D59D0108E89D01083F9C0108FF22014BED
:1009B0001A70704730070020064A13681968064B02
:1009C00019B94FF0FF321A6070471268D268D268C6
:1009D0005268F8E73C070020EC07002010B50446F9
:1009E00020B940F2F261084802F0E0F96269074B71
:1009F0009A4207D1A06A064B984203D0B0FA80F021
:100A0000400910BD0020FCE7199E01080C080020D9
:100A1000F4070020F8B51B4B1B4E1C6805463068D8
:100A20000F46043001F037FA334640B901203168EF
:100A3000164EC96A3268884022EA000232606A1C97
:100A400007D137B1196812480431BDE8F84001F008
:100A5000FFB91A686419546007D30E4A1068196800
:100A6000BDE8F840043101F0FFB90B4A106819687D
:100A7000043101F0F9F9094B1A68A24288BF1C60E1
:100A8000F8BD00BF3408002038070020BC07002054
:100A90000C080020400700203C070020EC07002045
:100AA00080B5DFF86480144F144C154E236863B989
:100AB000144B1B68012BF8D94FF08053C8F8003055
:100AC000BFF34F8FBFF36F8FEEE701F04BFAFB6878
:100AD000DD68281D01F0DFF93368013B33602368CE
:100AE000013B236001F05EFA286B01F007FC284609
:100AF00001F004FCDAE700BF20080020AC0700206A
:100B0000A80700204407002004ED00E02DE9F84F7D
:100B10004FEA820A804650460D4699460B9E01F0E8
:100B20005BFB0746002800F0AB805C2001F054FB23
:100B30000446002800F0A180076325B94FF45871DE
:100B4000564802F033F95246A521206B16F063FA9D
:100B5000236BAAF1040A9A442AF0070A6B1E04F1D7
:100B600034020F3513F8011F02F8011B197809B17F
:100B7000AB42F7D10A9D4FF0000B042D28BF04258E
:100B8000271DE562C4E9135B384684F843B001F0E1
:100B90005CF9C5F1050504F1180001F056F9C4F837
:100BA00054B02461A561646284F858B04A46414655
:100BB000504601F0AFF9206006B1346001F0D2F97F
:100BC000374B384E1A68DFF8188101321A603268E4
:100BD000002A58D134601B68012B25D1324801F01E
:100BE00029F9324801F026F9314801F023F9DFF8FC
:100BF000F490304801F01EF92F4D304801F01AF9F9
:100C0000484601F017F9284601F014F92C4801F084
:100C100011F92C4801F00EF92B4801F00BF92B4B80
:100C2000C3F800902A4B1D6001252A4A2A491368FF
:100C3000086801331360E26A636405FA02F3034350
:100C400014200B60184B394600FB023001F000F90C
:100C500001F0A8F9D8F8003063B13368DA6AE36AC2
:100C60009A4207D24FF080521C4B1A60BFF34F8F4D
:100C7000BFF36F8F2846BDE8F88F384601F03EFB82
:100C80004FF0FF35F6E7D8F80030002BCCD13368B1
:100C9000DA6AE36A9A4298BF3460C5E7199E010890
:100CA000A80700203807002044070020580700202C
:100CB0006C07002080070020D40700209407002044
:100CC000F4070020200800200C0800203C0700202A
:100CD00040070020B8070020BC07002004ED00E01A
:100CE00008080020C007002070B50446284D01F018
:100CF00039F904B92C68261D304601F0CCF860B9EA
:100D00001421E06A234B41435B5833B90122224945
:100D100082400B6823EA02030B60A36A1BB104F153
:100D2000180001F0B8F81D4A1368013313602B68EE
:100D3000A34220D131461A4801F08AF8194A1368B3
:100D40000133136001F02EF9174B1B6893B12B6828
:100D5000A3420FD1154B1B6823B140F2B641144892
:100D600002F024F84FF08052124B1A60BFF34F8FFD
:100D7000BFF36F8F70BD104A206B1368013B136087
:100D800001F0BCFA204601F0B9FAFFF715FED9E7E9
:100D90003807002044070020BC070020B8070020C7
:100DA00020080020AC07002008080020B40700201D
:100DB000199E010804ED00E0A8070020F8B50546DB
:100DC00020B940F24C51174801F0F0FF164B1B6858
:100DD000AB4220D001F0C6F8144B6C691F68144B6D
:100DE0001E6801F0DFF8BC4217D0B44215D0114B99
:100DF0009C4208D1AB6A83B995F85830012B0CBFDF
:100E000002200320F8BD0C4B9C4208D0002C0CBFE4
:100E100004200120F6E70020F4E70220F2E7042096
:100E2000F0E700BF199E0108380700203C070020AA
:100E3000400700200C0800202008002070B5044660
:100E400020B940F21C71194801F0B0FF184D2B6811
:100E5000A34229D044B301F085F82046FFF7BEFD38
:100E6000F0B1261D304601F016F801231149E26A5F
:100E700008689340034314200B600F4B314600FB7E
:100E8000023000F0E5FF2B68E26ADB6A9A4207D382
:100E90004FF08052094B1A60BFF34F8FBFF36F8F33
:100EA000BDE8704001F07EB870BD00BF199E01081A
:100EB00038070020BC0700204407002004ED00E0B4
:100EC00013B50024174B0094019350222346164972
:100ED0001648FFF71BFE012818D100F023FE012859
:100EE00014D14FF0500383F31188BFF36F8FBFF31A
:100EF0004F8F4FF0FF320E4B1A600E4B18600E4BA7
:100F00001C6002B0BDE8104001F0ACB8013007D160
:100F100040F60401094802B0BDE8104001F046BFA8
:100F200002B010BDE8070020659E0108A10A000874
:100F3000EC0700200808002034080020199E010852
:100F4000024A136801331360704700BFB4070020E2
:100F5000014B1868704700BF3408002008B501F045
:100F6000DBF8014B186808BD340800202DE9F84F64
:100F70003A4B1B68002B6AD1394B1C6801341C604A
:100F80009CB9384D2B681B6823B140F66221364866
:100F900001F00CFF354B2A68196829601A60344A41
:100FA000136801331360FFF707FD324D4FF0000B5C
:100FB0002B68314FA34211D93A68304BD16A1422C1
:100FC0004A439A58022A28BF4FF0010B2C4A126854
:100FD000002A0CBF58460120BDE8F88FDFF884A036
:100FE000DFF8A490DAF8002012681AB94FF0FF3247
:100FF0002A60E1E7DAF80020D268D66871688C428E
:1010000001D22960D8E706F10408404600F043FF0A
:10101000B16A19B106F1180000F03DFF01224FF04E
:10102000140CF06AD9F8003002FA00F11943134B9E
:10103000C9F800100CFB0030414600F009FF386889
:10104000F16AC26A914228BF4FF0010BCAE70D4A0C
:101050004FF0000B136801331360B7E7B4070020AB
:10106000340800203C070020199E0108400700209A
:10107000F0070020EC07002038070020440700207C
:1010800038080020B0070020BC0700202DE9F843F5
:101090002E4C236823B940F668012D4801F086FEE6
:1010A00000F060FF2368013B236024682CB100241A
:1010B00000F078FF2046BDE8F883264B1B68002B24
:1010C000F5D0254D254EDFF8A8801FE0EB680127FD
:1010D000DC6804F1040904F1180000F0DCFE484665
:1010E00000F0D9FE1420E26A316807FA02F30B43DC
:1010F00000FB02804946336000F0AAFE184BE26A0A
:101100001B68DB6A9A4201D3164B1F602B68002BC9
:10111000DCD10CB1FFF750FC134D2C6844B1012712
:10112000104EFFF723FF00B13760013CF9D12C606E
:101130000C4B1B68002BBAD04FF080520B4B1A603F
:10114000BFF34F8FBFF36F8F0124B1E7B4070020C7
:10115000199E0108A8070020F4070020BC07002002
:101160003807002038080020B007002004ED00E018
:101170004407002038B50C46054620B940F2CA4164
:10118000184801F013FE24B940F2CB41154801F094
:101190000DFE154B1B6823B140F2CC41114801F004
:1011A00005FEFFF7CDFE114B2A68186814192CBFF5
:1011B0000121002182422C600CD961B9FFF766FF42
:1011C00038B94FF080520A4B1A60BFF34F8FBFF30C
:1011D0006F8F38BD09B9A042F0D20021201AFFF765
:1011E00019FCEBE7199E0108B40700203408002021
:1011F00004ED00E010B5044640B94FF080520D4BAD
:101200001A60BFF34F8FBFF36F8F10BD0A4B1B687F
:1012100023B14FF4A461094801F0C8FDFFF790FE27
:1012200000212046FFF7F6FBFFF730FF0028E4D04F
:10123000EBE700BF04ED00E0B4070020199E0108B1
:10124000224B70B51A68224B12B101221A6070BD90
:10125000204E1A6033681B6B1A68B2F1A53F0BD1A0
:101260005A68B2F1A53F07D19A68B2F1A53F03D100
:10127000DB68B3F1A53F04D030683168343101F048
:1012800065FD154B1C68B4FA84F41423E4B2C4F170
:101290001F046343114DEB5823B940F688311048C1
:1012A00001F084FD142202FB04F3E91848680833B6
:1012B00040682B44984202FB045408BF43684860CE
:1012C00008BF4B606368DB683360C0E7B407002089
:1012D0003808002038070020BC0700204407002001
:1012E000199E010870B504462A4E00F03BFE04B971
:1012F0003468251D284600F0CEFD60B91421E06A4F
:10130000254B41435B5833B90122244982400B6885
:1013100023EA02030B60A36A1BB104F1180000F07A
:10132000BAFD29461E4800F093FD94F858301D4D33
:10133000012B04BF002384F8583000F033FE2A68E4
:101340002AB100F00FFEFFF737FB00F02BFE3368E9
:10135000A34211D12B6883B1134B1B6823B14FF407
:10136000D961124801F022FD4FF08052104B1A60F3
:10137000BFF34F8FBFF36F8F70BD094A11680D4ADD
:101380001268914201D13360F6E7BDE87040FFF783
:1013900057BF00BF3807002044070020BC070020CB
:1013A0000C08002008080020B4070020199E01083E
:1013B00004ED00E0A807002038B50D46044620B92A
:1013C00040F69F31074801F0F1FC074B20461968B1
:1013D000183100F049FD2846BDE838400121FFF7EB
:1013E00019BB00BF199E01083807002070B50E46D2
:1013F0001446054620B940F6CA310A4801F0D6FC29
:10140000094B28461968183100F022FD002C2146AE
:1014100008BF3046BDE8704018BF4FF0FF30FFF7FF
:10142000F9BA00BF199E01083807002038B5C36813
:10143000DC6824B940F6FA31154801F0B7FC04F134
:101440001805284600F027FD124B1B68E3B9251D3F
:10145000284600F020FD01230F49E26A0868934006
:10146000034314200B6029460C4B00FB023000F0B4
:10147000EFFC0B4BE26A1B68DB6A9A4285BF0120D6
:10148000084B0020186038BD29460748EFE700BF29
:10149000199E0108B4070020BC0700204407002063
:1014A0003807002038080020F4070020034B1B6891
:1014B0000360034B1B684360704700BFF0070020C8
:1014C0003408002070B50C46054620B940F6654149
:1014D000144801F06BFC24B940F66641114801F054
:1014E00065FC00F03FFD104B1A682368591C0FD0B3
:1014F0000E482E6800686968864201D091420ED974
:10150000521A934209D99B1A23602846FFF7CEFF4F
:10151000002400F047FD204670BD00232360012415
:10152000F7E700BF199E010834080020F0070020EB
:101530000122014B1A6070473808002070B50C4634
:101540001646054608B91B4A156805F13402626063
:10155000EA6A052B22612A6B2560E2616A6CA2604F
:10156000EA6C62614FF00002A2611BD01149096868
:10157000A9420BD12273D6B1296B0A46531A12F82D
:10158000010BA528FAD09B08238470BD032B23737D
:10159000F1D1FFF7D5FCAB6A0BB102232373FFF740
:1015A00075FDE8E72846FFF709FC2073E3E726848A
:1015B000EBE700BF3807002008B9064B1868026B3C
:1015C0001346981A13F8011BA529FAD0C0F38F000F
:1015D000704700BF38070020014B1868704700BFF4
:1015E00038070020054B1B6833B1054B1B68002BE7
:1015F0000CBF02200020704701207047080800201F
:10160000B40700202DE9F0410446002836D0234AD3
:10161000C36A11681746C96A8B4237D21426826999
:101620001F4D002AA8BF3A6806FB0353A2BFD26A27
:10163000C2F10502826142699A4221D100F1040897
:10164000404600F028FC174B48B9E06A4643AA59C7
:101650002AB901211A68814022EA01021A603A6817
:101660001968D26AE262012404FA02F008431860A1
:101670001420414600FB025000F0EAFB204603E044
:101680003B68DB6AC3620120BDE8F0811368C06C6F
:10169000DC6AA0422CBF00200120F5E738070020BB
:1016A00044070020BC070020F8B5044608B9002014
:1016B000F8BD1F4B1B68834204D040F67A711D4869
:1016C00001F074FB236D23B940F67B71194801F0DA
:1016D0006DFB236DE16AE26C013B91422365E6D02C
:1016E000002BE4D1251D284600F0D5FB124E134AED
:1016F00050B91421E76A794373582BB90120136854
:10170000B84023EA00031360E36CC3F10501A16153
:10171000E3620124116804FA03F008431060142006
:10172000294600FB036000F093FB2046C0E700BFA2
:1017300038070020199E010844070020BC0700203C
:10174000F8B50D460446002845D0036D23B940F690
:10175000C971214801F02AFBE36C9D4238BF1D4648
:10176000E36AAB4237D0236D012B34D11B4B1B688E
:10177000A34204D140F6E471174801F017FB142688
:10178000A269E36A002AE562A4BFC5F10505A56167
:10179000134D626906FB03539A421CD1271D38463C
:1017A00000F079FBE26A0F4C40B95643AB592BB9B4
:1017B00001212368914023EA0103236001231420BF
:1017C000216893400B432360394600FB0250BDE87B
:1017D000F84000F03DBBF8BD199E01083807002015
:1017E00044070020BC070020044B1A681AB119688E
:1017F0000A6D01320A651868704700BF380700207B
:101800002DE9F0411E4C1E4680460F46154600F05D
:10181000A9FB236893F85830022B14D001212368C8
:101820005A6D22EA08025A65236883F8581056B1A7
:101830003046FFF7EFF84FF08052124B1A60BFF3BB
:101840004F8FBFF36F8F00F0ADFB00F08BFB15B136
:1018500023685B6D2B602368002293F85830022BBD
:1018600009BF012500252368596D04BFB943596597
:10187000236883F8582000F095FB2846BDE8F081E6
:101880003807002004ED00E0F8B50E4617461D4667
:10189000044620B941F219212B4801F087FA00F0E3
:1018A00061FB0DB1636D2B60022394F8585084F8EE
:1018B0005830EDB2042F16D8DFE807F00A03070509
:1018C0001100636D1E43666502E0636D013363655D
:1018D000012D11D0012400F065FB2046F8BD022D3A
:1018E000F1D10024F7E7636D0133F1D041F24A21D1
:1018F000154801F05BFAEBE7261D304600F0CBFA05
:101900001420124AE36A11689D400D431560104A85
:10191000314600FB032000F09BFAA36A23B141F299
:101920005921094801F042FA0A4BE26A1B68DB6A56
:101930009A42CFD94FF08052074B1A60BFF34F8FB6
:10194000BFF36F8FC6E700BF199E0108BC070020D8
:10195000440700203807002004ED00E02DE9F8439B
:10196000DDF820800E4691461D46044620B941F21E
:101970008C21354801F01AFA00F0CEFBEFF3118705
:101980004FF0500383F31188BFF36F8FBFF34F8F76
:101990000DB1636D2B60022394F8585084F85830D1
:1019A000EDB2B9F1040F16D8DFE809F00A03070514
:1019B0001100636D1E43666502E0636D013363656C
:1019C000012D11D0012087F31188BDE8F883022D85
:1019D000F1D10020F7E7636D0133F1D041F2CF215F
:1019E000194801F0E3F9EBE7A36A23B141F2DA21E8
:1019F000154801F0DBF9154B1B6803BB251D284674
:101A000000F049FA01231249E26A0868934003434F
:101A100014200B6029460F4B00FB023000F018FA2F
:101A20000D4BE26A1B68DB6A9A42CBD90123B8F1FD
:101A3000000F01D0C8F80030084A1360C2E704F173
:101A400018010748EAE700BF199E0108B407002003
:101A5000BC07002044070020380700203808002079
:101A6000F407002038B5054608B9084B1D68002466
:101A700000F078FA95F85830022B04BF85F85840EA
:101A8000012400F08FFA204638BD00BF380700203F
:101A9000F8B50F4C00F066FA2568ADB90D4F0E4E43
:101AA000384600F0C7F9304600F0C4F90B4B2A461F
:101AB0001F600B4B0C210A201E6000F021FD2060EE
:101AC00010B1084901F0E0F8BDE8F84000F06ABA4A
:101AD0007008002044080020580800203C0800201E
:101AE000400800206A9E0108914208B541600061EB
:101AF0000AD8D21A83699A420DD2084B011D186880
:101B000000F0B2F9002008BD9A4201D2994202D2F7
:101B1000011D034BF3E70120F5E700BF400800205B
:101B20003C08002007B5FFF7B3FF0C4B1B6843B917
:101B30000B484FF4897101F039F9002003B05DF8CA
:101B400004FB084BC822019301230749009307486F
:101B50000023FEF7DBFF0028EAD0EFE77008002043
:101B60006F9E010874080020BC9E0108891C0008B3
:101B70002DE9F04180462C200D4617461E4600F008
:101B80002BFB044688B125B94FF4B671084801F023
:101B90000DF9FFF77DFF069BC4F80080C4E90657E6
:101BA00026626362201D00F050F92046BDE8F081F6
:101BB0006F9E01082DE9FF410D4690461F460646DF
:101BC00020B94FF4C3710F4801F0F0F80E4C2068B3
:101BD00078B1052DCDE9015803960DDCFFF702FD24
:101BE000002302280CBF0A9A1A4601A9206800F0B7
:101BF000ABFC04B0BDE8F08100233A4601A900F037
:101C000059FDF6E76F9E0108700800202DE9F743A3
:101C100000271A4DDFF86C802B681A6832B9184A11
:101C200011681360296003B0BDE8F083DB68DC68ED
:101C30001E6804F10409484600F02DF9636A204645
:101C40009847E369012BE7D1A36933449E4206D24A
:101C5000636024614946286800F006F9DCE7002348
:101C60000097324619462046FFF7A4FF0028D3D13B
:101C700040F27231404601F099F8CDE73C0800206F
:101C8000400800206F9E01082DE9F04F4FF0010839
:101C9000624D89B0DFF898B1DBF80020136843B3D8
:101CA0000024D368D3F80090FFF74AF9FFF750F902
:101CB0005B4B82461A681F4690425A4E1CD31860EE
:101CC000002C4CD0584B1B681A68B2FA82F25209A9
:101CD000A9EB0A01306801F00FF8FFF7D7F998B9BE
:101CE0004FF08052514B1A60BFF34F8FBFF36F8F8D
:101CF0000AE001249946D7E70393FFF787FF039B88
:101D0000C3F800A0FFF7C2F9002205A9306800F06F
:101D100075FD0028BED0059B002BF5DB079C636991
:101D200013B1201D00F0B7F8FFF712F93B688146A8
:101D3000984201D2FFF76AFF059BC7F80090092B74
:101D4000E2D808FA03F313F4047A57D113F0C70F5B
:101D500033D19B06D8D5204600F0D0FAD4E7814590
:101D600029D8FFF793F9DBF80030DB68D3F80CB023
:101D70000BF1040000F08FF8DBF81C30012B15D1BB
:101D8000DBF818104B46524649445846FFF7ACFE64
:101D900060B1009423464A4621465846FFF70AFFA1
:101DA00020B94FF4F471284601F000F8DBF8243034
:101DB00058469847A8E722468AE7A169069B4A4603
:101DC00019442046FFF790FE00289DD0636A204604
:101DD0009847E369012B97D1A2690699CDF800A035
:101DE0000A44534651462046FFF7E4FE00288BD1B3
:101DF00040F20131284600F0D9FF85E7069BA36138
:101E000023B94FF44671284600F0D0FFA1694B4634
:101E10004A4649442046FFF767FE75E76F9E010872
:101E20006C080020700800204008002004ED00E04D
:101E30003C0800204FF0FF3200F108034360C0E986
:101E4000022303610023036070470023036170478E
:101E500043689A684B608A609A6851609960036829
:101E600008610133036070470A6830B5531C0AD11A
:101E700003695A684A6091608B6059600368086121
:101E80000133036030BD00F108035C6825689542AA
:101E9000EFD82346F9E70369D0E901128A60826826
:101EA00051605968814208BF5A60002202611A6875
:101EB000013A1A601868704706480068006880F3A5
:101EC000088862B661B6BFF34F8FBFF36F8F00DF34
:101ED00000BF000008ED00E0002307B501930B4BA5
:101EE0001B68013303D0CA21094800F05FFF4FF09F
:101EF000500383F31188BFF36F8FBFF34F8F019BA4
:101F0000002BFCD003B05DF804FB00BF48000020AC
:101F1000C49E01084FF0807340F8043C054B21F04B
:101F2000010140F8081C40F80C3C40F8202C4038D7
:101F3000704700BFD91E000800000000000000002C
:101F4000074B19680868B0E8F00F80F30988BFF301
:101F50006F8F4FF0000080F311884EF00D0E704728
:101F6000380700204FF0500383F31188BFF36F8FC1
:101F7000BFF34F8F084A13680133012B136009D157
:101F8000064B1B6813F0FF0F04D040F27511044894
:101F900000F00CBF704700BF4800002004ED00E0D7
:101FA000C49E010810B5074C236823B94FF4BE71D5
:101FB000054800F0FBFE2368013B23600BB983F367
:101FC000118810BD48000020C49E010800000000D8
:101FD000EFF30980BFF36F8F0D4B1A6820E9F00F04
:101FE00010602DE908404FF0500080F31188FFF792
:101FF00027F94FF0000080F31188BDE80840196808
:102000000868B0E8F00F80F30988BFF36F8F70475E
:102010003807002008B54FF0500383F31188BFF351
:102020006F8FBFF34F8FFEF7A1FF18B14FF08052B3
:10203000024B1A60002383F3118808BD04ED00E011
:102040000022054B05491A600A6041F26701044A03
:10205000116007221A60704710E000E018E000E00D
:1020600014E000E013B5264B264C1A78D2B2019248
:10207000FF221A701B78244ADBB28DF803309DF8DA
:10208000033003F0500313700723002223609DF8F0
:102090000310581E090629D402B123602368032BBC
:1020A00004D04FF49B71194800F080FE2368144A55
:1020B0001B0203F4E06323600024019BDBB2137076
:1020C000134B1A6842F470021A601A6842F07042A8
:1020D0001A60FFF7B5FF0F4B1C60FFF7EDFEFFF72F
:1020E000AFF8FFF7F9FE204602B010BD9DF80330AF
:1020F00001225B00DBB28DF803300346C7E700BF67
:1021000000E400E07C08002078080020C49E01085C
:1021100020ED00E04800002008B5EFF305830F2B09
:102120000AD90D4A9B5C0D4A12789A4204D940F2B2
:10213000A5210B4800F03AFE0A4B0B4A1B681268B7
:1021400003F4E063934206D9BDE8084040F2B521AC
:10215000034800F02BBE08BDF0E300E07808002043
:10216000C49E01080CED00E07C08002010B50F4B68
:102170001A68824218D35C681919884201BF416805
:10218000184609195960446801198A4207D108495B
:1021900009688A421FBF5168126809194160984254
:1021A000026018BF186010BD1346E1E7904400209C
:1021B0008008002038B5064B064D1C68246804B919
:1021C00038BD6307FAD07921284600F0EFFDF5E726
:1021D00090440020249F01082DE9F8430746FEF7AC
:1021E000AFFE3F493F4D0B680BBB3F4A3F4E500788
:1021F0001DBFD01D20F0070002F570534FF470533F
:102200001CBF02461B1A00201344083B23F007039F
:1022100070603260C3E90000981A0B60C2E90030B8
:10222000334B1860334B18604FF000432B602B6822
:102230001F4252D1002F41D007F1080462071CBF92
:1022400024F007040834002C47D02A4B1A6898461B
:10225000A24242D3254B1E687268A24202D2306865
:10226000002837D10968B14237D01F683168121B86
:10227000102A07F10807196010D906EB040919F0B4
:10228000070F03D0D7211C4800F090FD7368484623
:102290001B1BC9F804307460FFF768FF14497268AB
:1022A000D8F8003008689B1A8342C8F8003038BF5D
:1022B0000B602B681343736000233360FEF7E6FE68
:1022C0007B0704D040F217110B4800F06FFD384631
:1022D000BDE8F88333460646BEE70027EEE700BFB9
:1022E00080080020844400208408002090440020BE
:1022F0008C44002088440020249F010838B50446FF
:1023000070B3184D50F8041C2A68114204D140F2F1
:102310002B11154800F04AFD54F8083C23B14FF446
:102320009671114800F042FD54F8043C2A681342AB
:1023300016D054F8081C99B923EA020344F8043C67
:10234000FEF7FEFD094A54F8043C1168A4F10800A8
:102350000B441360FFF70AFFBDE83840FEF796BE56
:1023600038BD00BF84440020249F01088844002019
:1023700010B50446FFF7F6FDA46BFFF713FEB4FAA1
:1023800084F0400910BD70B51546026C0446866B9A
:1023900042B905689DB98068FFF786F9A5600136E6
:1023A000A66370BD6DB9406814F011FE6368226CBD
:1023B0001344A2686360934201D3236863600020E2
:1023C000EDE7C06814F003FE236CE2685B4221680D
:1023D0001A448A42E2603EBFA2689B18E360022D65
:1023E000EDD10EB1013EEAE73046D8E703461A6C5C
:1023F00010B4084662B1D9689C681144A142D96002
:1024000028BF196810BC28BFD960D96814F0DFBD97
:1024100010BC704770B50446FFF7A4FD94F8455012
:1024200004F124066DB2002D14DCFF2384F845303E
:10243000FFF7B8FDFFF796FD94F8445004F110063D
:102440006DB2002D12DCFF2384F84430BDE87040EB
:10245000FFF7A8BD636A002BE7D03046FEF7E6FF22
:1024600008B1FFF765F8013D6DB2DCE72369002B89
:10247000E9D03046FEF7DAFF08B1FFF759F8013D21
:102480006DB2DEE738B50D46044620B940F20311BF
:10249000194800F08BFCFFF765FDD4E90F314B4381
:1024A0002268D0185B1A1344A060E3600020FF2369
:1024B000A063626084F8443084F8453095B923699C
:1024C00063B104F11000FEF7B1FF38B14FF0805254
:1024D0000A4B1A60BFF34F8FBFF36F8FFFF762FD98
:1024E000012038BD04F11000FFF7A4FC04F1240022
:1024F000FFF7A0FCF2E700BF829F010804ED00E0B7
:10250000F8B50D461746064620B94FF4BB710D4885
:1025100000F04CFC05FB06F05030FFF75DFE044672
:1025200048B155B92060C4E90F6501212046FFF785
:10253000A9FF84F84C702046F8BD00F150030360F9
:10254000F1E700BF829F01082DE9FF47884601920D
:102550001E46044620B940F2F1214B4800F026FC0B
:10256000B8F1000F06D1236C23B140F2F2214648A6
:1025700000F01CFC022E07D1E36B012B04D040F2CB
:10258000F321414800F012FCFFF72CF830B9019B11
:1025900023B140F2F6213C4800F008FC0027B94680
:1025A000DFF8E8A0FFF7DEFCA26BE36B9A4201D3F1
:1025B000022E19D1324641462046FFF7E4FE636AF7
:1025C0001BB104F12400FEF731FF38B14FF0805207
:1025D0002E4B1A60BFF34F8FBFF36F8FFFF7E2FCF4
:1025E000012004B0BDE8F087019D1DB9FFF7DAFCBA
:1025F0000020F6E717B902A8FEF758FFFFF7D2FC54
:10260000FEF79EFCFFF7AEFC94F84430FF2B08BFAA
:1026100084F8449094F84530FF2B08BF84F8459027
:10262000FFF7C0FC01A902A8FEF74CFF28BBFFF78B
:1026300099FCA26BE36B9A420ED1FFF7B3FC0199B0
:1026400004F11000FEF7B8FE2046FFF7E3FEFEF7A8
:102650001DFD48B10127A5E7FFF7A4FC2046FFF7C1
:10266000D9FEFEF713FDF5E74FF08053CAF80030AE
:10267000BFF34F8FBFF36F8FECE72046FFF7CAFE23
:10268000FEF704FDB4E700BF829F010804ED00E0FF
:1026900010B5024600210120FFF732FF044638B191
:1026A000002383600360C3601A461946FFF74CFF9E
:1026B000204610BD2DE9F843894690461F46044642
:1026C00020B940F2C331274800F070FBB9F1000F88
:1026D00006D1236C23B14FF47171224800F066FBE0
:1026E000022F07D1E36B012B04D040F2C5311D4806
:1026F00000F05CFBFFF710FDEFF311864FF0500385
:1027000083F31188BFF36F8FBFF34F8FA26BE36B1F
:102710009A4201D3022F22D194F845503A466DB225
:1027200049462046FFF72FFE6B1C13D1636A0BB995
:1027300001200BE004F12400FEF778FE0028F7D01A
:10274000B8F1000FF4D00120C8F8000086F311881A
:10275000BDE8F88301356DB284F84550E8E7002004
:10276000F4E700BF829F010870B50D46044620B90A
:102770004FF48C61204800F019FB236C23B140F228
:1027800064411D4800F012FB236833B9A36823B1EC
:1027900040F26941184800F009FBFFF7BDFCEFF378
:1027A00011864FF0500383F31188BFF36F8FBFF38F
:1027B0004F8FA26BE36B93421CD994F845300132E2
:1027C0005BB2A2635A1C10D1636A0BB9012009E005
:1027D00004F12400FEF72AFE0028F7D0002DF5D0E2
:1027E0000120286086F3118870BD01335BB284F844
:1027F0004530EBE70020F5E7829F01082DE9F04323
:1028000085B00F460192044620B94FF4A0614248BA
:1028100000F0CCFA37B9236C23B140F204513E48A2
:1028200000F0C4FAFEF7DEFE30B9019B23B140F29E
:102830000951394800F0BAFA0026B046DFF8DC90BA
:10284000FFF790FBA56BD5B139462046013DFFF758
:10285000CDFDA563236963B104F11000FEF7E6FD29
:1028600038B14FF080522D4B1A60BFF34F8FBFF33A
:102870006F8FFFF797FB012005B0BDE8F083019D46
:102880001DB9FFF78FFB0020F6E716B902A8FEF787
:102890000DFEFFF787FBFEF753FBFFF763FB94F892
:1028A0004430FF2B08BF84F8448094F84530FF2B58
:1028B00008BF84F84580FFF775FB01A902A8FEF761
:1028C00001FEF0B92046FFF753FDA0B1019904F1D4
:1028D0002400FEF771FD2046FFF79CFDFEF7D6FBB6
:1028E00038B94FF08053C9F80030BFF34F8FBFF3B2
:1028F0006F8F0126A4E72046FFF78CFDFEF7C6FB8D
:10290000F7E72046FFF786FDFEF7C0FB2046FFF7FE
:102910002FFD0028EDD0B6E7829F010804ED00E00E
:102920002DE9FF410446019120B940F291515248EE
:1029300000F03CFA236C23B140F295514E4800F070
:1029400035FAFEF74FFE30B9019B23B140F29A51A0
:10295000494800F02BFA00252F462E46DFF81C814F
:10296000FFF700FBA36BE3B1013BA363236813B93B
:10297000FEF73AFFA060236963B104F11000FEF78F
:1029800055FD38B14FF080523C4B1A60BFF34F8F6A
:10299000BFF36F8FFFF706FB0125284604B0BDE8A3
:1029A000F081019B4BB925B140F2E151324800F072
:1029B000FDF9FFF7F7FA0025EFE717B902A8FEF7D0
:1029C00075FDFFF7EFFAFEF7BBFAFFF7CBFA94F8C5
:1029D0004430FF2B08BF84F8446094F84530FF2B47
:1029E00008BF84F84560FFF7DDFA01A902A8FEF7E9
:1029F00069FD40BB2046FFF7BBFCF0B123683BB943
:102A0000FFF7B0FAA068FEF7FDFD0546FFF7CAFA2A
:102A1000019904F12400FEF7CFFC2046FFF7FAFCF1
:102A2000FEF734FB38B94FF08053C8F80030BFF3DD
:102A30004F8FBFF36F8F012792E72046FFF7EAFC25
:102A4000FEF724FBF7E72046FFF7E4FCFEF71EFB4A
:102A50002046FFF78DFC0028EDD0002D9DD0FFF71C
:102A600081FA616A19B1236B1968C1F10501A06887
:102A7000FEF766FE9DE700BF829F010804ED00E0BF
:102A80002DE9F04385B00F460192044620B94FF47A
:102A9000CD61424800F08AF937B9236C23B140F286
:102AA0006C613E4800F082F9FEF79CFD30B9019B55
:102AB00023B140F27161394800F078F90026B04640
:102AC000DFF8DC90FFF74EFAA36BD3B1394620460E
:102AD000E568FFF78BFC636AE56063B104F12400ED
:102AE000FEF7A4FC38B14FF080522D4B1A60BFF3B3
:102AF0004F8FBFF36F8FFFF755FA012005B0BDE888
:102B0000F083019D1DB9FFF74DFA0020F6E716B9D5
:102B100002A8FEF7CBFCFFF745FAFEF711FAFFF724
:102B200021FA94F84430FF2B08BF84F8448094F8CD
:102B30004530FF2B08BF84F84580FFF733FA01A921
:102B400002A8FEF7BFFCF0B92046FFF711FCA0B1C8
:102B5000019904F12400FEF72FFC2046FFF75AFCF0
:102B6000FEF794FA38B94FF08053C9F80030BFF33C
:102B70004F8FBFF36F8F0126A4E72046FFF74AFC73
:102B8000FEF784FAF7E72046FFF744FCFEF77EFAEB
:102B90002046FFF7EDFB0028EDD0B6E7829F010845
:102BA00004ED00E02DE9F84389469046054620B93A
:102BB00040F2FB61204800F0F9F8B9F1000F06D1AE
:102BC0002B6C23B140F2FC611B4800F0EFF8FFF7DB
:102BD000A3FAEFF311874FF0500383F31188BFF38B
:102BE0006F8FBFF34F8FAC6B1CB395F844604946B1
:102BF00076B22846FFF7FAFB013C731CAC6313D195
:102C00002B690BB901200BE005F11000FEF70EFC5B
:102C10000028F7D0B8F1000FF4D00120C8F8000068
:102C200087F31188BDE8F883013676B285F84460F1
:102C3000E8E72046F4E700BF829F010810B504468C
:102C400020B940F28A71054800F0B0F8FFF78AF920
:102C5000A46BFFF7A7F9204610BD00BF829F0108B3
:102C600038B5054620B940F2A471064800F09EF838
:102C7000FFF778F9A86BEC6B241AFFF793F920465D
:102C800038BD00BF829F0108002330B5064A52F8C4
:102C9000335002EBC3041DB942F83310606030BDFD
:102CA0000133052BF3D1FAE7C8500020002310B5FB
:102CB000074A02EBC3014C68844204D1002042F869
:102CC0003300486010BD0133052BF2D1FAE700BF95
:102CD000C850002010B5044620B94FF4F8610548EB
:102CE00000F064F82046FFF7E1FF2046BDE8104001
:102CF000FFF704BB829F010870B504460D461646D7
:102D0000FFF730F994F84430FF2B04BF002384F818
:102D1000443094F84530FF2B04BF002384F845303D
:102D2000FFF740F9A36B2BB93246294604F1240082
:102D3000FEF75CFB2046BDE87040FFF76BBB000070
:102D4000014B1860704700BF2445002073B5124C3A
:102D5000064623780D46114A1BB913780BB172B69B
:102D6000FEE70123002113700D48642214F053F98B
:102D70002B4600960B4A6421094814F0BBFF0A4B0E
:102D80001B6803B198470125054E304606F0ECFD5F
:102D900072B62570F9E700BF044500209844002072
:102DA0009A440020E19F010824450020F7B5144C07
:102DB000064623780D46134A1BB913780BB172B639
:102DC000FEE70123002113700F48642214F023F959
:102DD0002B4600960D4A64210B4814F08BFF0C4BD8
:102DE0001B6803B198470125074F0A4E384606F085
:102DF000BBFD304606F0B8FD72B62570F6E700BFA1
:102E000005450020994400209A44002009A00108AB
:102E10002445002018A001080368DFF888C080B5A9
:102E2000CCF80030164F4368164E3B608368164D51
:102E30003360C36815492B600369154A0B60436909
:102E4000144C13608369C0692360134B1860DCF86D
:102E50000000386830682868096810481268002146
:102E6000226864221B6814F0D6F823680C4A642197
:102E70000A4814F03FFF094806F076FDFEE700BF60
:102E8000144500201C450020204500201845002046
:102E900000450020084500200C4500209A440020F1
:102EA000CE9F010810450020074B1B6803B19847CF
:102EB0001EF0040F0CBFEFF30880EFF30980816967
:102EC000004A1047192E00082445002010B10121A6
:102ED00005F032BE704708B106F09EBD70478068AD
:102EE0007047406870474368012B08D1D0E904322D
:102EF000934204D01878003018BF0120704700209A
:102F000070474B6870B5042B04460E464FF0000323
:102F100004D0C0E900338360204670BDD1E90425A8
:102F2000AD1AC0E9003383602846FFF7D4FFC4E937
:102F300000000544A560D6E90453024629468B42A9
:102F400005D00AB10E78167001310132F7E75B1B2C
:102F500018446060E0E742680346022A06D1D3E9DC
:102F600004031B1A032B01D906F0CDBD00207047C6
:102F70004368032B06D1D0E904329A4208BF0023EC
:102F8000184670470023FBE7037870B58168044654
:102F9000B3B1284A284806F0A3FC6368022B12D17B
:102FA0002046FFF7D8FF0146244806F099FCE16867
:102FB0000B78002B3CD02248BDE8704006F090BC56
:102FC000204A2148E7E7032B05D12046FFF7D0FF31
:102FD00001461E48E9E7042B0ED100251C4ED4E91A
:102FE0000431C91A8D4205D2595D304606F078FC8D
:102FF0000135F4E71748D8E7012B08D12046FFF741
:1030000072FF1549154B002818BF1946E1E7002546
:103010000F4ED4E904239B1A9D4205D2515D3046E0
:1030200006F05EFC0135F4E70D4806F059FCBEE7FA
:103030000C48C1E7E89A0108BCA00108D0A001082B
:10304000F2A0010868A40108C6A0010885A2010831
:10305000C5D60108DAA00108B6A00108B1A0010890
:10306000E0A0010867A40108B1F5705F2DE9F843FD
:1030700004460F4602D9174805F020FD066883680C
:103080009B1B994219D9D0F804900846FFF723FFFB
:1030900005460346A9EB0608B14505D00BB13278C9
:1030A0001A7001360133F7E72068FFF70FFF05EBD1
:1030B000080325603D446360A56025683DB9284646
:1030C000C4E90155FFF702FF2846BDE8F883012057
:1030D000FBE700BF34A001082DE9F0410368561A50
:1030E000904682680446D21A96420D4615D930465B
:1030F000FFF7F1FE07460346A84505D02A7803B13D
:103100001A7001350133F7E720683E44FFF7DEFE11
:10311000C4E901662760BDE8F0814768481EFF1AD0
:10312000BE420ED81A469D19A91A002904DD10F8CE
:10313000011F02F8011BF7E7002EA8BF9B1963606F
:10314000E9E73D441F44FA1A002A04DD10F8012F74
:1031500003F8012BF7E763682E461846B04505D003
:10316000327800B1027001360130F7E7A8EB0508AC
:103170004344E4E708B509C81B1AC3F570508842F8
:1031800002D2104605F09AFC994238BF19465818E9
:1031900005D2B0F5705F28BF4FF4705008BD4FF4F2
:1031A0007050FBE72DE9F8430C46591C20461546A4
:1031B0001F46FFF759FF064680B14FF00003EA199A
:1031C00029462046FFF788FFD4E901539D4208D0E5
:1031D0000DB100232B706368013363603046BDE896
:1031E000F8831B4A01212046FFF7C4FF23680746E6
:1031F000A5EB0309FFF76FFE10EB090F1CBF0023BF
:1032000000F80930236880461A460146954205D0E9
:1032100009B11078087001320131F7E7D31A013390
:103220004344104619466568954207D019B192F893
:1032300000C081F800C001320131F5E72D1A1D44AC
:1032400020684744FFF742FEC4E90085A760C5E750
:103250006FA001081346426810B5032A06D1BDE8E5
:1032600010400A4600F11001FFF79CBF8168024838
:1032700006F036FB002010BDF9A001082DE9F04151
:1032800005460E4661B1D0E90132D21A8A4209D30D
:1032900000221E4403B11A700133B342FAD16B60AD
:1032A000BDE8F081114AFFF765FF8046FFF713FE86
:1032B000D5E9001407460A460346944205D00BB1EF
:1032C0001078187001320133F7E70023641A3C4488
:1032D000264404B123700134B442FAD12868FFF7C0
:1032E000F5FDC5E900744744AF60D9E7DDA10108E9
:1032F000D0E90032D21A914210B503D9891AFFF7EA
:10330000BDFF10BD3CBF5B184360FAE770B50C46CB
:10331000012120461646FFF7A7FE054628B10121E8
:103320002046FFF7E5FF23681E70284670BD0000A9
:10333000426808B5012A06D1BDE808400A4600F1F6
:103340001001FFF7E3BF8168024806F0C9FA0020C8
:1033500008BD00BF6CA1010810B50C1A134605D0BA
:1033600001462246184613F03DFE0346181910BDCB
:103370002DE9F0410446A2EB01081646A368226835
:1033800008469B1A98450F4615D94046FFF7A3FDFE
:1033900005460346BE4205D00BB13A781A70013794
:1033A0000133F7E72068FFF791FD25604544C4E944
:1033B0000155BDE8F0816568AD1AA84504D83146CD
:1033C000FFF7CAFF6060F4E70D442946FFF7C4FF2A
:1033D000636829461A468E4205D00AB108781070F3
:1033E00001310132F7E7751B1D446560E1E700001C
:1033F00070B5D0E9043100F110060446C91A304610
:10340000FFF732FE054640B1D4E90712914206D1DA
:10341000A168064806F064FA0025284670BD4FF002
:1034200000033046FFF7A4FFF7E700BF89A00108BB
:103430002DE9F0418368A2EB0108174602680446B3
:103440009B1A98450E4615D94046FFF744FD0546A0
:103450000346B74205D0327803B11A700136013302
:10346000F7E72068FFF732FD25604544C4E90155C0
:10347000BDE8F0814568AD1AA84505D83946304603
:10348000FFF76AFF6060F3E70D4429463046FFF717
:1034900063FF636829461A468F4205D0087802B157
:1034A000107001310132F7E77D1B1D446560DFE7D5
:1034B00037B50D4601A8114606F03EFB042128460B
:1034C000FFF7D2FD044630B14FF0000302AA01A974
:1034D0002846FFF7ADFF204603B030BDFFF7E8BF39
:1034E000426808B5022A06D1BDE808400A4600F144
:1034F0001001FFF7DDBF8168024806F0F1F90020F6
:1035000008BD00BFA4A10108FFF7EABFF7B50E464A
:1035100004461046154614F053FC00237268C4E9B3
:103520000033013AA360032A12D8DFE802F0022B2D
:103530003B412D49284614F031FC20B12B49284647
:1035400014F02CFC38B9012221463046FFF7DEFE8C
:10355000204603B0F0BD2649284614F01FFC20B1D8
:103560002449284614F01AFC08B90022ECE700228E
:1035700002A941F8042D284614F04EFD021C18BF84
:103580000122E1E702A941F8043D0022284614F097
:1035900043FD019B0246AB42DAD021463046FFF79D
:1035A00087FFD5E72A462146304600F025F8CFE7C9
:1035B00010F00106CCD1470839462046FFF754FDEC
:1035C0000028C5D039462046FFF792FEB742BFD04B
:1035D000022105EB460006F07EFA0028B8DB2368DE
:1035E00098550136F2E700BFB1A0010844A00108D8
:1035F000B6A0010849A00108F0B5436885B0032BC7
:103600000D46164615D0014601A8FFF77FFFDDE9FC
:10361000011291420BD04FF000032846FFF7A8FE9D
:1036200001240198FFF752FC204605B0F0BD0024AC
:10363000F7E7104614F0C4FB471C39462846FFF74D
:1036400013FD044618B9064806F04AF9ECE74FF0B6
:103650000003F21931462846FFF73EFDE4E700BFBC
:103660004FA001080A4600F11001FFF7C5BFF8B5E9
:103670000D461946284616461F46FFF7F5FC044638
:1036800030B14FF00003F21931462846FFF7D0FE63
:103690002046F8BD1346426810B5042A06D1BDE89D
:1036A00010400A4600F11001FFF7E1BF81680248AF
:1036B00006F016F9002010BD33A101082DE9F041F4
:1036C0000C4690461D46064640B139B10849184699
:1036D00005F02EFA074618B930602060BDE8F08189
:1036E0002A46414613F073FC37602560F6E700BFB9
:1036F000CCF5010870B5054610460E46144614F088
:103700005FFB2246034631462846BDE87040FFF77E
:10371000D5BF000010B50C4631B1044900F0E6FCFD
:10372000231A5842584110BD0846FCE77AA3010805
:1037300010B500B121B9064806F0D2F8002010BD3E
:103740001AB9044AFFF7D6FFF8E70120F7E700BFF0
:10375000F7A1010804A201082DE9F3410D46164620
:103760001F46FFF7E5FFB8B10E49222005F0E0F94A
:103770000446A0B13046FFF7B2FB80463046FFF763
:10378000F7FB14F01DFB3B46CDE90080064A2221E1
:10379000204614F0AFFA286002B0BDE8F08128603E
:1037A000FAE700BFCCF501083CA201082DE9F84377
:1037B0000E46984616F8013B02F1FF390370466049
:1037C000C0F80890044615463D214A46304613F09D
:1037D000E1FB074668BB4B46182B28BF1823C4F8EB
:1037E0003001A36204F10C05A26A3146284613F0A9
:1037F000EEFB0022A66AA3191A7337B1D4F8302160
:10380000791C04F12C0013F0E2FB0022D4F83031D3
:10381000234483F82C202EB12946404600F066FC54
:10382000C4F83401D4E901120A48BDE8F84306F0AF
:10383000CDB8831B023DED1A182B1A46A8BF1822DB
:10384000B5F5807F28BF4FF48075A262C4F830516F
:10385000C8E700BF44A2010830B504460D46084B36
:103860009DB00093074A084B642103A814F042FA64
:1038700003AA29462046FFF73DFF1DB030BD00BF1B
:1038800036A201082EA2010813A201082DE9F04377
:103890001646642203F10C048FB007468846204682
:1038A0001849ADF8042014F079FA70B9336B23B1DC
:1038B000154A322101A814F01DFA01AA41463846E2
:1038C000FFF718FF0FB0BDE8F08320460F4914F052
:1038D00065FA0446A0B9736B002BEED00125DFF822
:1038E0003490736B01A81B5DC5F1320128444A4630
:1038F000013414F0FFF9102C05F10205F1D1DCE7D9
:10390000034ADBE750A2010855A2010859A20108A9
:1039100061A20108C5D60108016000210273C0E957
:1039200001117047F8B5054617460E4639B332B354
:103930001D49182005F0F2F8044608B3C0E90067F5
:1039400000261A4B00F108074361C0E902660661D0
:103950008021384605F010F8D4E90012384605F009
:1039600049F81149082005F0D9F890B16B68C0E911
:10397000004603B96860AB6803B15860A860F8BD41
:103980000B4805F0ADFF01213046BDE8F84005F0D9
:10399000D3B8084805F0A4FF0121206805F0CCF851
:1039A00018212046F1E700BFCCF501088081828311
:1039B00000A3010805A3010870B54468054604B3D7
:1039C000266806F1080004F0DFFFD6E903239A42D7
:1039D000C4B216D16B681BB96A210B48FFF7E6F930
:1039E0006868082143686B6005F0A6F86B6803B946
:1039F000AB600121306805F09FF81821304605F0D2
:103A00009BF8204670BD00BF9DA2010810B504467A
:103A1000006810B1012105F08FF8204610BD7FB578
:103A20000546FFF75CFA14F0CBF90446861C2846DD
:103A3000FFF757FA013803281DD8DFE800F0020627
:103A4000080F0734601C04B070BD0D34FAE7284637
:103A5000FFF78EFA14F0B4F93418F3E701A82946F9
:103A6000FFF74FFADDE9014301A81B1B06EB4304F6
:103A7000FFF7CCFFE6E70B34E4E700002DE9F04761
:103A800086B08146884614461D46FFF751FE68B150
:103A90002046FFF7C4FF4049074605F049F80646AF
:103AA000C9F8000028B93D4805F01AFF06B0BDE886
:103AB000F0872046FFF715FA0138032864D8DFE8BD
:103AC00000F00214253D2046FFF709FA8146204602
:103AD000FFF709FA324B334A002814BF1846104644
:103AE000CDE900902B46304A0AE02046FFF7F7F96F
:103AF00081462046FFF72FFA2B46CDE900902B4A4E
:103B00003946304614F0F6F805463AE0612D204675
:103B10000DD1FFF7E4F905462046FFF729FA2B46B9
:103B2000234A00903946304614F0E4F8ECE7FFF7FA
:103B3000D6F981462046FFF71BFAD1E72046FFF76A
:103B4000CEF92B4600901B4A3946304614F0D2F885
:103B5000DFF868902146054603A8FFF7D2F9DDE9B2
:103B6000034AA2450AD0AF4214F8013B06D9791B9B
:103B700070194A4614F0BEF80235F2E703A8FFF7C1
:103B800045FFC8F8005091E72046FFF7A8F92B46FB
:103B90000090094AC6E700BFCCF5010800A3010860
:103BA000B1A00108B6A0010870A2010878A201081E
:103BB00081A2010888A201088EA20108C5D60108C9
:103BC0002DE9F0430E4607469046D1B04FF49C7263
:103BD000002102A81D46589C13F01DFA31463B46B1
:103BE000424602A8FFF7E2FD3678642E5AD01CD870
:103BF0003F2E44D008D82E2E4BD09DF808106A488E
:103C000005F06EFE694A48E0612E00F09380622E56
:103C1000F3D1674805F064FE664805F061FE4FF495
:103C200093716548FFF7C2F830E0722E45D00CD88A
:103C3000672EE2D105A9614805F052FE33464F9A3E
:103C400021462846FFF71AFF20E0732E50D0772E2A
:103C5000D3D15B4805F044FE0399002900F0A18010
:103C6000584814F09BF80446002840F09A805648C3
:103C700005F036FE2146384600F0C2FECCE7534838
:103C800005F02EFE21462846FFF7E6FD51B0BDE8BF
:103C9000F0834F4805F024FE4E4A21462846FFF7A0
:103CA00029FDF3E703994C4805F01AFE02AB3A46AA
:103CB00021462846FFF7EAFDE8E705A9474805F051
:103CC0000FFE0399464814F069F820B9384600F011
:103CD00027F9444AE1E74F993846FFF71BFD08B141
:103CE000414ADAE74F9808B1FFF782FB7223A6E753
:103CF00005A93E480DAA05F0F3FD4F993846FFF798
:103D000009FD0028ECD14F9810B10DA9FFF7AAFCCE
:103D100073234F9A21462846FFF7B0FE21683448A6
:103D200005F0DEFD2868216805F040FE314805F009
:103D3000D7FDABE70DF134092F484A4605A905F038
:103D4000CFFD4F9830B3FFF7CCF8032801D02B4AB2
:103D5000A3E74F98FFF70CF914F032F808F10106C9
:103D600006442749304604F0E3FE074690B14F98D9
:103D7000FFF7FEF8234A03463146CDF80090384657
:103D800013F0B8FF39464F98FFF76CFC0121384615
:103D900004F0D2FE61234F9A21462846FFF7DCFC4F
:103DA000BCE7012167E700BF47A4010869A4010837
:103DB000D9A301087AA40108A6A4010844A3010814
:103DC000FCA3010824A401082AA4010821A30108D6
:103DD0002BA3010839A2010835A3010855A3010846
:103DE000E89A010868A301086BA3010885A30108EC
:103DF0009EA3010867A40108AFA30108C8A3010896
:103E0000CCF50108D4A301082DE9F0410C46804609
:103E10000D4815461E46069F05F062FD04B14DB9DA
:103E20000A4805F05DFD39463046BDE8F041084AD4
:103E3000FFF760BC069733462A4621464046BDE858
:103E4000F041FFF7BDBE00BFEFA4010804A50108C3
:103E500017A501087FB504460D4600680C491646B3
:103E600000F00AFB78B100F079FC03AB0093324616
:103E7000294602ABFFF7C8FFDDE902122046FFF733
:103E800051FD04B070BD034805F02AFDF9E700BFFD
:103E90007AA30108E1A2010810B10C2104F04CBE84
:103EA000704710B1012104F047BE704730B513468A
:103EB0000D460446AC4207D01BB194E8070083E8E6
:103EC00007000C330C34F5E7184630BD10B5044636
:103ED000C069FFF7E6FF2069FFF7E3FF204610BD4A
:103EE00010B5044638B1FFF7F1FF2046BDE8104099
:103EF000282104F021BE10BD70B50446406AFFF7CA
:103F0000CBFFD4E90656AE4204D02846FFF7DEFFC9
:103F10002835F8E7A06908B1FFF7E2FF204670BD39
:103F2000F8B5054600242826074FD5E906031B1AD5
:103F3000DB107B439C4205D206FB0400FFF758FAD6
:103F40000134F2E7F8BD00BFCDCCCCCCF8B50446C7
:103F5000224805F0C5FC224805F0C2FCD4E9063130
:103F6000994218D0C91A1F4EC91071431E4805F056
:103F7000B7FC00252827D4E906031B1ADB1073437E
:103F80009D4205D207FB0500FEF7FEFF0135F2E773
:103F9000164805F0A5FCD4E90931154EC91A891057
:103FA0007143144805F09CFC00250C27D4E9090353
:103FB0001B1A9B1073439D4205D207FB050000F0BE
:103FC00071FF0135F2E70C4805F08AFC0B4805F05B
:103FD00087FCBDE8F8400A4805F082BC06A6010847
:103FE0000DB40108CDCCCCCC10A6010822A6010846
:103FF000ABAAAAAA5BA6010867A401086BA60108E0
:10400000F39D01082DE9F043002487B00646684679
:10401000CDE90044029404F00DFB684604F0A2FBD5
:104020004FF028082F4F304DD6E906239B1ADB109E
:104030007B439C424ED208FB04F302EB0309D35CA2
:10404000002B43D14846FEF74AFF0146684604F07C
:104050007BFB4846FEF745FF042837D8DFE800F031
:104060003803101A24004846FEF73DFF0146684613
:1040700004F020FB50BBC2212846FEF797FE25E046
:104080004846FEF768FF0146684604F0F9FAE8B9C9
:10409000C621F1E74846FEF76BFF0146684604F08B
:1040A00053FB98B9CA21E7E7494603A8FEF729FF61
:1040B000DDE903126846521A04F01EFB18B9CF213D
:1040C0002846FEF773FE0398FFF7EBFE0134ABE7DB
:1040D000D321D1E7684604F06DFB029807B0BDE834
:1040E000F08300BFCDCCCCCC3EA501082DE9F04338
:1040F00005460E4600244FF028081A4F8DB0D5E92A
:1041000006239B1ADB107B439C4224D208FB042924
:1041100031461822684613F06DFE4846FEF7DFFE72
:10412000182201460DEB020013F064FE684605F00C
:1041300031FD684605F040FD06A805F02BFD06A8F8
:1041400005F03AFD182268460DEB020113F040FE1F
:1041500018B10134D3E74FF0000948460DB0BDE86F
:10416000F08300BFCDCCCCCC2DE9F04F06460F46F6
:1041700000244FF00C09DFF86C808DB0D6E90953AC
:104180005B1B9B1008FB03F39C4224D21822394688
:10419000684613F02FFE182209FB04FB0DEB02000A
:1041A00055F80B1013F026FE684605F0F3FC684640
:1041B00005F002FD06A805F0EDFC06A805F0FCFCE4
:1041C000182268460DEB020105EB0B0A13F000FE06
:1041D00018B10134D2E74FF0000A50460DB0BDE8E7
:1041E000F08F00BFABAAAAAA10B51446FFF77EFF56
:1041F00020B12146BDE81040FFF734BA10BD0000E1
:10420000F8B50C46064640F201120021224812F091
:1042100002FF4FF4807221461F4812F0D8FE1E495B
:104220001E4805F05DFB1E491B4813F013FE1C4998
:104230000546002013F00EFE294607463046FFF7DC
:1042400055FFA0B929463046FFF78EFF044600B35C
:104250000168144805F044FBA368384698470124D8
:104260002046F8BD3946104805F03AFBF8E73A46D3
:1042700029463046FFF7B8FF04460028F2D00B4825
:1042800005F02EFB0A4805F02BFB3046FFF75EFEDB
:10429000E6E729460748E7E7AC460020FADA0108D6
:1042A0008CA2010884A60108ADA6010899A6010800
:1042B00067A40108C6A6010810B54FF48072044631
:1042C0000649043004F0FAFA002805DD2046BDE86E
:1042D00010400249FFF794BF10BD00BFAC4500205D
:1042E00038B514461D46FFF701FF28B12A4621467E
:1042F000BDE83840FEF7AEBF38BD10B51446FFF735
:10430000F5FE20B12146BDE81040FFF7E9B810BD29
:1043100010B51446FFF7EAFE10B12146FFF708F882
:10432000002010BD38B514461D46FFF7DFFE28B14A
:104330002A462146BDE83840FFF7ACB938BD000039
:104340002DE9F04700248CB0074603A8CDE90344CB
:10435000059404F06FF9214603A8009404F086FA4E
:104360000146002834D0214603A804F008FA40F2A0
:10437000E7330446009300263546DFF8F890009BAB
:10438000B34273D9214603A804F02BFA82460028D1
:104390006CD1182321460DEB030203A804F0B2F9F7
:1043A0000444214603A804F02AFA8046B0B10CAABE
:1043B000214642F828AD03A804F042F9029A0444C9
:1043C00006A93846FFF799FF00B101350136D6E757
:1043D0006A4603A804F0DAF90446CCE7214603A8AC
:1043E00004F057FA70B10CAA02F8288D214603A8F0
:1043F00004F050F99DF80820044406A93846FFF758
:1044000087FFE1E7214603A804F014FA804668B16B
:1044100002AB01AA214603A804F085F9DDE90123D6
:10442000044406A93846FFF75BFFCDE7214603A801
:1044300004F0F2F990B10CAB43F8288D01AA2146A3
:1044400003A8CDF8048004F046F99DF80830044430
:10445000019A06A93846FFF765FFB5E7039B484672
:10446000195D01F0E00105F03BFAAFE728460CB01A
:10447000BDE8F08795A5010808B5FFF737FE18B12C
:10448000BDE80840FEF72FBD08BD10B5044608463C
:104490001146FFF72BFE014620B9C4E90000A060D9
:1044A000204610BD2046FEF72CFDF9E708B5FFF7C2
:1044B0001DFE18B1BDE80840FEF74DBD08BD08B5AA
:1044C000FFF714FE18B1BDE80840FEF751BD08BD66
:1044D000037810B5044643B1044805F001FA002101
:1044E000204600F08DFA0023237010BD80A501083E
:1044F000002370B5D1E90025AD1A0446C0E90033A8
:1045000083600E46284601D005F086FAC4E9000013
:104510000544A560D6E90053024629468B4205D0E2
:104520000AB10E78167001310132F7E75B1B1844AF
:104530006060204670BD38B504460D460B781030DB
:1045400000F8103C4B68103140F80C3C51F8083C26
:1045500040F8083C51F8043C40F8043CFFF7C8FF21
:1045600005F11C0104F11C00FFF7C2FF204638BD15
:104570002DE9F843D0E90054641B9146A2101F4C6A
:1045800006465443B4F5705F0F4602D11C4804F050
:1045900095FA002C14BF22460122A418A1EB0505B0
:1045A00026D2B4F5705F23D82CB30C20604305F0FD
:1045B00033FA804618EB05031CBF99E8070083E82F
:1045C0000700424639463068FFF770FC716800F119
:1045D0000C023846FFF76AFC05463068FFF75CFCC2
:1045E0000C2303FB0484C6E90085B460BDE8F883AE
:1045F0004FF47054D9E7A046DCE700BFABAAAAAAE3
:104600006FA001082DE9F043054685B008460C4629
:1046100017461E4613F0D4FB172803D982212D48D4
:10462000FEF7C4FBCDE90147D5E9097803962A4A8C
:10463000A8EB0706B41054430134B4F5705F02D9F7
:10464000264804F03BFAEB6ADB1B9B1053439C4269
:1046500015D94FF00C0909FB04F91CB1484605F0C7
:10466000DBF90446224641463846FFF71FFC686ADC
:10467000FFF712FC26446C624C44AE62EC62EA6ABC
:10468000D5E9090314491B1A9B10121A4B439210C7
:104690004A430133934206D9114805F021F98C2190
:1046A0000C48FEF783FBD5E90A3293420AD023B1C6
:1046B00004AA12E9070083E807000C33AB6205B0D7
:1046C000BDE8F08301AA194605F12400FFF750FF69
:1046D000F5E700BF3EA50108ABAAAAAA34A00108CD
:1046E00023A50108002310B504460370C0E9063372
:1046F000C0E90833C0E90A33C0E90C33064B802116
:104700004361043004F0D3F82046044B044A0549C1
:10471000FFF778FF204610BD2C45002061470008B8
:10472000E9A60108F5A6010810B5084C2368DB07C7
:1047300009D40748FFF7D6FF0123064A0649044873
:10474000236010F0F5FF024810BD00BF284500208F
:10475000B047002000000020F93E0008FFF7E4BF4A
:1047600008B5FFF7E1FFBDE80840FFF7EFBB002207
:10477000C0E90022826010B50C6804600A604268DB
:104780004C6844604A6082688C6884608A6010BDAE
:1047900070B50E4605461446B54217D09CB12B782D
:1047A00005F1100123706B6804F110006360AB68C1
:1047B000A360EB68E360FFF7DAFF05F11C0104F189
:1047C0001C00FFF7D4FF28342835E5E7204670BDEC
:1047D0002DE9F843D0E90064A41BE310234C0546FF
:1047E0005C43B4F5705F0F46914602D1204804F057
:1047F00065F9002C14BF23460123E418A1EB06063B
:1048000023D2B4F5705F20D814B32820604305F09C
:1048100003F9804618EB060002D04946FFF78BFEED
:10482000394642462868FFF7B3FF696800F128025D
:104830003846FFF7ADFFD5E900690746B14509D015
:104840003046FFF743FB2836F8E74FF47054DCE7B7
:10485000A046DFE7286808B1FFF742FB282303FBE7
:104860000484C5E90087AC60BDE8F883CDCCCCCC2E
:104870006FA001082DE9F047D0E9065704460E461F
:10488000DFF80C818AB0AF421BD029466846FFF79B
:1048900052FE6846FEF723FB81463046FEF71FFBBB
:1048A0000146484605F0B7F930B13046FEF717FB30
:1048B0000146404605F014F86846FFF707FB283527
:1048C000E1E7D4E906892E4AA9EB0807FD10554314
:1048D0000135B5F5705F02D92A4804F0EFF8236A74
:1048E000A3EB0803DB1053439D4220D94FF0280A65
:1048F0000AFB05FA1DB1504605F08EF805464946FB
:1049000040462A46FFF744FFD4E90689C14505D051
:104910004046FFF7DBFA08F12808F7E7A06908B17D
:10492000FFF7DEFA2F44A5615544E7612562226A4C
:10493000D4E9060312491B1ADB10121A4B43D2109A
:104940004A430133934206D90F4804F0C9FF772147
:104950000E48FEF72BFAD4E90703984209D010B1AC
:104960003146FFF7E8FDE3692833E3610AB0BDE8AB
:10497000F0870146324604F11800FFF729FFF5E7FA
:10498000CDCCCCCC34A00108E7A501083EA5010898
:10499000B5A50108002313B502A941F8043D094B50
:1049A0000422D3E90140084B20445B689847044641
:1049B00028B1064804F094FF204602B010BD044818
:1049C000F8E700BFFC470020EC4700205BA9010886
:1049D0006FA9010808B5084804F082FFFFF7A4FE9C
:1049E000FFF79EFA054804F07BFFFFF79DFEBDE848
:1049F0000840FFF7ABBA00BF8CA90108A4A90108C1
:104A000073B505464FF400700C4605F005F80646F0
:104A100030B9214804F064FF20212048FEF7C6F990
:104A20004FF400720021304612F0F5FA3146284664
:104A30004FF40072FFF7E6FA194D014601902CB3CE
:104A4000184804F04DFFD5E901431C44164DEB68AE
:104A50001BB101992046083198476B680422104920
:104A60002046984704226B680DEB0201A018984776
:104A70006B68019A314604F1080098470B4804F02E
:104A80002FFF304604F0B2FF02B070BD084804F0BA
:104A900027FF6C68DAE700BFF2A70108FDA701084D
:104AA000FC4700204DA80108EC47002087A801081A
:104AB0006CA801082DE9F74FFFF736FE2F4F064689
:104AC0002F4804F00DFFB846DFF8D090DFF8D0A0F3
:104AD000FCF73EFA2B4D38602B68AB462A4C002B76
:104AE00037D003F56A436033984232D223782BB92A
:104AF000264804F0F5FE264804F0F2FE0123304675
:104B00002370FFF7D9FB41F2883352464FF0FF3153
:104B10000020FCF775FE0190FCF71AFA019BC8F81B
:104B2000000023B9237813B13046FFF7C5FBDAF84C
:104B30000030DA0744BFD8F800202A609B07C7D5A9
:104B40000023CBF80030D9F80830002BBED09847AE
:104B5000BCE723786BB100213046FFF751FF0D48C9
:104B600004F0BEFE0C4804F0BBFED9F8083003B1D7
:104B70009847002323702B60C5E700BF144800202E
:104B8000CBA801081048002008480020E0A8010830
:104B900003A9010826A9010838A90108EC4700204B
:104BA0000C48002010B5FFF7BFFD04460021FFF7B9
:104BB00027FF2046FFF7CAF9BDE81040034800234D
:104BC000012202210068FCF75FBE00BFE847002019
:104BD00010B5FFF7A9FD04460021FFF711FF20469D
:104BE000BDE81040FFF7B2B92DE9F743194E07466B
:104BF000884675680AB1B3681D440024DFF86090E8
:104C000002A941F8084D0422D9F8003028469847F7
:104C1000326800998A4204D00F4804F061FE2046B1
:104C200014E00422D9F800300DEB0201A8189847CF
:104C300001990A4804F054FE019A4245EFD8D9F888
:104C40000030394605F108009847019803B0BDE8E7
:104C5000F08300BFFC47002096A80108B1A8010816
:104C6000EC470020F0B589B002AC84E80F00039B4C
:104C700023B940F221117648FEF798F8029B23B938
:104C80004FF491717248FEF791F894E80F00714D5E
:104C9000714C85E80F000EAB93E8070084E807002D
:104CA00012B94FF48063A360236823B940F22D1139
:104CB0006748FEF77BF82368013304D140F22F11D7
:104CC0006348FEF773F8FFF72FFD0646634B644A0F
:104CD0006449FFF797FC644B644A65493046FFF727
:104CE00091FC644B644A65493046FFF78BFC4FF4F6
:104CF000007004F091FE0746002870D04FF4007257
:104D0000002112F088F9D4E901032D68042207A9D3
:104D10001844A847002856D02268079B9A4252D1CF
:104D2000574804F0DDFD01224FF400713846FFF7CB
:104D30005BFF0446534804F0D3FDFFF72BFE002C25
:104D40003DD001233370224639463046FFF7F8FA4A
:104D5000384604F04BFE3478FCB94FF4007004F090
:104D60005BFE05464FF40072214612F054F92246CC
:104D70004FF400712846FFF737FF074600283CD163
:104D800004F034FE284604F031FE3F4804F0A8FD4C
:104D9000FFF7CAFC0021FFF733FE3C4BFA220193D8
:104DA00001233B4900933B480023FBF7AFFE20B9AA
:104DB0004FF4A4712648FDF7F9FF09B0F0BD36485D
:104DC00004F08EFD347000224FF400713846FFF776
:104DD0000BFF04460028B6D1384604F007FE2F48E2
:104DE00004F07EFD3046FFF79BF800233370FFF799
:104DF000D1FD2B4804F074FDADE74FF4007004F0D2
:104E00000BFE044618B987211148FDF7CFFF4FF478
:104E100000720021204612F0FEF84FF40072214685
:104E20003046FFF7EFF808B92046A9E78742FBD1E3
:104E30000023E15CEA5C9142F6D101339F42F8D154
:104E4000204604F0D3FD284604F0D0FDA5E700BFBE
:104E5000FDA70108EC470020FC470020D14B0008CB
:104E6000F9A6010805A70108D54900080AA7010805
:104E700025A70108A54B00082DA7010845A7010893
:104E80004AA701086EA70108D0A70108E84700203B
:104E9000E7A70108B54A000883A70108ACA70108E5
:104EA000A4A9010810B504460168074804F018FDDC
:104EB000616831B10B7823B10448BDE8104004F0BB
:104EC0000FBD0348F9E700BFBCA90108F2A0010823
:104ED00067A4010810B50446C06908B104F086FD56
:104EE000206908B104F082FD606808B104F07EFD1D
:104EF000204610BD10B504460068FDF7EBFE2046C5
:104F000010BD00001FB50B4654680178029412785A
:104F100001925A68009242681B68024804F0E0FC63
:104F200004B010BDC1A90108C9210148FDF73EBF69
:104F3000DFA90108FE2307B502A901F8043D054BCE
:104F40001868002300681A46FDF7B4FB03B05DF84B
:104F500004FB00BF24480020D0B51F467423C0E9DD
:104F600000310023044683600820164603F0C4FD88
:104F7000C0E90067A0602046D0BD00002DE9D04305
:104F8000DDE9066799467223C0E9003100239642A5
:104F9000836077EB09030446904603DA2B21074828
:104FA000FDF704FF102003F0A7FDC0E90089C0E968
:104FB0000267A0602046BDE8D08300BF29AA01088F
:104FC000036837B5632B04460D4601D0FFF7ACFFED
:104FD000002302AA42F8043DA168284604F066FABC
:104FE000019B1BB138210248FDF7E0FE03B030BD44
:104FF00029AA010870B563230025C0E900310446E1
:1050000085601A20164603F077FD1A22294612F011
:1050100002F83146A0602046FFF7D2FF204670BD5F
:1050200081647047C16470472DE9F843D0E901738A
:10503000884600254FF00C09DB1B0A4E9B105E438F
:10504000ECB2B4420BD209FB04724146506812F034
:10505000A5FE01350028F3D12046BDE8F8834FF0C6
:10506000FF30FAE7ABAAAAAA2DE9F843D0E9047306
:10507000884600254FF00C09DB1B0A4E9B105E434F
:10508000ECB2B4420BD209FB04724146506812F0F4
:1050900085FE01350028F3D12046BDE8F8834FF0A6
:1050A000FF30FAE7ABAAAAAA2DE9F0410E464968FB
:1050B0000446FFF7B9FFC0B2FF2803D07C2129487E
:1050C000FDF774FED4E90123274F9B1A9B107B4305
:1050D0007E2B03D97F212348FDF768FED4E9011216
:1050E0000C25E068531A9B10121A7B4392107A43E6
:1050F0000133934205FB03F80ED84144A160D4E983
:10510000013496E80700E31A04E9070016489B10EB
:1051100058430138BDE8F081404604F07DFC054667
:1051200018B969211148FDF741FED4E901C30027F0
:10513000A3EB0C039A100C4B5343002B09DD05EB3A
:10514000070E0CEB070207CA013B8EE807000C377D
:10515000F3E7604604F04AFC65604544C4E9025543
:10516000CDE700BF29AA0108ABAAAAAA40AB010853
:105170001FB56E23CDE90131002301A90393FFF789
:1051800093FF05B05DF804FBFF2270B5002380F8A3
:1051900028204FF000424FF0FF31C0E90D23C263D9
:1051A0006FF07F42C0E910120522254DC0E914239B
:1051B0002A68044612F00102C0E90033C0E9023354
:1051C000C0E90433C0E90633C0E908330363C0E92A
:1051D000123313D101211B4E084632607160FDF776
:1051E0008FF9306018B912211748FDF7DFFD012350
:1051F000164A174913482B6010F09AFA154B1A6893
:105200000AB9104A1A6014492046FFF7B1FF134B40
:10521000134918702046FFF7ABFF124B1249187064
:105220002046FFF7A5FF114B114918702046FFF7E4
:105230009FFFFE220F4B18700F4B20461A7070BD57
:10524000204800209848002080AB01080000002082
:10525000F54E000824480020C2AB01082C4800206D
:10526000CAAB01082A480020D2AB01082848002018
:10527000D7AB01082B4800202948002010B5084C66
:105280002368DB0709D40748FFF77EFF0123064A9E
:1052900006490448236010F04BFA024810BD00BFD5
:1052A0001C4800204048002000000020D54E000887
:1052B0002DE9F0410E4649680446FFF7D5FEC0B21D
:1052C000FF2803D087212948FDF770FDD4E9042386
:1052D000274F9B1A9B107B437E2B03D98A2123489F
:1052E000FDF764FDD4E904120C25A069531A9B1044
:1052F000121A7B4392107A430133934205FB03F861
:105300000ED841446161D4E9043496E80700E31AF9
:1053100004E9070016489B1058430138BDE8F081A6
:10532000404604F079FB054618B969211148FDF79C
:105330003DFDD4E904C30027A3EB0C039A100C4BEA
:105340005343002B09DD05EB070E0CEB070207CAE0
:10535000013B8EE807000C37F3E7604604F046FB9C
:1053600025614544C4E90555CDE700BF29AA0108D8
:10537000ABAAAAAA40AB010838B5D0E901239B1A11
:10538000074A9B105343CDB29D42044603D3A62146
:105390000448FDF70BFD0C20636800FB053038BDA9
:1053A000ABAAAAAA29AA010838B5CCB21149054668
:1053B0000B6813F0010307D10F4A70201372012309
:1053C00010600E480B605060FF2C10D0D5E904230C
:1053D0009B1A0B4A9B1053439C4203D3B2210948AA
:1053E000FDF7E4FC0C23286903FB040038BD0248E8
:1053F000FCE700BF184800203048002073AA0108CD
:10540000ABAAAAAA29AA010810B5D0E90730C9B2E7
:10541000D2B2834209D01C788C4204D15C78944289
:1054200001D1987810BD0333F3E74FF0FF30F9E76F
:105430002DE9F041D0E904239B1A4F4A9B105343B6
:105440000D4609780446994203D393214B48FDF752
:10545000ADFCD4E901239B1A474A9B10534369785A
:10546000994203D394214548FDF7A0FCD4E90423D5
:105470009B1A414A9B105343A978994205D3FE29B0
:1054800003D095213D48FDF791FC6A7829782046A4
:10549000FFF7BAFFC3B2FF2B064629D02978204672
:1054A000FFF782FF697807462046FFF765FF314620
:1054B00080462046FFF778FF414602463846FFF710
:1054C00021FD29782046FFF76FFF697806462046C0
:1054D000FFF752FFA97807462046FFF765FF3946D8
:1054E00002463046FFF70EFD9C212448FDF75EFC86
:1054F000D4E90723204F9B1A7B437E2B03D99F219E
:105500001E48FDF753FCD4E90762616A931B7B4395
:10551000521A57430133BB4203EB43080AD84644AF
:1055200026622A88236A23F8032CAA7803F8012C20
:10553000BDE8F081404604F06FFA064618B96921CB
:105540000F48FDF733FCD4E90702131A0A4A5A43FD
:105550000023002A0ADDC118B1F800C0F71826F8A8
:1055600003C08978013AB9700333F2E704F03EFAD8
:10557000E66146446662D3E7ABAAAAAA29AA010853
:1055800040AB010813B5FF24084A02AB106803F8CA
:10559000044D0A4600681946FDF730F9012814BF8A
:1055A00020469DF8040002B010BD00BF2448002032
:1055B00038B5816800681D46144604F0DEFA0346DB
:1055C000201845EBE37138BD08682DE9F0417228D9
:1055D0001F461FD074280FD0632820D1886804F09C
:1055E00025F8002871F1000304460D460EDADD218E
:1055F0000D48FDF7DBFB09E08B68D3E90045B5F109
:10560000004F08BF002C01D0A4187D412046294638
:10561000BDE8F0818868BDE8F041FFF7C9BF00240C
:105620004FF00045F2E700BF29AA01082DE9F0413B
:105630000F4606460024FFB2FFF7B6FED6E907582C
:10564000454511D02B78BB420CD169783046FFF725
:1056500093FE0368692B05D183681B6803B19847E3
:105660000134E4B20335EBE72046BDE8F0812DE9D3
:10567000F34180460F460025FFF796FED8F81C4000
:10568000D8F8206003340336FFB2A6421BD023466D
:1056900033F8032D9B78ADF804208DF8063014F80C
:1056A000033C9F420DD19DF805104046FFF764FE74
:1056B0000368692B05D183685B6803B1984701359E
:1056C000EDB20334E1E7284602B0BDE8F081000006
:1056D000836C73B504460D46164623B94FF48C719E
:1056E0000B48FDF763FBCDE9006423462A460949D0
:1056F0000948FBF70BFA012807D04FF48F710448D3
:1057000002B0BDE87040FDF751BB02B070BD00BFF4
:1057100029AA010835AB0108695C000838B590F882
:1057200047300446032B0D4604D940F23111064898
:10573000FDF73CFB94F847305A1C84F847201C4482
:1057400084F8425038BD00BF29AA010810B590F86E
:105750004730044623B94FF49B710648FDF726FBFA
:1057600094F84730013BDBB284F847301C4494F88E
:10577000420010BD29AA0108CBB2FE2B10B5044689
:105780000AD0FFF711FE03686D2B05D1017A204680
:10579000BDE81040FFF708BE10BD00002DE9F8433A
:1057A00004460026114FD4E904239B1A9B107B4327
:1057B0005FFA86F8434516D941462046FFF7DCFFDD
:1057C000D4E90759A9450CD02B78434507D169780E
:1057D0002046FFF7D1FDA9782046FFF7CDFF03351E
:1057E000F0E70136DFE7BDE8F88300BFABAAAAAA5D
:1057F00038B50546002495F84730A34207DD2B193C
:1058000093F842102846FFF7CFFD0134F3E738BD87
:1058100000232DE9F74FC0E9043388461946D8E93B
:1058200007594FF000430446C0E90213C0E90013D2
:10583000FF208A469B46D2B2207401924D45D4E99E
:1058400000671FD02B78019A934219D1697840469E
:10585000FFF792FDDDE90C2301464046FFF7B4FE59
:10586000594508BF50450BD05F4508BF564503D08A
:10587000B04271EB070303DA6B78C4E900012374CB
:105880000335DBE7B7F1004F08BF002E08D0DDE994
:105890000C23B21A67EB030316461F46C4E90267DE
:1058A000204603B0BDE8F08FF8B50D460B4B896874
:1058B00006464B434FF47A71B3FBF1F1FFF762FEFA
:1058C0000446C7B2B06C03681B689847FF2FC6E94F
:1058D0000E010CBF287C2046F8BD00BF40420F00DF
:1058E00038B5C36C04460D461BB9BDE83840FFF718
:1058F000DBBF806C134903685B699847A06C036841
:10590000DB689847A06C03689968D5E9002388474D
:10591000A06C03681B699847E36C9847A06C036808
:10592000DB689847A06C03681B689847C4E90E01C0
:1059300000212046FFF726FEC0B2FE2808BF287CC3
:1059400038BD00BF354F0008F8B5D1E90067B7F1A1
:10595000004F08BF002E05460C4608D11AB1BDE81D
:10596000F840FFF7A1BFBDE8F840FFF7B9BFD1E9A4
:105970000267012E77F1000301DA087CF8BD8AB1D5
:1059800021462846FFF790FF237CC0B28342F5D121
:10599000D5E90E67D4E90023964277EB0303B8BF3D
:1059A000FF20EBE7D0E91423964277EB0303E7DB14
:1059B000FFF796FFE8E700002DE9F04389B00446C1
:1059C0000D46FFF7F1FC03680646702B04D04FF438
:1059D0009E713C48FDF7EAF9A06C03681B68984784
:1059E0002A46C4E90C01CDE90001214602A8FFF7CF
:1059F0000FFF29462046FFF719FE9DF8183007468D
:105A0000FF2B05D120B940F247112E48FDF7CEF902
:105A1000D4E90C0103F0E4FE01462B4803F060FFDB
:105A200039462A4803F05CFF9DF81810FF2920D161
:105A300000224FF00043CDE90423254F327A02A91A
:105A40002046FFF781FFC3B2FF2B804632D1D4E955
:105A50000E23DDE90201801A61EB030189468046CD
:105A6000CDE9048903F0D2FE0146384603F038FF41
:105A7000E4E72046FFF780FCD0E90078DDE9020189
:105A800003F0AEFE424603463946124803F028FFB3
:105A9000D4E90C23DDE90201801A61EB0301884699
:105AA0000746CDE9047803F0B1FE01460A4803F049
:105AB00017FFC2E729462046FFF7D9FD404609B047
:105AC000BDE8F08329AA010881AA0108A0AA01085B
:105AD000FDAA0108BBAA0108DFAA010870B50446A7
:105AE0000D46FFF761FC03686D2B11D0702B09D0B8
:105AF000612B14D1836894F8411094F84000BDE8FC
:105B00007040184729462046BDE87040FFF754BF53
:105B1000034840F22B11FDF749F94FF0FF3070BDFB
:105B200029AA01082DE9F04790F828300446FF2BF8
:105B300004D14FF4D6714848FDF738F994F828108D
:105B40002046FFF731FC94F82830DFF8188184F8FC
:105B5000463094F846102046FFF726FC03680546B9
:105B60006D2B204694F846100BD1FFF7D7FD297A0C
:105B7000204684F84610FFF717FC2046FFF738FE52
:105B8000E7E7FFF7ABFFC3B2FF2B06460BD140F2AE
:105B9000C1113148FDF70AF940F2C1112F4B304ACB
:105BA0002D4811F0C1F8024694F846102046FFF740
:105BB0002BFCC5B2FF2D09D140F2C7112648FDF7D5
:105BC000F5F8264B264A40F2C711E9E794F846104B
:105BD000FE2D204621D1FFF7B9FD0746014620469C
:105BE000FFF7E2FB324639462046FFF70DFCC5B20F
:105BF000FF2D0DD131462046FFF7BEFB40F2D311F9
:105C00001548FDF7D3F8154B154A40F2D311C7E7F5
:105C10002046FFF7EDFD3946DAE7FFF7C5FB3146D1
:105C200007462046FFF7A8FB294681462046FFF796
:105C3000BBFB8246404603F053FE52464946384677
:105C4000FFF760F994F8463084F8416084F84030FA
:105C500084F846507DE700BF29AA0108B6A00108D4
:105C6000DFAB010825AB010808B5FFF707FBFFF71D
:105C700059FFD0B51F461646FFF77EFB03688468C0
:105C8000742B01D0FFF750F9C4E90067D0BD0000C4
:105C9000836C10B5044623B94FF41F710248FDF719
:105CA00085F8A06C10BD00BF29AA0108FF23054A92
:105CB0001370054A1370054A1370054A1370054A9C
:105CC000137070472C4800202A48002028480020E4
:105CD0002B48002029480020014B1878704700BF4E
:105CE0002848002010B504460068FCF7F3FF204662
:105CF00010BD00002DE9FF4805F04EF94FF6FF7189
:105D00002E4A2F4C13888B421CBF01331380FFF7A0
:105D1000B5FAFFF7BDFF03681B689847637806462E
:105D20000F4603BB274BDB88EBB1274AD2E900BC07
:105D3000BCF1004F08BFBBF1000F0FD083457CEBD7
:105D4000010210DA214AB0EB0B0002FB03F261EB17
:105D50000C01D317904271EB030304DB1C4803F0E2
:105D6000BFFD012363700023ADF80C3063782BB1C5
:105D700001238DF80C30144BC3E900672378154CD0
:105D8000BBB1012514488DF80D5003F0A9FD257015
:105D9000124B13481A78134B1978002300930068AC
:105DA000039B05F07BFA30B10F4B187804B0BDE8C7
:105DB000F0882370ECE70D4BF7E700BFE2480020C6
:105DC000C4480020D048002060000020805101001D
:105DD00024AD0108CD4800204DAD0108C748002082
:105DE000C0480020C6480020284800202A4800203B
:105DF0001D4B10B5DB882BB91C4803F071FD1C4B03
:105E0000187810BD1B4BD3E90023B3F1004F08BF36
:105E1000002A01D01848F0E7184C23780133DBB290
:105E2000032B237001D91648E7E7012B0BD90A2170
:105E3000002003F0A2FE134B58434FF47A73B0FBDB
:105E4000F3F0FBF7D7F921780F4803F049FD002361
:105E50000E4A13700E4A13700E4A13600E4A1370E6
:105E6000012353700D4BCBE7D048002062AD0108F1
:105E700028480020580000207EAD0108F848002086
:105E800098AD010840420F00AFAD0108C74800209F
:105E9000C6480020C0480020C44800202B480020ED
:105EA00008B500231A46FCF705FC431E584258412A
:105EB00008BD000007B50B78012B12D005D3022BCB
:105EC00013D00C4803F00CFD08E0002302A941F8B0
:105ED000043D094B1B681868FFF7E2FF03B05DF84B
:105EE00004FB02A94FF0FF33F1E7034B04311B68B9
:105EF000F1E700BF15AE0108B04800201FB57023C0
:105F0000CDE90131002301A98DF80C30FFF7D0F95C
:105F100005B05DF804FB00002DE9F04F4A4B85B059
:105F20001A780446002A40F08B80012747491F70E9
:105F3000FFF71EF9464B474918702046FFF718F93E
:105F4000DFF868A144498AF800002046FFF710F9FD
:105F5000DFF85C910A22002389F800003F4901A87C
:105F6000FEF7FAFF01A92046FFF79EF83C4E3D4997
:105F700030702046FFF7FCF83B4B3C491870204638
:105F8000FFF7F6F83A4B3B4918702046FFF7F0F858
:105F9000394B3A4918702046FFF7EAF8384B394A2E
:105FA000187039492046FAF76DFBDFF808B1374A17
:105FB0008BF8000036492046FAF764FB3549054660
:105FC0002046FFF79BFF70230193334B804601A9C6
:105FD000204602938DF80C70FFF76AF907462F4AA6
:105FE0002B4612789BF800102046FAF756FB4346E2
:105FF0009AF8002029462046FAF74FFB3B4699F8CD
:10600000002029462046FAF748FB2B4632784146C5
:106010002046FAF742FB2B46327839462046FAF7FB
:106020003CFB1F4A2B46127829462046FAF735FBDF
:106030001C4B1D4A1B78127829462046FAF72DFB87
:1060400005B0BDE8F08F00BFF94800206BAF010834
:10605000C848002075AF010880AF01088CAF010867
:10606000A948002099AF0108E1480020A7AF010826
:10607000E0480020B3AF0108E4480020C0AF0108A9
:10608000E5480020F55C0008CEAF0108156F000858
:10609000D8AF0108ECAF0108FFAF01082848002085
:1060A0002B480020294800202C480020CC48002004
:1060B000A8480020CA48002008B504F04BFF18B1DA
:1060C000BDE8084004F068BF08BD000030B50446D4
:1060D00085B00D46FFF720FF6D22064B01A91B7806
:1060E0002046CDE901258DF80C30FFF7E1F805B029
:1060F00030BD00BFCA4800202DE9F84F424B434D48
:106100001A68044612F0010F01BFFF222A70012213
:106110001A602B78FF2B73D1FFF7FEFE3C4A3D49F6
:106120002046FAF7AFFA3C4A28703C492046FAF775
:10613000A9FA3B4F3B4A38703B492046FAF7A2FA8E
:106140003A4E3B4930702046FFF7C0FF394982463E
:106150002046FFF7D3FE384983462046FFF7CEFEA0
:106160008146364A3B78127829782046FAF795FA24
:10617000334ADFF8E0803378127829782046FAF73E
:106180008CFA337898F8002039782046FAF785FAA7
:106190002B7898F8002031782046FAF77EFA294AC1
:1061A0005B46127839782046FAF777FA26493B7829
:1061B0000A7820465946FAF770FA244A4B46127874
:1061C00039782046FAF769FA1F493B780A78204661
:1061D0004946FAF762FA1A4A53461278317820464D
:1061E000FAF75BFA337898F8002051462046FAF720
:1061F00054FA174A2B78127831782046FAF74DFA7C
:106200002878BDE8F88F00BFA4480020FB48002094
:10621000256900080BB101084164000815B10108A7
:10622000C9480020F15D00081FB10108CB480020DB
:1062300029B1010835B1010843B10108C84800205F
:106240002B480020CC480020A94800202A480020E4
:10625000284800202C48002038B504460D46FFF79A
:106260005BFE034A29462046FAF70CFA38BD00BF08
:10627000AD660008344B2DE9F04F1A89002304461F
:1062800089B0CDE900230391002300222F4905A8FE
:10629000FEF774FE05A92046FEF706FF2C4982464C
:1062A0002046FFF72BFE2B4983462046FFF7D4FFFD
:1062B000294A804629492046FAF7E4F9284A054642
:1062C00028492046FAF7DEF90646274FDFF8A8905E
:1062D0003B7899F8002029462046FAF7DEF9234A50
:1062E0005B46294620461278FAF7D7F9204A4346FA
:1062F000294620461278FAF7D0F9334652465946D5
:106300002046FAF7CAF93346524641462046FAF784
:10631000C4F9184A3B78414620461278FAF7BDF98D
:106320003B7899F8002031462046FAF7B6F96D23FC
:106330000593039B05A9204606938DF81C50FEF794
:10634000B7FF09B0BDE8F08FD048002052B1010876
:106350005FB101086FB10108456A000880B101080A
:10636000D95C00088FB1010829480020E4480020CA
:10637000E5480020E1480020284800202DE9FF479B
:1063800090468A461E4A1F490446FAF77BF91E4981
:1063900005462046FFF7B2FD1C4981462046FFF71F
:1063A0005BFF06461A4A4B46294620461278FAF702
:1063B00074F9184A184F3346294620461278FAF7DE
:1063C0006CF93B78424649462046FAF766F93B7835
:1063D000424631462046FAF760F9104A3B78127877
:1063E00031462046FAF759F96D2301A92046CDE937
:1063F000013A8DF80C50FEF75BFF04B0BDE8F08762
:10640000696A0008E0B00108EAB00108FAB00108C2
:10641000E4480020E548002029480020E148002009
:1064200070B50D460446FEF729FF044922462B4667
:10643000BDE870400978FFF71CBC00BFA9480020E8
:10644000F7B55E4C2668A6B9082002F055FB054654
:1064500006600120324668600421FCF751F828608C
:1064600018B912215648FCF7A1FC5648256004F0E3
:10647000B3FD554D554F296855480131296003F04A
:106480002FFA04F089FD3B781BB901233B7004F01F
:10649000B9FD002302A941F8043D23684D4A18685C
:1064A000FCF7ACF9012807D04B4803F019FA4FF478
:1064B000C7714A48FCF77AFC019E731C51D14848C9
:1064C00003F00EFA2B68042B0FD9FEF747F9037877
:1064D0005BB1444803F004FA4FF47A70FAF78AFE8D
:1064E00040F299113D48FCF761FC00233B702B689A
:1064F0001E22013BDBB21E2B28BF1E2302FA03F330
:10650000394A934226D8B3F5616F1E464FF0000713
:1065100022D2B3F5167F77F1000320DA3C2E77F113
:106520000003ACBF1E210A21002003F026FB341813
:1065300047EBE0752946204603F068F901462B48F1
:1065400003F0CEF920462946FFF76AFF284B18785A
:1065500003B0F0BD0027244E4FF41671E4E73C2150
:10656000E2E74EB13146234803F0BAF90198002121
:10657000FFF756FF204BEAE720482E6003F0B0F902
:1065800004F0BAFCFEF77AFEFFF782FB03681B6893
:1065900098471B4BC3E9000123686BB1304604F0F8
:1065A0001BFD256835B12868FCF794FB08212846B7
:1065B00002F0C2FA00232360124BC8E7B048002063
:1065C00080AB0108B55E0008F4480020F0480020C8
:1065D00004AC0108A086010017AC010831AC010829
:1065E00085AC01089CAC010800A30200E9AC0108DD
:1065F0002A480020FFAC0108CC48002014AD010857
:10660000500000202C480020054B1870054B1A70D4
:106610000022054B1960054B1A705A70704700BF75
:10662000C7480020C6480020C0480020C4480020B9
:10663000027901684079FFF7E7BF08B504F026FE4C
:10664000C0B2DE2828BFDE2008BD00004FF47A73F8
:1066500037B5002403FB00F2074802A9056841F89A
:10666000044DB2FBF3F22868FCF7C8F8012814BF08
:106670002046019803B030BDAC4800204FF47A7337
:1066800037B5002403FB00F2074802A9056841F86A
:10669000044DB2FBF3F22868FCF7F2F9012814BFAD
:1066A0002046019803B030BDAC4800202DE9F04FE2
:1066B0008FB0FEF7E3FD4FF00009064690F846B0B4
:1066C000FFF7FAFCDFF8C4A0DFF8C480B06C02ADBD
:1066D000036808AC1B6898475A46CDE9000131466B
:1066E00008A8FFF795F80FCC0FC5DDE9080123686E
:1066F000B1F1004F08BF00282B70DDE90A4516D123
:106700001C4803F0EDF8002501271B4C4FF47A7369
:10671000A4FB030103FB0511FFF7B0FF10B3012237
:10672000164B5A72164B18780FB0BDE8F08F03F075
:1067300057F829460746204603F068F839460246CE
:10674000504603F0CDF8A04579EB050308DA0021A7
:10675000094803F05BF801460A4803F0C1F8D2E7A4
:106760000027D3E71FB1084803F0BAF8AEE79DF859
:106770001800D9E79DAE010880510100B4480020FF
:10678000E1480020D7AE0108F0AE0108B5AE01081F
:106790008551010010B500200021FFF76FFF10B1F7
:1067A000084B187810BD084C2368984720B9074B50
:1067B0001B780BB9064BF4E7637A0BB1054BF0E796
:1067C000054BEEE7E1480020B4480020E6480020F1
:1067D000284800202C4800202B480020022818BF01
:1067E000002004F005BF0000F8B53B4B05461E78BD
:1067F000002E6FD101271F7004F07EF8374928461C
:10680000FDF754FEC31F052B354C42D820710E23D3
:10681000344928466371FDF752FE3349074611F0AB
:10682000BDFA00283AD1E06030492846FDF724FE41
:106830002F4960702846FDF739FEB0F57A7F3AD8C7
:10684000E0802C492846FDF731FE42F21073984251
:1068500036D8208128492846FDF70EFE2749A0702A
:106860002846FDF723FEB0F57A7F2ED260812449B9
:106870002846FDF701FEE07036B1224803F030F8FB
:1068800071212148FCF792FAE068BDE8F840FFF773
:10689000A5BF1E4803F024F83E46B8E71C49384619
:1068A00011F07CFA10B90223E360BDE7194803F048
:1068B00017F80126B8E7184803F012F80126C0E7D8
:1068C000164803F00DF80126C4E7154803F008F850
:1068D0000126CCE7F8BD00BFFA48002013B001083C
:1068E000D04800202CB00108CBB00108D8DB01084B
:1068F0004FB0010876B001087AA301089EB00108E4
:10690000C8B00108CDB0010831AC010816B00108CB
:10691000B7C8010833B0010858B001087FB00108BA
:10692000A9B0010870B5234BC0B21B78984206D1BC
:10693000FDF714FFFDF7CCFD1F4B187870BD1F4D00
:10694000FDF70CFFFFF750FF95F9050006F098FDE5
:1069500004F062FD287906F061FD04F051FD6878CD
:1069600004F030FE164B1A681C4612F0010213D1D7
:106970000421144E084632607160FBF7C1FD30609F
:1069800018B912211048FCF711FA01230F4A1049D7
:106990000C4823600EF0CCFE0E4B1A680AB9094A67
:1069A0001A600D4804F034FEEB780BB10B4BC4E7D2
:1069B0000B4BC2E7CB4800202C480020D0480020D9
:1069C000A0480020E848002080AB0108000000201B
:1069D000E55C0008AC480020996E0008C84800201B
:1069E0002B480020034B93F83230022B0CBF0220BF
:1069F00000207047B800002008B5FFF7F3FF30B95A
:106A000004F0A8FA18B9BDE8084004F075BAFFF719
:106A1000E9FF022806D104F09DFA18B1BDE808404C
:106A200004F0BABA08BD000008B5FFF7DBFF022882
:106A30000CBF024B024B187808BD00BFE548002090
:106A4000E4480020054B1B8913B9054B18787047A3
:106A5000044B5B7A002BF8D1FFF7E6BFD04800204B
:106A600028480020B4480020FFF7DEBF01232DE9AD
:106A7000F348394C002000216372FFF7FFFD10B18D
:106A8000364B18781AE02368984718B9344B1B78AE
:106A9000002B3CD004F0C2FD012871F10003064632
:106AA0000F460EDB2F4802F01BFFFEF7E7FB3246D6
:106AB0003B46217AFFF7DDF8FFF7B6FF02B0BDE8ED
:106AC000F08823689847054688B1274802F008FFF8
:106AD000002364680093ADF80430FFF7AEFD014673
:106AE0006846A0476846FFF7A3FD204BC9E71C4B4B
:106AF0001B7863B11E4802F0F3FE1E4B1B88022B6D
:106B000028D82A4629462846FFF77EFDEDE71A4D8C
:106B10006B89EBB1EB78DBB1FEF7B0FBFFF7B8F8B0
:106B200003681B6898476B89144A154D5A43D5E989
:106B30000067861B61EB0707D317B242BB4107DA38
:106B4000104802F0CDFE40F24A310F48FCF72EF912
:106B5000002363720D4B94E7B4480020E148002005
:106B6000E648002043AE010854AE0108E04800208A
:106B700066AE0108E2480020D048002080510100A4
:106B8000500000207DAE010831AC010828480020EB
:106B90002DE9F04F0446574D87B0C5E90023019118
:106BA00000230A22544903A8FEF7D6F903A9204678
:106BB000FEF77AFA514A8146287251492046F9F780
:106BC00061FD504A054650492046F9F75BFD4F49A3
:106BD00007462046FFF77AFA4D498DF80200204615
:106BE000FFF78CF94B498DF803002046FFF734FB83
:106BF000494982462046FFF73DFB8346474EDFF872
:106C00003881337898F8002039462046F9F745FD59
:106C1000434A3378394620461278F9F73EFD414A17
:106C20005B46394620461278F9F737FD3E492B4638
:106C30000A7820463946F9F730FD394A2B4659463D
:106C400020461278F9F729FD337898F80020594644
:106C50002046F9F722FD337898F80020294620468F
:106C6000F9F71BFD2E4A3378294620461278F9F7AA
:106C700014FD2E4A9DF80230294620461278F9F775
:106C80000CFD29492B460A7820469DF80210F9F799
:106C900004FD274A9DF80330294620461278F9F76B
:106CA000FCFC2B464A469DF803102046F9F7F5FCFC
:106CB000204A5346294620461278F9F7EEFC2B4627
:106CC0004A4651462046F9F7E8FC337898F8002008
:106CD00051462046F9F7E1FC6D230393019B03A97C
:106CE000204604938DF81470FEF7E2FA07B0BDE871
:106CF000F08F00BFB44800209EB101086D6A000803
:106D0000AEB1010895670008BCB10108C9B101081E
:106D100075AF010880AF0108D5B1010829480020EE
:106D2000284800202B4800202C480020E048002064
:106D3000E4480020E5480020E1480020F8B51D4661
:106D400000234171BDF8181004460360C180174646
:106D500002B115B923712046F8BD0749284601F054
:106D6000E7FE064610B920712660F4E72A46394648
:106D700010F02DF92571F7E7CCF5010810B50446A0
:106D8000006808B101F0D6FE204610BD70B5364E41
:106D900086B03268044622B94FF4E6713348FCF7F6
:106DA00005F8002C5DD00022314B1A80D4E91C2359
:106DB00013431FD02F4B1D68FAF7CAF801462E481F
:106DC000A847D4E91C0102F00BFD226F01462B48B5
:106DD00002F086FDD4E91C2303A802F099FCD4E953
:106DE0001C23274903A8C1E900232649C1E9002340
:106DF00008F0D8FCFEF742FAFEF74AFF03681B686A
:106E00009847214B214AC3E90001237AC3F3C00309
:106E10001370637F2BB3237F1BB31D49082001F040
:106E20007DFE054630B16289237F617F0092A26EAC
:106E3000FFF784FF0395A5B1002330681A4603A924
:106E40000068FBF781FB01280BD0124802F048FDD7
:106E5000039C34B12046FFF791FF0821204601F042
:106E60006BFE06B070BD00BFAC48002031AC01081D
:106E7000E2480020B800002006AF010813AF010867
:106E8000580000206000002050000020E64800204C
:106E9000CCF5010840AF010810B50446FFF776FFB6
:106EA00024B12046BDE8104006F072BE10BD0000BF
:106EB00038B542F2107004F095F80446124802F01A
:106EC0000FFDECB12578022D16D160680021FFF787
:106ED000A7FAD4F89800FFF759FF237A2BB10B4893
:106EE00002F0FEFC00220A4B1A70204605F0C4F89E
:106EF000032D06D1284638BD032DEAD10020E5E751
:106F00000125FFF779FDF5E7CAAD0108E8AD0108F5
:106F1000CD480020002310B5144C84F8363004F01E
:106F200019F808B104F038F8FFF7C2FF032815D8A4
:106F3000DFE800F005020A080D4802F0D1FC0D4B15
:106F4000187810BD0C4BFBE7FFF74CFD022809BF7A
:106F500001230A4B84F83630094BF1E7094840F227
:106F6000BB21FBF723FF4FF0FF30EAE7B80000201A
:106F7000FBAD01082C4800202B480020CC48002005
:106F8000A848002031AC0108FF2300210D4A1370EE
:106F90000D4A13700D4A13700D4A13700D4A137089
:106FA0000D4A13700D4A13700D4A13700D4A137079
:106FB0000D4A13700D4A13700D4AC2E90011137285
:106FC000704700BFCA480020C9480020CB480020B5
:106FD000E1480020E0480020E5480020E448002087
:106FE000C8480020CC480020A8480020A94800201C
:106FF000B448002038B50A4C05460121204608F067
:10700000AFF9002320461A46012108F0E7F885F081
:1070100001022046BDE83840012108F0ADB900BFAB
:107020000000024008B50120FFF7E4FFBDE808407A
:10703000032009F0C5B80846FFF7DCBF10B50446C9
:10704000024B036002F0EEFD204610BDE8B10108DE
:1070500010B50446054B503040F8503C044B40F806
:10706000083CFFF7EBFF204610BD00BFC4B5010888
:10707000E4B7010810B50446FFF7E0FF20460821F9
:1070800001F05AFD204610BD10B50446FFF7E0FFA1
:107090002046742101F050FD204610BD024B012115
:1070A000186803681B68184708490020021C18BFAD
:1070B00001220321014808F05FB900BF000402402B
:1070C00010B50C46FAF78EFA022808D14FF47A7000
:1070D0004443B4FBF0F0BDE81040FAF78BB820460B
:1070E000BDE8104007F096BE0321014808F04DB9F5
:1070F0000004024010B5094C094802F0F1FB20469B
:107100000B2108F02DF9002320461A460B2108F028
:1071100065F8BDE8104007F063BE00BF0000024004
:107120005EB5010808B5022007F0BEFD07F020FE9D
:1071300000F046FC07F046FE00F054FE08F0AAFB03
:107140000C48FBF7FDFD4FF4E13008F095FE0A4BCB
:107150001A680AB9094A1A60094B1A680AB9074A33
:107160001A60084802F0BCFBBDE80840064802F07F
:10717000B7BB00BF25700008EC49002019FD0008CE
:10718000F049002058B2010870B20108F7B5044672
:1071900012F0CCFB234600252146204A04F148008A
:1071A00043F83C2BE5635D601D4B1E4E41F8443FA8
:1071B00000F0D8FF1C4B84F85C50A3651B4BC4E95E
:1071C0001A5523661A4B84F870506366194802F00A
:1071D00087FB3368184F01933B68184D00932B6869
:1071E000174A1B2104F1210010F084FD296804F1E5
:1071F000110002F0AAFC396804F1150002F0A5FCA8
:10720000316804F1190002F0A0FC296804F11D00A6
:1072100002F09BFC204603B0F0BD00BFC4B50108DE
:10722000B8B601086400F81F10B7010840B701089C
:107230002CB7010892B501085400F81F5000F81F40
:10724000A7B5010810B5094CFFF76CFF2368DB07F1
:1072500009D40748FFF79AFF0123064A0649044864
:1072600023600EF065FA024810BD00BF00490020FF
:107270000C490020000000205170000838B5064D70
:10728000064C2B6813F0010F04D1FFF7DBFF01233D
:1072900020602B60206838BD044900208049002010
:1072A0004FF4FA7112F06CBB08B50B21054808F0D9
:1072B00071F828B1BDE808400B21024808F07EB8FB
:1072C00008BD00BF0000024008B519B1BDE8084084
:1072D000FFF710BF044802F003FBBDE8084002229C
:1072E0000B21024807F0B8BF7AB501080000024040
:1072F00070B504462F4804F1440502F0F1FA28461F
:10730000002100F097FD0021284600F0A9FD20464D
:1073100012F016FB0CF0E8FE03F0EEFD2046002113
:10732000FFF7D2FF0CF03EF901220C21224807F0B2
:1073300093FF08F0CDFB04F1480000F0F5FE236850
:107340002046DB6804F16405002198471B4E0021AC
:10735000284600F00BFE08F08FF8194802F0C0FA3A
:1073600008F078FC07F02EFD304601220D2107F0D1
:1073700073FF012230460E2107F06EFF0021084600
:1073800008F064FB04F1580000F080FD012128465C
:1073900000F0ECFD4FF4E13008F06EFD094802F01A
:1073A0009FFA0CF025F808F091FB2046BDE87040EC
:1073B00012F0D6BA2CB501080004024000000240C9
:1073C00050B5010876D5010838B50546FFF76CFFC2
:1073D000044628B100212846FFF776FF07F000FD9C
:1073E00007F006FC05460CB1FFF784FE284638BDC1
:1073F00070B50C460646154920460FF08BFA20B9A9
:10740000002120460FF068FA70B1114920460FF0B4
:10741000C5F80FF089FA01460E4802F061FA4FF400
:10742000BB710D48FBF7C2FC3046FFF73DFF054638
:1074300048B93046FFF7C8FF014620460FF06AFA08
:1074400008B1FFF757FE284670BD00BF33335340E5
:1074500000007A4486B20108B5B2010870B52D4A21
:10746000D6B013680546DB0705D42B4900F1640349
:107470000B600123136029492846FFF7B9FF064630
:10748000274802F02DFA002105F1440000F0E8FC45
:10749000244C254BE360254B2361254BA360254BF2
:1074A0006360254B2360254B6361254BA361254B0E
:1074B000E36104F110030FCB8DE80F0094E80F0097
:1074C0000DF0FAF8002305A8EB632B640DF080F8AB
:1074D0009DF8143005F13C04012B14D1DDF8153072
:1074E00005A8EB63DDF819302B640DF041F8164860
:1074F00002F0F6F90821204602F058FABDF91611FB
:10750000124802F0EDF931462846FFF7DDFE56B08D
:1075100070BD00BFFC48002008490020000040402A
:10752000F1B101087C51002015EE00089DED000826
:107530009D700008E9700008AD700008E19800082F
:10754000651F0008A51F000812B2010838B2010823
:1075500008B5FFF739FF03490FF020F80FF00AFADA
:1075600080B208BD00007A4470B507490546FFF7B0
:107570003FFF06460CF0C4FF044631462846FFF79D
:10758000A3FE204670BD00BF000040407FB5F82339
:1075900000F1580504AC0646284604F8013D00F009
:1075A0007BFC0223214600930122A123284600F000
:1075B00077FC4FF400430822009306F16801A123F1
:1075C0000446284600F096FC0440E4B2284600F049
:1075D00065FC204604B070BD30B58BB0044608F0A1
:1075E0001DFE0146554802F07BF9554802F078F936
:1075F000204600F0ADFB04F1580500F0BDFA00F0A4
:1076000067FA5048504902F06BF9284600F03EFCFA
:1076100038B94E4802F064F940F233114C48FBF798
:10762000C5FB07F0DDFB2046FFF7B0FF20B94FF4A4
:107630009C714748FBF7BAFB94F86F0094F86A30E6
:10764000049094F86E0094F86920039094F86D000B
:1076500094F86810029094F86C00019094F86B0014
:1076600000903C4802F03CF9284600F033FA2846E6
:1076700000F094FA04F14405002184F870002846D3
:1076800000F0D8FB012000F07BFD0021284600F02F
:10769000E7FB012000F092FD2046FFF7DFFE00F03F
:1076A000C9FA2D4802F01CF94FF4FA700FF050FCA3
:1076B000054600283AD1294802F012F9284802F07C
:1076C0000FF9284802F00CF9274802F009F9274879
:1076D00002F006F9264802F003F9264802F000F904
:1076E000254802F0FDF8254802F0FAF8244A254919
:1076F000254802F0F5F82549254802F0F1F825481B
:1077000002F0EEF804F12101234802F0E9F807A89D
:1077100008F058F807A802F039F801461F4802F0AF
:10772000DFF8104802F0DCF80BB030BD1C4802F066
:10773000D7F828460FF014FCC0E700BFFDB20108DF
:1077400013B301082AB30108A086010045B301085C
:10775000B5B201085BB3010890B30108C3B30108D7
:1077600066A4010801B4010832B4010841B401085B
:1077700063B4010886B40108AAB4010867A401082B
:1077800036A2010813A20108CDB40108DDB4010836
:10779000E4B40108EFB401080FB501081AB50108F7
:1077A000F7B301082DE9FF4100F15805284600F024
:1077B00073FB04240226284F013C14F0FF0433D04D
:1077C000A123012239460096284600F069FB4FF4B8
:1077D0000043804600930422A12302A9284600F01A
:1077E00089FBB8F1000F01D10028E5D09DF80830E1
:1077F000442B20D19DF809306E2B1CD10DF10A00CD
:1078000002F095F90223013084B221460DF10900FE
:107810008DF8083002F0ACF9002303220093A02376
:1078200002A9284600F03CFB284600F037FB204622
:1078300004B0BDE8F0814FF488430024ADF808306F
:107840006E2300210DF10B008DF80A3002F090F943
:107850000094A0230522E3E7F0B1010838B50C46F7
:107860001131054603F010FA214651F8683F2846C9
:107870002B604B686B6038BD024B186803685B680F
:10788000184700BF90490020024B186803689B68A6
:10789000184700BF904900202DE9FF4100231546FD
:1078A0001370022206460D4F04AC386804F8011D1F
:1078B00003680092D3F80C80012233462146C0476A
:1078C00048B14FF4004238682946036800921C69A9
:1078D00001223346A04704B0BDE8F0819049002062
:1078E00030B585B08DF80D200022074B8DF80C10B7
:1078F0001C6803A923680092DD6802220346204623
:10790000A84705B030BD00BF9049002037B54FF4FF
:107910000045064B1C68236800951D6913460A46FE
:1079200001462046A84703B030BD00BF8C49002067
:1079300037B50025054B1C6823680095DD681346A4
:107940000A4601462046A84703B030BD8C490020B6
:1079500037B50225054B1C6823680095DD68134682
:107960000A4601462046A84703B030BD8C49002096
:10797000024B186803681B68184700BF8C49002039
:10798000024B186803685B68184700BF8C490020E9
:10799000024B186803689B68184700BF8C49002099
:1079A0004FF47A735843B0FBF3F0F9F723BC10B5EA
:1079B0000446FFF763FC2146BDE81040FFF7F2BE26
:1079C00010B5424C0BF040FE20460222002107F089
:1079D00043FC01222046114607F03EFC20460122CE
:1079E000022107F039FC20460222032107F034FC73
:1079F00020460022042107F02FFC20460222082105
:107A000007F02AFC20460122092107F025FC204628
:107A100001220A2107F020FC204602220B2107F058
:107A20001BFC07F0CFF9002320461A460C2107F073
:107A3000D5FB204600220C2107F09EFC20460022A8
:107A400004F580640F2107F007FC20460122002185
:107A500007F002FC20460022022107F0FDFB204631
:107A60000022032107F0F8FB20460222062107F03E
:107A7000F3FB20460022082107F0EEFB20460022FF
:107A8000092107F0E9FB204601220C2107F0E4FB65
:107A9000204602220D2107F0DFFB204602220E21A4
:107AA00007F0DAFB204602220F2107F0D5FB002366
:107AB00004F5806420461A460D2107F08FFB20460E
:107AC000BDE8104000220D2107F056BC0000024026
:107AD00007F0E0BE1D4B00B51A6889B0D2075FBF42
:107AE0001B4A106001221A601A4B1B4A04931B4B5D
:107AF00005931B4B03931B4B02931B4B079308AB44
:107B000043F8082D93E803008DE8030002AB0FCB88
:107B10000CF086FC90B1154801F0E2FE00221448FA
:107B2000114607F099FB0F2302220021104807F0AD
:107B300033FA09B05DF804EB0CF00CBC69210D4878
:107B400009B05DF804EBFBF731B900BF88490020AC
:107B50009049002079780008A17900088978000808
:107B600099780008E1780008E198000856B6010805
:107B70000000024067B60108002307B5ADF80430E5
:107B800001238DF8063001980BF0BAFC07F01AF9C2
:107B900003B05DF804EB0BF005BD0000194B10B508
:107BA0001A688CB0D2075FBF174A106001221A60B2
:107BB000164B0793164B0593164B0693164B0893DB
:107BC000164B0993164B0A93164B0B930CAB13E908
:107BD00007008DE8070005AB0FCB0CF045FB044612
:107BE00001220F21104807F037FB3CB10F4801F08C
:107BF00077FE0CF017FB20460CB010BD0C4801F0CE
:107C00006FFEF8E7844900208C4900200D790008B8
:107C100031790008517900087179000881790008EC
:107C200091790008E198000800000240D8B50108E9
:107C30000BB601082DE9F04FA9B002F02BFCDFF8DC
:107C40000C9168B9384B394ACDE923332292384A2E
:107C50000093CDF88090219220AB0FCB02F020FC56
:107C6000344B00251993344B4FF0010A1893334BD2
:107C70004FF003081A93324B2B4C1B93314B2C4F74
:107C80001C930423294E09A918A8CDE909351D9490
:107C90001E971F968DF829A009F048FF09F03AFFBA
:107CA0000FF0C0FF2946142223A80C95CDF82C8094
:107CB0000FF0B1F9EE460DF1A00C4CF8186DBCE8D0
:107CC0000F00CDE92047AEE80F009CE803008EE8E6
:107CD00003000DF1800B0BA99BE80C0003C90CF00D
:107CE00061F9294610220EA80FF095F9164BCDE93F
:107CF0001244CDF834808DF83EA002AC0DADCDE934
:107D000015761793CDF850900FCD0FC42B682360D4
:107D100016AB93E803008DE8030012AB0FCB02F023
:107D2000DDFF29B0BDE8F08FE1980008ED9900086B
:107D3000199A000829350108F133010801330108B7
:107D400099320108AD320108AF79000881F80008C6
:107D50002DE9F047044606F04BFF1E4905460EF09C
:107D60001DFC0EF0E1FD01461B4801F0B9FD4FF08E
:107D7000804128460EF0B0FD48B30025DFF8609042
:107D8000DFF85080154E06F033FF494607460EF0E7
:107D9000B7FDA8B9414638460EF000FC0EF0C4FD10
:107DA0000146304601F09CFD236885F00105204620
:107DB000DB68294698474FF47A7007F02BF8E2E722
:107DC00023682046BDE8F047DB6800211847BDE87E
:107DD000F08700BF00007A4429B601083BB60108CD
:107DE0000000204008B50D49012007F0A9FB0C490F
:107DF0000B2007F0A5FB0B490A2007F0A1FB0A495D
:107E0000042007F09DFB0949072007F099FBBDE816
:107E100008400749052007F093BB00BF612E010809
:107E20007D3101080930010895320108E931010866
:107E300071320108002310B50C461A460D2107487F
:107E400007F0CCF914B1012C00D010BD2246BDE8DA
:107E500010400D21014807F08FBA00BF0008024012
:107E6000002310B50C461A460C21074807F0B6F956
:107E700014B1012C00D010BD2246BDE810400C21E9
:107E8000014807F079BA00BF00000240014807F03E
:107E9000E1BA00BFA086010007F0ACBA07F0C6BA8D
:107EA0002DE9F041069F1E4607F00303032B804691
:107EB0000C46154603D12F210D48FAF777FF2046CF
:107EC000BC07324629460AD507F0FEFA10B1012058
:107ED000BDE8F0810123002088F80430F8E7FB07B3
:107EE00002D507F0FFFAF1E707F0E0FAEEE700BF8E
:107EF000C0B601082DE9F041069C0D46E107804619
:107F000016461F4603D54C210D48FAF74FFFA2072E
:107F100003D54F210A48FAF749FF23043A46314670
:107F200028460AD507F0ECFA10B10120BDE8F0812F
:107F30000123002088F80430F8E707F0A9FAF3E7F6
:107F4000C0B6010808B50321034807F01EFA003047
:107F500018BF012008BD00BF000402400A460248C5
:107F6000032107F009BA00BF0004024008B581B13F
:107F7000012303211A460A4807F030F90321084873
:107F800007F0EEF9BDE8084003220548114607F066
:107F900005B90122BDE808400321014807F05CB99A
:107FA0000004024007F06CBC1FB501A801F0B0FB53
:107FB00001A807F0F7FB05B05DF804FB1FB501A8A9
:107FC00001F0A6FB01A807F03BFD05B05DF804FB3E
:107FD00007F0A4BC07F0BCBC084607F033BBDFB514
:107FE0000023CDE90133ADF80C3001238DF80730C3
:107FF0008DF808306FF01D038DF809300723044613
:1080000001A88DF80A3001F0A8FB236806461B681A
:1080100020460F469847864277EB0103B4BF012004
:10802000002004B0D0BD7047704700007FB500F15C
:108030000806054630460C4601F01EFE60BB33487C
:1080400001F04EFCA27C617C314801F049FC637C6C
:108050003BB16868002103681B689847022000F064
:108060008FF8A37C3BB16868002103685B68984780
:10807000022000F0A3F861684E2918D04F2916D0CD
:10808000452914D015212348FAF790FE1621224BDA
:10809000224A20480EF048FE6421304601F0D8FD07
:1080A0000028CFD142211B48FAF780FECAE7A26818
:1080B000082A0BD0092A09D0072A07D023211548FE
:1080C000FAF774FE144B164A2421E2E7E3680A2B00
:1080D00010D009DC052B0ED033210E48FAF766FECE
:1080E0000D4B104A3421D4E70F2B04D0142BF3D1BD
:1080F000022300E00123A07C0290607C0190207CA0
:108100000090206807F0F2FE04B070BD5CB7010873
:10811000BDB7010875B70108B6A0010804B8010889
:1081200068B8010834B8010810B5044607F0B0FE7D
:1081300004F10800BDE8104001F0A1BD084607F0B9
:10814000BDBF38B50C468D18AC4204D014F8010BF5
:1081500007F0B4FFF8E738BD07F0C0BE084607F0E7
:10816000DDBF000010B50446044BC0E90031012119
:10817000083001F08FFD204610BD00BFE4B70108B4
:10818000042817D8DFE800F00309100E12000023BE
:1081900003211A46084807F021B8002203210648A7
:1081A00007F05AB80222F9E70122F7E70321024853
:1081B00007F078B8704700BF00000240042817D8C5
:1081C000DFE800F00309100E1200002302211A4616
:1081D000084807F003B800220221064807F03CB81F
:1081E0000222F9E70122F7E70221024807F05AB814
:1081F000704700BF000002402DE9FF4705460024FC
:10820000174E04AF306807F8011D99460368904681
:108210005B68984730686D000368EDB20094D3F84E
:108220000CA039462B460122D047374688B130682A
:108230004A4603680094D3F810A041462B46D04725
:1082400038B1306803689B689847204604B0BDE8A1
:10825000F087386803689B6898476FF00100F5E77E
:108260009849002010B501460446064801F038FB45
:108270004FF47A704443B4FBF0F0BDE81040F8F7D7
:10828000B9BF00BF79B901082DE9F04305461F4683
:108290001A4C8FB020688846036816465B6898477A
:1082A0006D00282FEDB204D94FF48B711448FAF702
:1082B0007DFD314600260DF138093A460DF10D00DD
:1082C00009F82C8D0EF083FE20687A1C0368009656
:1082D000D3F80C8049462B46C04738B12068036864
:1082E0009B68984730460FB0BDE8F083206803686C
:1082F0009B6898476FF00100F5E700BF98490020A0
:108300003BB9010838B504460D460D4801F0E8FABE
:10831000257304F108000CF094FD622305462372D6
:1083200038B9084801F0DCFA012384F8683028469F
:1083300038BD0146044801F0D3FA0023F5E700BF39
:10834000ECB80108F5B8010815B9010807B500F146
:1083500008010DF106000DF00FF8BDF8060003B09E
:108360005DF804FB38B5114B04460364A1B1012349
:1083700080F846300E4B04F10801A3640123DF208E
:1083800084F84C300CF07DFE054640B101460948AA
:1083900001F0A6FA284638BD80F84610EAE72046E4
:1083A000FFF7D4FF01460448F2E700BF02040302CE
:1083B00040019600A0B80108CAB8010870B500F1E4
:1083C0000804054620460E460CF01CFE78B92846E7
:1083D000FFF7BCFF4FF47A735843B0FBF3F0F8F7A4
:1083E00009FF21463046BDE870400CF0F9BF70BD72
:1083F0000023C0E9183380F868300B4BC0E9001245
:108400001A68D2075FBF094A116001221A607623F9
:10841000437201238372064B0365064B4365064B8B
:1084200083651923037370479449002098490020FD
:10843000F98100088982000865820008F0B508B952
:108440000020F0BD002746684D1CB5421760F7D8E4
:1084500003685C185B5C03F01F03A3F11801032998
:108460008FBF38460D49C91811F8180C0544AE42A3
:10847000E6D304280DD8DFE800F00403070C0C0055
:10848000637813600130DCE7B4F801305BBA9BB26B
:10849000F7E7D4F801301BBAF3E700BF96B901083B
:1084A000F7B51F46436816464A1C9A4205460C46D5
:1084B00017D803685B5C03F0C003402B11D196B161
:1084C00001AAFFF7BBFF50B1019A04446B68A118E1
:1084D000994206D8296810440C4434603A6003B0CD
:1084E000F0BD0020FBE73046F9E72DE9F743994658
:1084F000436817464A1C9A4280460D4624D80368B2
:108500005B5C03F0C003402B1ED1FFB101AAFFF753
:1085100095FF0446A0B1019E09F10109B14513D3AD
:108520000544D8F8043072199A420DD8D8F80010D2
:108530003246294438460EF04AFD00233444BB55E8
:10854000204603B0BDE8F0830024F9E73C46F7E796
:10855000F0B5002931D0172A1CD8D3B2A3F11804E2
:10856000032C8CBF0024164C8D689CBFE41814F8B3
:10857000184C6F1C4E6804EB070CB4451DD20E68F6
:1085800018438F60705500200130231A5D1C0BD1F9
:10859000601CF0BDFF2A05D9B2F5803F2CBF1A231D
:1085A0001923DBE71823D9E78E680D68DB00771CF9
:1085B00022FA03F38F60AB55E6E70020E9E700BF3E
:1085C00096B90108172BF8B50D4616461C4612D869
:1085D000DBB2A3F11802032A8FBF0022144A9B18B2
:1085E00013F8182CAB680132234413446A68934291
:1085F0000BD30020F8BDFF2B05D9B3F5803F34BF66
:1086000019231A23E5E71823E3E722462946FFF753
:108610009FFF07460028ECD02868AB683146184415
:108620000EF0D5FCAA68E0192244AA60E2E700BF78
:1086300096B9010818B10023C0E9001283607047A1
:10864000436873B514464A1C9A4206460D4602D941
:10865000002002B070BD03685B5C13F0C00FF7D15F
:10866000002CF5D001AAFFF7E9FE0028F0D032680F
:10867000019B525D12F0E00F18BFDB432360E8E777
:108680000A1EABBF014601460020D243B8BF2020DE
:10869000FFF75EBF03685B5C03F0E001E02907D1F0
:1086A00032B1A3F1F5014B424B41137001207047E9
:1086B00000207047836810B544685A1CA24208D253
:1086C000002914BFF524F424016882600120CC54F1
:1086D00010BD0020FCE7F0B446684F1CB74208D834
:1086E00005686C5C04F0E004402C02D1F0BCFFF79C
:1086F000D7BE0020F0BC704713460A460146402012
:10870000FFF760BFF0B446684F1CB74208D8056851
:108710006C5C04F0E004602C02D1F0BCFFF7E5BE15
:108720000020F0BC7047F0B446684F1CB74208D830
:1087300005686C5C04F0E004602C02D1F0BCFFF72B
:10874000AFBE0020F0BC704770B5054608460C4629
:108750000FF036FB224603462946BDE870406020F4
:10876000FFF730BF836841685A1C8A423FBF82606E
:10877000BF220168012034BFCA540020704703683B
:10878000585CA0F1BF0358425841704713B50368C5
:1087900014465B5C03F0E003A02B07D142B101AAB1
:1087A000FFF74CFE019B236002B010BD0020FBE7E9
:1087B0001046F9E7836841685A1C8A423FBF8260CD
:1087C000FF220168012034BFCA540020704730B135
:1087D0008068013888428CBF00200120704701204A
:1087E000704708B50246FFF7F2FF30B91268505CD7
:1087F000A0F1FF035842584108BD0120FCE743683F
:108800008B4207D903685B5C13F0C00F0CBF0120DB
:10881000002070470020704743688B4208D90368E6
:10882000585C00F0E000A0F1400358425841704706
:108830000020704743688B4208D90368585C00F0F9
:10884000E000A0F160035842584170470020704793
:1088500043688B4208D90368585C00F0E000A0F13F
:10886000A0035842584170470020704710B5044695
:10887000FFF7EEFF50B163688B4208D92368585C5C
:1088800000F01F00A0F11F035842584110BD002006
:10889000FCE743688B4208D90368585C0C30C0B2CF
:1088A00001288CBF00200120704700207047002362
:1088B000C0E9013303690160C3607047F8B503681C
:1088C0000446002B0D46164603DC3E212948FAF7E4
:1088D0006DFA3246002128460EF09DFBD4E9017066
:1088E000B8420CD00021236801EB070C9CFBF3F28B
:1088F00003FB12C2904205D10020884204D14FF000
:10890000FF3031E00131EFE7C21992FBF3FE03FBC8
:108910001E2ED4F80CC01CF80EE0BEF10A0F26D1B2
:1089200028B3013A92FBF3F103FB1122002106F177
:10893000FF3E71450ED2E7686368FB5C6B54676865
:108940002668013797FBF6F306FB1377013188425F
:108950006760EEDA1CF802300D2B4FF0000304D1F3
:10896000054405F8013C0138F8BD2B54FCE7013003
:10897000C3E700BF9AB901084B1C017343738B1CFA
:1089800003318373C17370472DE9F0410746884670
:108990001E4615461AB952211548FAF707FAD7E9C3
:1089A0000143A34221D2E41ADEB1A3B9A5420ED3FA
:1089B0003B7B3370BB6839682246194440460EF051
:1089C00006FBBB682344BB602046BDE8F0817B7B8F
:1089D00033702C46EEE7A54201D3FB7BE9E7BB7B76
:1089E000F6E7AC4228BF2C46E4E70024ECE700BFE2
:1089F000EAB901080023C0E900128360704710B58E
:108A000004460846C4E900120021A16021730EF05B
:108A100002FB204610BD000038B51546D0E9012301
:108A200004465819904202D9257B55B1D51A2068C1
:108A30002A4618440EF0CBFAA3681D44A560012510
:108A400003E01B210248FAF7B1F9284638BD00BF00
:108A50002EBA010807B502AB03F8011D0122194621
:108A6000FFF7DAFF03B05DF804FB00687047806829
:108A7000704713B5044601A801F07AF8022201A953
:108A80002046FFF7C9FF02B010BD13B50446684683
:108A900001F064F8052269462046FFF7BDFF02B0E9
:108AA00010BD13B5044601A801F062F8022201A925
:108AB0002046FFF7B1FF02B010BD000008B5014627
:108AC000044800F00DFFBDE808400C210248FAF709
:108AD0006DB900BF6EBA01088CBA010808B5044828
:108AE00000F0FEFEBDE808401E210248FAF75EB91C
:108AF000F7BA010824BB010810B500F08DFF044649
:108B000030B9044800F0ECFE27210348FAF74EF98B
:108B1000204610BDE5BA010824BB010800F07CBF67
:108B200010B9024800F0DCBE00F060BFD0BA010806
:108B300000F072BFFFF7F4BFFFF7F2BF10B5074CAC
:108B40000A44914200D110BD11F8013B83EA102381
:108B500034F8133083EA002080B2F2E768BB0108E2
:108B6000F8B50E46054680B14F1C384600F054FF5C
:108B7000044640B13A4600210EF04DFA32462946ED
:108B800020460EF024FA2046F8BD0446FBE738B52F
:108B90000D46044628B10FF013F9234620448342C2
:108BA00001D1002038BD13F8012BAA42F7D10120D2
:108BB000F8E737B504460D460EF0E2F8002201A9A9
:108BC000026020460FF028FA04460EF0D9F8036838
:108BD000222B08D0019B1B782BB9002C03DB2046ED
:108BE0002B6003B030BD012300202B60F9E70000AB
:108BF0002DE9F04F05464FF0010B002687B0CDE977
:108C0000031206F10903122B8CBF0320022000F08F
:108C100003FF0090E8B1324636490FF09FF8039BFE
:108C200053F82690EDB90024009800F0DFFEBBF168
:108C3000000F02D1284600F0D9FE84B1049B013612
:108C4000B34225464FF0000BDBD1204607B0BDE80C
:108C5000F08FBBF1000F02D1284600F0C7FE0024C0
:108C6000F3E7254B4FF00008B9F1000F08BF994614
:108C700048460FF0A5F8019000980FF0A1F8029077
:108C8000284649460FF0CBF8B8B928460FF098F8B7
:108C9000DDE9012301309B1A08FB030000F0BCFE54
:108CA00004460028BFD003462F4618F1FF3809D2EA
:108CB000394618460FF07CF8B6E7019B08F1010829
:108CC0001844DEE74946384605930FF0A8F8059B9F
:108CD000A0EB070A5246394618460FF08BF8009968
:108CE00050440FF065F8019A029B9244C318574410
:108CF000DBE700BF41A2010868A4010830B580B1DC
:108D00000346021F00F1180452F8045F8D4208D098
:108D1000A242F9D11C301A4614680433013401D13F
:108D2000116030BD8342F6D1FBE770B5044680B1D7
:108D3000064600EB8105AE4204D12046BDE87040F6
:108D400000F054BE56F8040B0028F4D000F04EFE9C
:108D5000F1E770BD2DE9F74F89460092002838D021
:108D60000027C45D8CBB05468346264600EB070AF8
:108D7000D34538D104B10136002E6FD001373846C3
:108D800000F04AFE8346002866D03A4600210EF0E5
:108D900042F9B00000F040FE0446002860D04FF0D9
:108DA00000084146AA4532D131B15846FFF7D8FEF6
:108DB000002855D044F82800584600F017FE009BC4
:108DC0001E60204603B0BDE8F08F0137B7F5807F05
:108DD000C7D100242646204600243146FFF7A5FFD0
:108DE000009B1C60EDE79BF800304B4505D10CB1B2
:108DF000002401360BF1010BBAE70EF09BF89BF84B
:108E00000030184443781B0758BF0134F2E72B7831
:108E10004B4513D181B15846FFF7A2FE00B308F1CC
:108E2000010344F8280000213A46584601930EF009
:108E3000F2F8019B002198460135B3E701910EF04D
:108E400079F82B7801991844407810F0080F04BF86
:108E50000BF801300131EFE70446BCE73446B0E7D8
:108E6000584600F0C3FDB6E72DE9F7430025064656
:108E70000820884691461F46009500F0CDFD044627
:108E8000002868D0C0E9005530460EF099FF01284F
:108E90000FD133782A2B0CD109F1FF33C4F80080AD
:108EA000636022684A4502D263684B4543D32B4B2B
:108EB0000EE02D213046FFF76AFE0546C0B902A933
:108EC00041F8040D3046FFF774FE019B63B1244B5B
:108ED0003B6000992846FFF728FF002C37D020463A
:108EE00000F084FD002432E0C4E900001D46D8E70C
:108EF0006A462D213046FFF72DFF009B0546013BBA
:108F0000012B01D9174BE3E7002302AE46F8043DDD
:108F100031460068FFF74DFE2060019B0BB1124BFC
:108F2000D6E731466868FFF744FE6060019B002B7E
:108F3000B7D00E4BCCE7424501D3434501D20C4B91
:108F4000C6E700992846FFF7F0FE00233B60204665
:108F500003B0BDE8F0830546BBE700BF44BE01088F
:108F6000BEBD0108DDBD010806BE010825BE010821
:108F700064BE010838B590B1451E15F8014F0CB913
:108F8000204638BD0DF0D6FF23462044427802F03B
:108F90000302022A08BFA4F120032B70EDE7012091
:108FA000EFE708B520B34A1C22D0062920D8DFE815
:108FB00001F0040D101316191C00002303600EF0BD
:108FC0000DF90840431C5842584108BD0023436036
:108FD000F5E700238360F2E700238361EFE70123D5
:108FE000C360ECE700230361E9E700234361E6E7A0
:108FF0000120EAE770B506460D1F01F1180455F887
:10900000041F4B1C03D1A542F9D1002070BD30468E
:10901000FFF7C7FF0028F6D0F8E708234A4291FB84
:10902000F3F302F0070201F0070158BF5142012299
:10903000DBB2C9B202FA01F1C25C1143C1547047FC
:1090400008234A4291FBF3F302F0070201F0070103
:1090500058BF51420122DBB2C9B28A40C15C21EA49
:109060000201C1547047082391FBF3F3DBB2C05CEB
:109070004B4203F0070301F0070158BF5942C9B240
:10908000084100F0010070472DE9F047089E8A462C
:1090900090461D46DDF82890074610B11446A245BB
:1090A00007D875B9012200240B9B1A602046BDE841
:1090B000F08721463846FFF7D6FF002861D10134FA
:1090C000EDE7099B023B042B04D8DFE803F0282CD2
:1090D0002C3034006B6801336B6028460EF07EF84C
:1090E000013108BFB0F1FF3FDCD031462846FFF721
:1090F00058FF0028D6D12FB3044621463846FFF743
:10910000B2FF002841D10134A245F6D10446013E08
:10911000042E19D8DFE806F02B2D2F313300AB6871
:109120000133AB60D9E7EB680133EB60D5E72B691E
:1091300001332B61D1E76B6901336B61CDE7002D02
:10914000E5D1AFE73C46E2E72C6028460EF046F852
:10915000013108BFB0F1FF3FA4D0B9F1000FA1D099
:1091600049462846FFF746FF00289FD09AE76C60E3
:10917000EBE7AC60E9E7AC61E7E7EC60E5E72C61C1
:10918000E3E7A045DBD1444690E7A045BFD1FAE72D
:1091900000232DE9F04F06468BB01C200C4690466C
:1091A000099300F039FC0546002800F0E4801C20FB
:1091B00000F032FC0746002800F0DD804FF0FF3160
:1091C000021F2B1F05F1180043F8041F984242F8B4
:1091D000041FF9D100230121D4F800A00DF12409C6
:1091E000CDE90031CDE902793C2123465246304693
:1091F000FFF74AFF099900296ED1824502D128461E
:10920000FFF77CFD02234FF0010AD4F804B0CDE94A
:1092100000A3CDE9025923465A463C2106F1080035
:10922000FFF732FF099B002B56D183454CD15146A5
:109230002846FFF763FD03234FF0020AD4F808B075
:10924000CDE900A3CDE9025923465A46182106F17B
:109250001000FFF719FF099B002B3DD1834546D134
:1092600051462846FFF74AFD40F26F1BA36905935C
:10927000E368049306F114030693DDF810A006F1E9
:109280001303079351460698FFF7EDFE28B10599A1
:109290000798FFF7E8FE002836D1BBF1010B33D069
:1092A000E36820460133E3600DF098FF013108BF09
:1092B000B0F1FF3F24D0A36929462046D4F80CA082
:1092C0000593FFF797FEDDE7424621463046FFF75C
:1092D0005FFF09900028AED0284600F087FB17B149
:1092E000384600F083FB09980BB0BDE8F08F42468A
:1092F00021463046FFF74CFF09900028ECD1B3E738
:1093000001234FF0000A0993099B002BE4D1049B31
:10931000534520D104212846FFF7F0FC05230622FF
:10932000D4F810A0CDE90032CDE9025923465246C7
:109330000C2106F11800FFF7A7FE099B002BCBD1EB
:109340008245C9D06369A3EB0803042B0CD94FF005
:10935000FF330993C0E7424621463046FFF718FF26
:1093600009900028B8D1D9E7424621463046FFF798
:109370000FFF0990B0E74FF0FF330993002DB2D0F3
:109380000027A9E72DE9F04F002487B0924606AAEE
:10939000894642F80C4D2C219846109DFFF7DAFCC7
:1093A000074688B93E4B2B6003993846FFF7BDFC52
:1093B00007B0BDE8F08FD0F800B072685A451CD2F3
:1093C000304600F013FB0134039BA342ECD957F85D
:1093D00024602F213046FFF7DAFBA8B92B46304630
:1093E00042465146FFF740FD2B680646002BE2D06F
:1093F0000028D9D000F0FAFAD6E759464846FFF7D8
:109400000CFE0BF1010BD8E700232F21304604AAF4
:109410000493FFF79FFC049906464B1E012B04D9C9
:10942000204B2B60FFF781FCBEE742462B4651469E
:109430000068FFF719FD2A6883462AB108B100F0D9
:10944000D5FA04993046EDE72D213068FFF79FFBF0
:1094500018B908F1FF32CBF80420002306A941F81F
:10946000043D7068FFF7A5FB059A00901AB10E4AFB
:1094700058462A60E3E7DBF80020DBF8041091424D
:1094800005D230460499FFF750FC584699E711463B
:1094900048460192FFF7C1FDDDE900321A44ECE7CE
:1094A00089BE01089BBE0108C0BE01082DE9FF412D
:1094B00000230E460393144602B902AC236048B958
:1094C0000546564B236003992846FFF72EFC04B04F
:1094D000BDE8F08103AA2021FFF73CFC039B054671
:1094E000062B02D04E4B2360EDE71A2200213046B6
:1094F0000DF091FD009400223C2331462868FFF7CF
:1095000041FF2268002ADED100943C2306F10801C5
:109510006868FFF737FF2268002AD4D10094182327
:1095200006F11001A868FFF72DFF2368002BCAD1B0
:109530006869FFF71FFD07223A496869FFF758FB82
:1095400080460EF03DFC012806F1130706D198F87D
:1095500000303F2B04BF2A2388F800300022082364
:10956000394640460094FFF70DFF404600F03EFAB2
:109570002268002AA7D107213846FFF774FD30B1D1
:1095800011463846FFF749FD0721FFF759FDEF68FF
:1095900006F1140838460EF013FC012804D13B787C
:1095A0003F2B04BF2A233B7020230022414638462C
:1095B0000094FFF7E7FE00214046FFF741FD2368D6
:1095C000002B80D12F693846FFF7D4FC00287FF4A8
:1095D0007AAF38460D221449FFF70AFB07460028E8
:1095E0003FF471AF183600940D2301223146FFF786
:1095F000C9FE384600F0FAF9012421463046FFF74B
:1096000032FD30B1611E3046FFF707FD2146FFF7FE
:1096100017FD01340D2CF0D155E700BF68BD0108DE
:1096200080BD01086800002084000020F0B58DB0E6
:10963000CDE90023054628B94FF0FF304FF0FF3148
:109640000DB0F0BD2422002103A80DF0E4FC03A915
:1096500068460DF0BFFB04460028EDD00DF0BEFDBE
:109660004A1C08BFB0F1FF3F06460F46E4D06269CE
:1096700021462846FFF78CFD0028DDD120460DF05D
:10968000ADFD4B1C08BFB0F1FF3FD5D08F4208BFE6
:10969000864203D020460DF0A1FDD1E72368204685
:1096A000013323600DF09AFD013108BFB0F1FF3F97
:1096B000C2D0626921462846FFF76AFD0028E9D03A
:1096C000BAE770B53C258AB0DDE90E64019496FBDB
:1096D000F5F405FB14640294182493FBF4F505FBE0
:1096E0001433CDE90330481E0C2190FBF1F301FB4C
:1096F00013010023CDE907339DF84030A2F26C72CC
:1097000001A80591069209930DF068FD0AB070BD9D
:10971000F7B5044602A860E902230DF049FB02698F
:10972000037A551C426990F804C0077B02F26C7101
:10973000067EC2690068A3700033207018BF012341
:109740002046013284F801C0E7702571A4F80510A5
:10975000E6712272637203B0F0BD30B5457A85B010
:10976000C4788378B0F805200179029505780195D1
:10977000407800902046FFF7A4FF05B030BD90422E
:1097800071EB0303B4BF012000207047032210B522
:10979000104986B00B78013393FBF2F202EB4202E0
:1097A0009B1A0D4A0B7052F823400278B0F805302E
:1097B000049242781A21039282780292C27801922E
:1097C000027920460092054A0EF094FA204606B02F
:1097D00010BD00BFEA4900206CBF01082FBF01087F
:1097E000B1F1004F08BF00281FB502460B4608D054
:1097F00001A8FFF78DFF01A8FFF7C8FF05B05DF8CE
:1098000004FB0148FAE700BF61BF01082DE9FF47EB
:1098100003220D462B4900280B78044603F101036F
:1098200093FBF2F202EB4202A3EB0203264A0B7017
:1098300052F8236075F100033EDA4FF0010A44420A
:1098400065EB4505214A0023204629460DF0B2F874
:109850001E4A07460023204629460DF0ABF8104665
:1098600019464FF4616200230DF0A4F84FF46162D1
:1098700080460023204629460DF09CF810461946E4
:109880003C2200230DF096F83C228146002320461E
:1098900029460DF08FF8CDF80080CDE901923B46C6
:1098A000BAF1000F0BD00A4A1A2130460EF022FA04
:1098B000304604B0BDE8F0874FF0000AC2E7054A21
:1098C000F2E700BFEA4900206CBF010880510100A7
:1098D0004DBF01084EBF01080FB404B0704700002F
:1098E0000FB437B51B4C256855B903222946012012
:1098F000F8F706FE2B462A4629462060F8F724FE94
:10990000154D2A68013A03321ED864212068F9F700
:1099100007F88022002111480DF07DFB07AB069A65
:1099200080210E4801930EF0E7FD7F2803DD0C49EE
:109930000C480EF03DFA2B68084898470023206831
:109940001A461946F8F700FE03B0BDE8304004B0EF
:10995000704700BF744A0020EC490020F449002001
:10996000E0BA01086F4A00200FB410B50D4CA2B048
:109970002268013A033210D825AB249A802102A82C
:1099800001930EF0B9FD7F2804DD07490DF1830036
:109990000EF00EFA236802A8984722B0BDE81040E6
:1099A00004B07047F0490020E0BA010870B50446E1
:1099B000054E4518AC4200D170BD14F8011B30466D
:1099C000FFF78EFFF6E700BFC5D6010838B50C4695
:1099D0001546FFF785FF20462946FFF7E7FFBDE85C
:1099E00038400148FFF77CBF67A4010810B5044662
:1099F00070B1F8F7DFFB2046F8F780FCF8F7B2FA11
:109A0000BDE81040034A938801339380F8F7CABA3F
:109A100010BD00BFF050002070B5214C8AB0226804
:109A200006460132632A22601E4D0BDDF7F7D4FD96
:109A30000523002201A9F7F781FDF7F789FA002332
:109A400028602360F7F784FA2B6803F57A7398424D
:109A500004D9F7F77DFA002328602360124A134CDB
:109A600013781BB92360636001231370F8F7A2FB1E
:109A70003046F8F7B1FB054668B1324600210DF0DB
:109A8000CAFAF8F76FFA238801332380F8F78AFAC5
:109A900028460AB070BD638801336380F8E700BFD1
:109AA0007C4A0020804A0020784A0020F0500020A4
:109AB000A0F14103052B02D83738C0B27047A0F19E
:109AC0006103052B01D85738F7E73038C0B20A28B0
:109AD00028BFFF2070470022013910B50144441E01
:109AE0008C4204D014F8010F08B1002A01DA1046A4
:109AF00010BDFFF7DDFF0F2802D840EA0212EFE7A2
:109B00004FF0FF32F3E70068704700687047006865
:109B100000BA7047837842781B04007843EA022336
:109B2000184370474278007840EA02207047027874
:109B3000407840EA022070470B12017043700B140A
:109B400009168370C170042070470B1603700B1444
:109B500043700B128370C170042070470370130EA2
:109B60004370130C8370130AC37002710520704791
:109B70000B12037041700220704738B505460C4641
:109B80000EF074F8611B013190FBF1F303FB11003F
:109B9000284438BD38B5451E15F8014F04B938BD05
:109BA0000DF0C8F923462044427802F00302012A4E
:109BB00008BF20332B70EFE72DE9F04106460EF089
:109BC000FFF830B3002734180DF0B4F914F8013C55
:109BD000354618444378621E19070DD42F463B784A
:109BE000A4EB050801355BB908F10102394630469E
:109BF000BDE8F0410DF0F6B904F8017C1446E3E746
:109C00000DF098F915F8013C184443781B07E5D48A
:109C1000EAE7BDE8F08108B50EF0C0F8B0FA80F0D0
:109C2000400908BD10B50446034B03604068F9F7CE
:109C300051F8204610BD00BFC8BF010810B504464A
:109C4000FFF7F0FF20460821FEF776FF204610BD03
:109C500038B5436804460D461BB90E210548F9F78F
:109C6000A5F829466068F8F75BFE431E5842584144
:109C700038BD00BF78BF01084068F8F7DFBF08B5FE
:109C8000002340681A461946F8F75EFC431E584206
:109C9000584108BD38B50D4600210B4B04464160C4
:109CA000036003220120F8F72BFC606018B95721EC
:109CB0000648F9F77BF82DB1002360681A4619466B
:109CC000F8F742FC204638BDE8B1010878BF01082A
:109CD000014BDB68184700BF844A00200120704711
:109CE00001B1096818B1806A431A58425841704757
:109CF00010B5044618B9D2210748F9F757F8074BB1
:109D00005B689847D4E90623904271EB0304B4BF23
:109D1000101A002010BD00BF09C40108844A0020A9
:109D20002DE9F8498846044610B10369012B03D197
:109D3000E7211748F9F73AF8D4E906BC5BEA0C03C7
:109D400023D0D4E90867BBEB06006CEB07010CF0ED
:109D5000E7FB0546206901380CF0C8FB01462846A0
:109D60000CF0D0FC054640460CF0C0FB29460CF038
:109D700015FC29460CF008FB0CF0FCFD321847F1ED
:109D8000000310461946C4E90601BDE8F88900BF82
:109D900009C4010838B50C4B0546186800F0E9FB0A
:109DA00010B90023184638BD4FF47A7403686C4329
:109DB0001A68A242F6D000F0D3FB0028F1D0036865
:109DC0001A689442F6E700BF844A002041F65832F0
:109DD000A0F55223A3F61833934224D8A0F55423B8
:109DE000A3F1F902622A1ED96FF454729A18C62A96
:109DF00019D9A3F21353302B15D9104B984214D90B
:109E000003F6B833984212D903F51673984210D965
:109E100003F5167398420ED903F5E173984294BF87
:109E2000052006207047002070470120704702205F
:109E30007047032070470420704700BFE8320D00D0
:109E4000F8B5054618B9F3212248F8F7AFFF224EBE
:109E5000306800F08EFB00283BD0002D39D003681D
:109E60001A79AA4231D11F7B00F07AFB20BB87B35D
:109E7000062D03D940211748F8F798FF174B53F8E0
:109E8000354024BBFE211348F8F790FF306800F0FE
:109E900070FB0646E8B17C4337683B79AB4204D19E
:109EA00021463846FFF73CFF3C61304600F058FB46
:109EB00006460028F0D10CE003681A79AA42D3D1F3
:109EC0001B7B002BD0D00137CEE70027CCE7012C3D
:109ED000DCD1F8BD09C40108844A0020D0BF0108C4
:109EE0002DE9F04F044687B058B3254B00681D6933
:109EF0000CF0FCFA0BF0E2FE1FA3D3E900230CF0F8
:109F00005FF8227B06460F462379D4F82890D4F8D0
:109F10001080D4F808A0BAB1062B98BF194A204681
:109F200094BF52F823B0DFF868B0FFF7E1FE324685
:109F30003B46CDE90198CDE903A01348CDF800B028
:109F4000A84707B0BDE8F08F062B98BF0D4A204602
:109F500094BF52F823B0DFF838B0FFF7C9FECDE95F
:109F60000189CDE903A0CDF800B032463B46074851
:109F7000E6E700BFAFF300800000000080842E41C0
:109F8000844A002008C00108F0C2010845C3010846
:109F9000E2C2010810B5104C206820B923690F48AF
:109FA000BDE81040184700F0EDFA2369014660B1A2
:109FB0000B489847206800F0DCFA044638B9204680
:109FC00000F0CEFA044610B910BD0648E8E7206854
:109FD000FFF786FFF3E700BF844A002064C2010850
:109FE00082C20108BCC20108F8B5134D06462B7E9B
:109FF0000F4623B94FF4B1711048F8F7D7FE2C681B
:10A0000024B96B690E4898472046F8BD0D4B204691
:10A01000002E08BF1E4600F0ACFA054608B9002421
:10A02000F2E7046839462046B0470028ECD12846BC
:10A0300000F096FAF1E700BF844A002009C4010845
:10A0400025C20108DD9C00082DE9F04F3E4D91B07E
:10A050002B7E83468946924623B94FF4C9713B480B
:10A06000F8F7A4FE2C6834B96B6939489847204644
:10A0700011B0BDE8F08F374B2046B9F1000F08BF93
:10A08000994600F076FA064620B96B69324898473F
:10A090003446ECE70468237BF3B94FF0FF37002424
:10A0A0004FF00008304600F05BFA064608BBBAF1F4
:10A0B000000F01D0CAF80070002FD8D1B8F1010FFD
:10A0C000D5D908F1FF313846FFF757FD10AB03EB48
:10A0D000800050F8404CCAE7A3685B45DDDB0021F7
:10A0E0002046C8470028D8D02046FFF701FE074683
:10A0F000D6E735682B7B002BD4D0AB685B45D1DB32
:10A1000000212846C8470028CCD02846FFF7F0FD9C
:10A1100048B9B8F10F0F9FBF10AB03EB880343F8AA
:10A12000405C08F101086CB187420AD8BAD1D4E981
:10A130000823D5E90801FFF722FB002818BF2C46A9
:10A14000B0E707462C46ADE7844A002009C4010861
:10A1500025C20108DD9C000849C20108000000007A
:10A160002DE9FF470D46044620B940F2E1112A4887
:10A17000F8F71CFE236923B94FF4F1712648F8F76C
:10A1800015FEDFF89CA04FF00009DAF8043098477C
:10A1900002460B460646C4E9082320690F460CF028
:10A1A000A5F929460CF0FAF929460CF0EDF80BF068
:10A1B00085FD17A3D3E900230BF002FF0BF0C0FAD3
:10A1C0000CF06EF8361847EB0907C4E906678046BD
:10A1D00020680CF08BF90BF071FD0DA3D3E900237F
:10A1E0000BF0EEFE064628460F46CDE902890BF03D
:10A1F00065FD3246CDE900013B46DAF8101007480C
:10A20000884704B0BDE8F047FFF7C4BEAFF3008055
:10A210000000000080842E4109C4010824C0010808
:10A22000844A002008B5FFF7D1FD003018BF012097
:10A2300008BD000038B50D4D04462A7E22B94FF402
:10A2400007710B48F8F7B2FD74B1237B63B10023AB
:10A2500020792373FFF7F4FD2B69064898472046C1
:10A26000BDE83840FFF73CBE38BD00BF844A00203F
:10A2700009C40108F4C1010838B50D4D04462A7E11
:10A2800022B94FF40A710B48F8F790FD74B1237BA3
:10A2900063B9012320792373FFF7D2FD2B690648A8
:10A2A00098472046BDE83840FFF71ABE38BD00BFCA
:10A2B000844A002009C401080DC20108F8B5194DEF
:10A2C00006462B7E23B94FF40D711748F8F76EFD43
:10A2D0002C6824B96B6915489847204601E00EB9EF
:10A2E0000020F8BD204600F044F904460028F7D0CD
:10A2F00023689E420CD137793046FFF7E9FC2146AE
:10A30000286800F04DF93846FFF79AFD0120E8E78C
:10A31000204600F025F904460028E9D16B6904487D
:10A32000DAE700BF844A002009C40108C1C301085C
:10A33000E3C301082DE9F843384D06462B7E8846D5
:10A34000914623B940F2F9113548F8F72FFD304610
:10A35000FFF768FF044630B96B69314631489847CA
:10A360002046BDE8F8833046FFF714FD044630B1BF
:10A370002D482B69314698472046FFF79FFF2B7EDB
:10A380001BB976212648F8F711FDAB6830209847B5
:10A39000044640B96B69254898476B6931462448A3
:10A3A00098470024DCE7302200210CF034FE3046D0
:10A3B000FFF70CFD0746207138B9EB682046984737
:10A3C0006B6931461B489847E7E7062803D94021C7
:10A3D0001348F8F7EBFC184B214603EBC70253F880
:10A3E0003730526823614FF47A73A2605E430022D3
:10A3F0000023C4E90623012326602373C4E90A89E4
:10A40000286800F097F82079FFF71AFD2B690B48B0
:10A4100098472046FFF764FDA2E700BF844A00206A
:10A4200009C40108DCC0010813C1010848C10108C2
:10A43000B9C1010876C10108D0BF0108A1C1010856
:10A4400070B50F4C0546237E23B94FF41C710D489F
:10A45000F8F7ACFC23685BB10B4E29463046FFF79A
:10A46000C3FD50B923692946BDE870400748184725
:10A4700063690748BDE870401847FFF729FCECE71F
:10A48000844A002009C40108E19C00089BC301081C
:10A49000C1C30108014B187E704700BF844A0020E9
:10A4A00084B070B504AC84E80F00154B1A7E1C46CE
:10A4B0002AB1BDE870405B69124804B018471D1D01
:10A4C00004AE0FCE0FC533682B600BB90E4B636122
:10A4D00023690BB90C4B2361E3680BB1A36833B953
:10A4E00023690A4898470A4BE3600A4BA36000F0CF
:10A4F00013F8012320602376BDE8704004B0704754
:10A50000844A002068C00108D9980008A1C0010849
:10A51000616F0108516F010810B50820FFF77CFA40
:10A520000446F6F70DFD0023C4E90034F6F7AEFD4E
:10A53000204610BD70B505460C200E46FFF76CFA9C
:10A54000044660B10660F6F7FBFC002363606B68AD
:10A55000A3601C6004346C60F6F798FD012070BDA8
:10A5600010B50446F6F7ECFC6468F6F78FFD20465C
:10A5700010BD10B50446F6F7E3FC2468F6F786FD37
:10A58000204610BD10B50446F6F7DAFC2368002417
:10A590001BB9F6F77BFD204610BD01345B68F7E779
:10A5A00038B50C460546F6F7CBFCD4E901324BB181
:10A5B0009A60A2681360F6F769FD2046BDE838404E
:10A5C000FFF714BA6A60F4E770B50446044E451804
:10A5D00014F8011B3046FFF783F9AC42F8D170BD87
:10A5E000C5D6010870B515460022C0E901150270F4
:10A5F000C0E90332C0E90522C0E907224262DDE971
:10A600000412044600F11C06F9F744F838B929464B
:10A610000748FFF765F92B210648F8F7C7FBDDE986
:10A62000042331462046F9F722F8204670BD00BFCA
:10A63000EA9A0108159B01082DE9F04100259DF8D3
:10A640001860C0E901120570C0E90335C0E905557D
:10A65000C0E90755456231460446174600F11C081B
:10A66000F8F766FE38B939460748FFF739F920216F
:10A670000648F8F79BFB324641462046F8F746FE6F
:10A680002046BDE8F08100BFEA9A0108159B010849
:10A69000F8B50025C0E901120570C0E90335C0E92D
:10A6A0000555C0E90755456206990446164600F16E
:10A6B0001C07F8F729FF38B931460748FFF710F9AA
:10A6C00020210648F8F772FB069A39462046F8F72B
:10A6D00005FF2046F8BD00BFEA9A0108159B010856
:10A6E000F0B50126044608270D468DB0694B6A4A2D
:10A6F0003146009602A8FFF79FFF02A92046FAF70D
:10A70000B9F802A8F9F7E2FB644BCDE900571A4605
:10A7100004210DEB0700FFF765FF0DEB0701204655
:10A72000FAF7A8F80DEB0700F9F7D0FBEB195C4A34
:10A730000197009304215B4B0DEB0700FFF752FFDD
:10A740000DEB07012046FAF795F80DEB07001027EF
:10A75000F9F7BCFBEB190093534B04211A46019700
:10A7600002A8FFF73FFF02A92046FAF783F8203539
:10A7700002A8F9F7ABFB4D4B4D4A00950421019718
:10A7800002A8FFF72FFF02A92046FAF773F802A8E4
:10A79000F9F79CFB0C23474A00930221464B02A881
:10A7A000FFF776FF02A92046FAF764F802A8F9F746
:10A7B0008DFB424B424A3146009602A8FFF73CFF10
:10A7C00002A92046FAF756F802A8F9F77FFB032200
:10A7D000002303923B4D3C4A3C4902A88DF80830C7
:10A7E0000495CDE90523CDE90733CDE909330B9372
:10A7F000F8F738FF38B929463548FFF771F82021B6
:10A800003448F8F7D3FA0025304A09A902A8F8F726
:10A81000F3FE02A92046FAF72DF802A8F9F756FB35
:10A820002D4B2E4A0095022102A8FFF731FF02A905
:10A830002046FAF71FF802A8F9F748FB284B294AE7
:10A840000095022102A8FFF723FF02A92046FAF78C
:10A8500011F802A8F9F73AFB0121234B234A009192
:10A8600002A8FFF7E9FE02A92046FAF703F802A8BA
:10A87000F9F72CFB1E4B1F4A0095022102A8FFF797
:10A8800007FF02A92046F9F7F5FF02A8F9F71EFB1A
:10A890000DB0F0BDE7C40108C8B00108FAC4010852
:10A8A0006BC8010852C8010808C5010873C801082F
:10A8B0009DC8010813B001080FC5010868C501084B
:10A8C000D8DB01082CB00108A4C80108CBB00108EE
:10A8D000EA9A0108159B0108B9C801084FB00108A0
:10A8E000F7C8010876B0010832C901087AA3010847
:10A8F0004EC901089EB0010830B504468DB001462E
:10A900007A4A6846F9F7C1FD794A214603A8F9F762
:10A91000BCFD784A214606A8F9F7B7FD76492046DE
:10A92000F9F7AAFD05467548FEF7DAFF0123039AF9
:10A9300002F11001914205D011F8010D002818BF55
:10A940000023F7E7002B53D06D48FEF7C9FF5DB336
:10A950006C48FEF7C5FF6C4A214609A8F9F795FD3A
:10A960006A48FEF7BDFF08210098FFF72DFE6848F2
:10A97000FEF7B6FF08210998FFF726FE6548FEF7A7
:10A98000AFFF10210698FFF71FFE6348FEF7A8FFF0
:10A990000998069A009900F0F7FE09A8F9F736F829
:10A9A0005E48FEF79DFF61E05D48FEF799FF5D4858
:10A9B000FEF796FF0699009800F044FE5A48FEF70D
:10A9C0008FFF042100980844FFF7FEFD5748FEF76B
:10A9D00087FF10215648FFF7F7FD5648FEF780FF26
:10A9E00010215548FFF7F0FD4B48FEF779FFD7E7F8
:10A9F000102206980CF0DCFA5049514B002808BF91
:10AA000019465048FEF76CFF002D3DD03D48FEF73B
:10AA100067FF3D4A214609A8F9F737FD4A48FEF786
:10AA20005FFF08210098FFF7CFFD4848FEF758FF69
:10AA300008210998FFF7C8FD4548FEF751FF10218E
:10AA40000398FFF7C1FD4348FEF74AFF102106981F
:10AA5000FFF7BAFD3048FEF743FF0998039B069ABB
:10AA6000009900F0A9FE09A8F8F7D0FF2A48FEF7E0
:10AA700037FF06A8F8F7CAFF03A8F8F7C7FF68462C
:10AA8000F8F7C4FF0DB030BD2548FEF729FF324866
:10AA9000FEF726FF039A0699009800F017FE224859
:10AAA000FEF71EFF042100980844FFF78DFD2B4898
:10AAB000FEF716FF10211E48FFF786FD2848FEF717
:10AAC0000FFF10212748FFF77FFD2748FEF708FFFB
:10AAD00010212648FFF778FD2548FEF701FF1648AC
:10AAE0001021FFF771FD0C485BE700BFFAC40108B5
:10AAF0009DC8010808C50108C8B001089AC5010829
:10AB0000B1C50108CCC501086BC80108D2C5010850
:10AB1000E3C50108F5C5010867A401089DC6010841
:10AB200015C601081AC601084CC601085EC6010810
:10AB3000600100208AC601089001002068A4010875
:10AB400083C50108BCC60108D9C60108EBC60108C7
:10AB5000FEC601081EC7010867C70108A1C7010892
:10AB60000DC801087001002024C8010880010020E0
:10AB70003BC8010810B5084CD4F82C211AB964213F
:10AB80000648F8F713F9D4F82C010023BDE810406B
:10AB900003222021F6F778BEB800002017CE010866
:10ABA000F0B51F461446C7B005460E46F1220021F7
:10ABB00009A80CF030FA09AA1021384602F07EFDEF
:10ABC00020460DF0FDF807461022002101A80CF0E8
:10ABD00022FA102F3A46214628BF102201A80CF075
:10ABE000F6F909AA05A901A802F0E2FD324605A975
:10ABF00028460CF0ECF947B0F0BD000038B50E4C1B
:10AC00000E4D94F83230022B11D123680C4898472E
:10AC1000082394F8FF20D4F80011012002F004FD6D
:10AC20006B6B00209847042384F8303038BDEB6A02
:10AC300098470123F8E700BFB80000205CF1010845
:10AC40005FCE010810B5044601F0D6F940B9054BB6
:10AC500005481B6898472046BDE8104001F0A2B99E
:10AC600010BD00BFB8000020E6CD0108054B93F8E9
:10AC7000212022B993F8350080F0010070470020B0
:10AC8000704700BFB8000020F0B570279DB00646A1
:10AC90000D463A46002168460CF0BDF908212B46C6
:10ACA0000DEB010004AC0B4AFFF77AFF2B46204660
:10ACB000094A102108ADFFF773FF94E80F0085E8FB
:10ACC0000F003A46694630460CF081F930461DB017
:10ACD000F0BD00BF08CE010810CE010884B070B5E9
:10ACE0008AB00EAC84E80F00784C4FF49C72254675
:10ACF000002120460EAE0CF08EF90FCE0FC596E85F
:10AD0000030014AE85E803000FCE04F118050FC54B
:10AD100033682B600E9B0BB96D4B23600F9B0BB9F7
:10AD20006B4B2360109B23B94FF4A9716948F8F766
:10AD30003DF8129B23B94FF4AB716648F8F736F82B
:10AD4000119B23B94FF4AD716248F8F72FF8139BAC
:10AD500023B94FF4AF715F48F8F728F8A36923B916
:10AD600023685D4898470323A361E3690BB90A236D
:10AD7000E36194F8233013B9012384F8233002F0FF
:10AD800097F994F8243013B9012384F8243002F0A1
:10AD900087F9A36A0BB9514BA36202F075F906F06B
:10ADA000DDFCC4F828010138033004D963684C483D
:10ADB0009847002082E0032200210120F7F7A0FB42
:10ADC000C4F8300120B940F287114248F7F7EEFF8E
:10ADD00000220421E069F7F793FB606420B940F298
:10ADE0008B113C48F7F7E2FF00220421E069F7F7F6
:10ADF00087FBA06420B94FF4C7713648F7F7D6FF38
:10AE0000002204210120F7F77BFBE06420B940F227
:10AE100091113048F7F7CAFF082384F80931042359
:10AE200084F80A31002384F83630012384F80D3188
:10AE3000FFF730FB05AD68B9A36822690593236865
:10AE400007920893E26863680692009395E80F0002
:10AE5000FFF726FB02F052F92368224E079363683E
:10AE600006F1A0020893236904960693E368DC3692
:10AE700005930AAB43F81C2D93E803008DE803000B
:10AE800095E80F0002F01CFE0196A3694FF4CD7205
:10AE90000093154901231548F5F738FE01280546AA
:10AEA00011D1002303220421D4F82C01F6F7ECFC85
:10AEB0000F4823689847284684F834500AB0BDE804
:10AEC000704004B0704763680A4871E7B80000201A
:10AED000D998000817CE010894CA010808E6D333B0
:10AEE000DDCA01080801002010CB01088DB0000860
:10AEF00018CB010835CB010810B5124CD4F82C3111
:10AF000023B94FF4DF711048F7F750FF03220421F3
:10AF10000023D4F82C01F6F7B7FC23680B489847B8
:10AF200042F21071D4F83001F7F7FAFC0023D4F89C
:10AF300030011A461946F7F707FB23680448BDE8B5
:10AF400010401847B800002017CE0108F1CB0108C7
:10AF500018CC010838B50E4DD5F8303123B940F280
:10AF6000CF110C48F7F722FF0021D5F83001F7F791
:10AF7000D7FC0128044608D10023D5F830011A4631
:10AF80001946F7F7E1FA204638BD0020FCE700BF7C
:10AF9000B800002017CE010810B5FFF7DBFF0B4CFF
:10AFA00078B1002303220821D4F82C01F6F76CFCB9
:10AFB000236807489847D4F82C01BDE81040F5F7FE
:10AFC0003DBF23680348BDE810401847B800002083
:10AFD00033CC010855CC0108014BD863704700BF42
:10AFE000B8000020002307B502A941F8043D044B36
:10AFF0000246D86CF7F702FC019803B05DF804FB39
:10B00000B800002070B5FFF7A5FF1B4D044620B126
:10B010006B681A489847002070BD686CF7F70EFE01
:10B02000EB69834202D22B681548F3E7214620469C
:10B0300002F076FD064610B92B681248EAE7047064
:10B0400000F09EFF044618B9304602F0A1FDE2E789
:10B050000D4A13680133136063B913680133136039
:10B06000636001236370032320462370FFF7EAFD2A
:10B070006068D1E71368F3E7B800002065CB0108EA
:10B0800091CB0108BCCB0108A04A00202DE9F84370
:10B0900001236F4CDFF8C0816E4E84F830300A23F4
:10B0A0006D4A4FF0FF310020F6F7AAFB012872D15C
:10B0B000D8F8000043071DD5337833B106F09CFA69
:10B0C000002006F0EDFA00233370F6F74BFF2368FB
:10B0D00062489847F6F766FF022384F83030002371
:10B0E000D4F830011A461946F7F72EFA0020F6F781
:10B0F000F9F8D4E710F0080524D0337893B941F279
:10B10000883006F0A5FA18B9A0215548F7F74EFE89
:10B11000544806F0C5FA0123534833702368984712
:10B12000FFF76CFD0020F6F79DFC4FF4FA61D4F8B0
:10B130003001F7F7F5FB0028B1D1A7214848F7F710
:10B1400035FEACE710F0200055D0337803B394F807
:10B150003030042B1CD1454F2A463946D4F82801FB
:10B16000F7F78EFC0128814612D13B78072B32D1AC
:10B170003F4823689847284600F002FF40B1052267
:10B18000C0E90155056180F801900270FFF75AFD92
:10B190000020F6F767FC3378002B80D000F044FFE6
:10B1A000054600283FF47BAF032384F83030037852
:10B1B0004168052B98BF2F4A276894BF52F8232077
:10B1C0002D4A2E48B8472B78052B3DD8DFE803F0F1
:10B1D000161D1D3131392A463946D4F82801F7F7B2
:10B1E0000DFB0128D4D12368397825489847384683
:10B1F00006F05CFACCE7F6F735FC50E7D6211848A4
:10B20000F7F7D4FDFFF7FAFC49E7FFF72FFD38B950
:10B21000284600F0F5FA80B1284600F0C3FEF1E7B9
:10B220002368184898472846FFF70CFDFFF7EAFE09
:10B23000E8E7284601F0BAFCEDE72846FFF702FDF3
:10B24000E0E700F01FFEE7E763680F489847E3E791
:10B25000B8000020A44A0020B44A0020A0C9010878
:10B2600017CE010875AB0008C3C90108A84A002021
:10B27000F3C9010880C9010898C901082FCA01084B
:10B280000ACA01084DCA010874CA0108024B93F8A2
:10B29000FC0002F021B900BFB80000202DE9FF41F9
:10B2A00080460F461646ADF80430FFF753FE4A4D70
:10B2B000044638B16B68494898470024204604B0DA
:10B2C000BDE8F081686CF7F7B9FCEB69834203D203
:10B2D0002B6843489847F1E7FFF7D8FF87420146BC
:10B2E00005D92B6895F8FC203E489847E6E71EB93B
:10B2F0003FB12B683C48DFE7DF2E02D92B683B4883
:10B30000E8E73946404602F00BFC044610B92B68CA
:10B310003748DFE79DF80530C3B3042323709DF859
:10B3200004303BB10D2304A901F8043D012220465D
:10B3300001F0BCF895F8312095F83230934203D1F2
:10B3400095F83330934217D02023022A18BF0022E9
:10B350008DF80C3094F8783003A90BBF43F0040348
:10B3600043F001038DF80D208DF80D20204684F860
:10B370007830022201F09AF86677204600F000FE4D
:10B38000064628B9204602F003FC96E70223C5E7EB
:10B390000023184A83601368013313609BB9136854
:10B3A0000133136073600A9B30463361012373706D
:10B3B000337000F009FE044638B9304600F0F2FD63
:10B3C0006B680D4886E71368ECE72B6871680B48DB
:10B3D0009847746872E700BFB800002065CB010889
:10B3E00091CB010895CC0108F1CC010816CD0108DC
:10B3F00036CD0108A04A002071CD010899CD010881
:10B40000082808BF0120034B83F8230083F8FC00C1
:10B41000704700BFB8000020024B83F8240083F877
:10B42000FD007047B800002008B5FEF770FB014B27
:10B43000586508BDB8000020034630B5054C00F142
:10B440001005224618685968083303C2AB421446F7
:10B45000F7D130BD80010020034630B5054C00F126
:10B460001005224618685968083303C2AB421446D7
:10B47000F7D130BD70010020034630B5054C00F116
:10B480001005224618685968083303C2AB421446B7
:10B49000F7D130BD60010020034630B5054C00F106
:10B4A0001005224618685968083303C2AB42144697
:10B4B000F7D130BD9001002010B50446FFF7BCFF66
:10B4C0002046FFF7C9FF2046BDE81040FFF7D4BF74
:10B4D00030B51025C3B0224CF122002105A80BF095
:10B4E0009AFD2A46002101A80BF095FD94F86730DB
:10B4F00005AA8DF8053094F8663029468DF8063097
:10B5000094F8653004F178008DF8073094F86430D1
:10B510008DF8083094F863308DF8093094F8623073
:10B520008DF80A3094F861308DF80B3094F8603063
:10B530008DF80C3002F0C2F8052305AA04F1980139
:10B5400001A88DF8043002F033F9062305AA04F1AE
:10B55000880101A88DF8043002F02AF943B030BD0B
:10B56000B80000200246024B0068516803C37047D0
:10B57000100100200246024B0068516803C3704767
:10B5800018010020034630B5054C00F11005224695
:10B5900018685968083303C2AB421446F7D130BD6E
:10B5A00020010020034630B5054C00F1100522466D
:10B5B00018685968083303C2AB421446F7D130BD4E
:10B5C00030010020014B83F822007047B8000020B2
:10B5D00030B1044B044A02280CBF1846104670478D
:10B5E000024870478DCC010898C9010885CC010834
:10B5F00070B50546FFF7ECFF034C0146266803488B
:10B60000B04784F8315070BDB8000020CBCD0108A0
:10B61000014B1864704700BFB800002013B5002428
:10B62000064B02AA42F8044D054993F8FD00FEF7C7
:10B630000BFD2146019802B010BD00BFB8000020EC
:10B64000F1B7000830B50430C7B00D46FFF7ECFE87
:10B650001C4B0DF1050203F10C0153F8040B8B4256
:10B6600042F8040BF9D11B880124138000238DF8C4
:10B670001330022309AA102128468DF8043002F065
:10B680001DF809AA05A901A802F092F805A8FFF77C
:10B6900003FF09AA102128468DF8044002F00EF895
:10B6A00009AA05A901A802F083F805A8FFF704FF7D
:10B6B0001022054B83F8214083F8202083F8502086
:10B6C00047B030BDE2CB0108B800002030B50430EF
:10B6D000C7B00C461546FFF7A7FE294B0DF1050232
:10B6E00003F10C0153F8040B8B4242F8040BF9D11F
:10B6F0001B882046138000238DF813300223012479
:10B7000009AA10218DF8043001F0D8FF09AA05A973
:10B7100001A802F04DF805A8FFF7BEFE09AA102106
:10B7200028468DF8044001F0C9FF09AA05A901A81F
:10B7300002F03EF805A8FFF77FFE032309AA05A93A
:10B7400001A88DF8043002F033F805A8FFF784FE55
:10B75000042309AA0DEB030005A98DF8043002F0BB
:10B7600027F805A8FFF788FE1122064B83F8214031
:10B7700083F8202083F8502083F8074147B030BD7C
:10B78000E2CB0108B800002038B50D461446FFF79B
:10B79000E9FE2846FFF7EEFE2046FFF7F3FE2046BF
:10B7A000FFF700FF0022034B83F82120102283F8CB
:10B7B000202038BDB800002070B50E4615461C4646
:10B7C000FFF7D0FE3046FFF7D5FE2846FFF7DAFE3A
:10B7D0002046FFF7E7FEBDE870400022034B83F8E8
:10B7E0002120112283F82020FFF772BEB80000202C
:10B7F00028B1836A012B01D1007B7047002070477C
:10B800002DE9F04F044689B010B10378012B03D025
:10B810001C219448F7F7CAFA63691BB91D219148A6
:10B82000F7F7C4FA63691B78042B05D0022B03D009
:10B830001E218C48F7F7BAFA0026DFF85C928A4896
:10B84000D9F80020904799F8FF3099F8FD800293CD
:10B8500008AAD9F8003142F80C6D8449404699F89D
:10B86000FCB099F8FEA00393FEF7EEFB4D460746A9
:10B8700058B9D9F800307E489847204600F044FC7B
:10B880000127384609B0BDE8F08F059BB3B1FEF73C
:10B8900081FB0599042904D9204600F06DFC00279E
:10B8A000EFE7D9F80030734898470598724B434347
:10B8B0004FF47A70B3FBF0F0F5F79CFCA36801330A
:10B8C000012BA3600FD1D5F8F03060690133C5F8C2
:10B8D000F03095F80831013385F8083100F0BAFCF2
:10B8E000606900F011FE6B6D66697360D5F8F03029
:10B8F000738195F804316BB3002385F80431337AF2
:10B9000043F00403337295F8FC30384686F87C30F7
:10B9100001F036FC86F87D000121606900F0C6FC6C
:10B9200095F80D214FF47A7312F00F0208BF01222F
:10B9300000265A4307AB019306AB0093394602F544
:10B940007A736069069600F07FF9074628B92B687C
:10B950004A4891E7A6F87A30D5E7F5F7F9FAE060BA
:10B96000069860B1314600F0A1FC069B1B78052BC0
:10B9700004BF012385F80431002385F806310698B9
:10B9800000F032FCDDE9060101F0C0F8069911B3C0
:10B990000A7A12F0040320D0B9462B684989384846
:10B9A000984795F80B31A360069A32B16269127814
:10B9B000022A04BF95F80B21A26000F04DFB064659
:10B9C00050BB8A212748F7F7F1F92E4B2E4A8B21DD
:10B9D00024480BF0A9F98946E6E79946E4E73146A1
:10B9E000606898476420F5F705FC304600F044FB9A
:10B9F0002B6895F80B21A1682448984795F80B31DE
:10BA0000A2689A422B6802D32148984739E7214817
:10BA100098470323337042E78022616918300BF0A6
:10BA2000D6FA00229DF808300699F373039BC6F8F6
:10BA3000981021787272336195F83530C6F88020FD
:10BA40003375236986F80CB086F80D8086F80EA051
:10BA50003270717086F80890002BC0D1304600F02B
:10BA600031FBC5E7AFCE0108F4CE0108F1B70008FD
:10BA700018CF010852CF010840420F007FCF0108C4
:10BA8000BFCF0108DBCF0108A1CE0108E4CF010838
:10BA900001D0010815D00108B80000202DE9F043BD
:10BAA00085B006460C468DF80F202BB101220DF112
:10BAB0000F01002006F0E0F9F5F74AFA1C4B1D4D86
:10BAC000DFF878809DF80F1007469B6A204698475C
:10BAD00041F288322946D8F82801F6F78FFE28B3BC
:10BAE0002B78012B1DD12846AC6805F0DFFD4FF403
:10BAF0007A70A4EB070909FB00000AF0F7FC014685
:10BB00003046FEF72DFB9DF80F10CDE90049D8F81F
:10BB100000503B4632680848A847204605B0BDE8BB
:10BB2000F083284605F0C2FD0024F6E70446F4E75A
:10BB30005CF10108B84A0020D7D10108B800002004
:10BB40002DE9F84F394E9846736B054689461446E1
:10BB50004FF47A7A9847DFF8DCB0354F0AFB05F2EC
:10BB600002F59C328032B2FBFAF23249D7F8280152
:10BB7000F6F744FE20B9336B98474FF0FF302FE0C3
:10BB80009BF80030072B07D1584605F08FFD4FF486
:10BB90007A6506F0F5F8E1E7032B366B22D1DBF886
:10BBA000045028792968844228BF04464846224622
:10BBB0000BF00DFA3F6895F90830B5F90620A98811
:10BBC0001D48B847B8F1000F05D0EB88A8F8003041
:10BBD0002B7A88F80230174805F068FDB0472046F8
:10BBE000BDE8F88F042B0BD1124805F05FFDB0477C
:10BBF0003C68F5F7ADF901461048A0470020EFE793
:10BC0000052B0AD10B4805F051FDB0473C68F5F70C
:10BC10009FF901460A48A047AFE7D3210948F7F743
:10BC2000C5F8044805F042FDB047A6E75CF10108FD
:10BC3000B8000020C44A002049D0010873D0010890
:10BC40008BD00108A1D001082DE9F04FC9B08B4677
:10BC5000904608A9FF2202901F46DDF84CA101F092
:10BC6000B1FF7A4D044630B92B68794898470020D7
:10BC700049B0BDE8F08F95F8FC1095F8FE60DBF850
:10BC800000208E4298BF8E1B084694BFF6B2002655
:10BC9000D5F800900592049101F0CAFB039095F845
:10BCA000FD0001F0DBFBDDE90412039B0090694815
:10BCB000C847DBF800203046D5F80090039201F029
:10BCC000B7FB039A034631466348C84795F8FF100F
:10BCD000D5F800210846D5F800900492039101F0B0
:10BCE000A7FBDDE9031203465C48C84795F8FD3021
:10BCF00095F8FC20DBF8001000200DF1200901F080
:10BD000093FC2246002349465846FFF7C7FE0446E7
:10BD100010B92B685248A9E7029B4C4D93F8783034
:10BD200013F0050F12D013F0040F0CBF00200220F7
:10BD300095F83230834209D02B6885F8320002939F
:10BD4000FFF746FC029B014646489847FF22002128
:10BD500048460BF060F932464FF47A760823DBF858
:10BD60000010012001F060FC06FB08F1A1F51C4168
:10BD70004039B1FBF6F106A80694F5F7FBF95346F6
:10BD8000FF2249464FF44D70FFF7DAFEB0F1FF3F56
:10BD9000804602D12B68344868E700282ADD2E68E7
:10BDA000F5F7D6F82346024641463048B047BAF187
:10BDB000000F02D001238AF803300024529BA045D3
:10BDC0001C6015DD5FFA88F1484602F06DFA529B5F
:10BDD000274E18602B682748984719F804102B68DD
:10BDE000304601349847A045F7D12B682248984740
:10BDF00001203DE7082395F8FF20D5F80011012028
:10BE000001F012FC06FB07F1A1F51C414039B1FB22
:10BE1000F6F107A80794F5F7ADF95346FF22494616
:10BE20004FF44D70FFF78CFEB0F1FF3F804602D11A
:10BE30002B6812481AE70028BFDD01462B6810481E
:10BE40009847BAF1000FB8D00223B4E7B800002039
:10BE50007BD2010898D20108CBD20108F2D20108A6
:10BE600019D3010838D301085ED3010887D301082C
:10BE7000C5D6010807D4010867A40108BBD301088F
:10BE8000E4D301082DE9F041314CC2B023684FF4EE
:10BE90007A61304802AF984701ABFF2239464FF430
:10BEA0007A60FFF74DFE061E25464EDD23683146BB
:10BEB000294898472368294898470024DFF8BC8020
:10BEC000395D2B68404601349847A642F8D12B686B
:10BED000234898476A6DF1B2384601F0B5FF044631
:10BEE00038B303782F68052B27D0032B2AD11D499F
:10BEF000627F237F1C48B8472B6818489847217FEA
:10BF0000A06EFDF753FD2B68154898470021204689
:10BF100000F0CCF9204600F067F90199204600F0C6
:10BF2000F5FD2B6C5BB92B6810489847204601F053
:10BF30002FFE304642B0BDE8F0810D49D8E72046DB
:10BF40009847F6E70B48B847F0E723680A48F7E751
:10BF5000B8000020E7D0010814D1010807D4010877
:10BF600067A40108E4D001082DD1010878D10108A7
:10BF700068A40108A0D10108C6D10108C5D60108EE
:10BF800038B5074B0546DB6818209847044620B1B2
:10BF9000142200210BF03FF86561204638BD00BF38
:10BFA000B800002010B5044650B1406901F0F0FD22
:10BFB00000236361034B2046BDE810401B6918470E
:10BFC00010BD00BFB8000020037807B5052B4FF067
:10BFD000000302A941F8040D06481A460CBF806C04
:10BFE000406CF6F7B1FA431E5842584103B05DF871
:10BFF00004FB00BFB800002007B5037802A941F890
:10C00000040D0848052B4FF000024FF001030CBF50
:10C01000806C406CF6F798FA431E5842584103B0C2
:10C020005DF804FBB800002037B5002202AC094DD2
:10C0300044F8042D2146A86CF6F7E0FB019B33B9C8
:10C0400095F836201AB92146686CF6F7D7FB0198A7
:10C0500003B030BDB8000020064B10B5DB68A0204F
:10C060009847044618B1A02200210AF0D4FF2046C8
:10C0700010BD00BFB800002070B504460E4D0F483B
:10C080002B689847B4B1D4F8803033B12B680C4892
:10C0900098472B69D4F880009847D4F8980020B1CD
:10C0A00001F076FD0023C4F898302B692046BDE8E6
:10C0B0007040184770BD00BFB80000204ED2010884
:10C0C00067D201081FB50E4C0190E06CF6F7C8FD71
:10C0D000024638B903A9E06CF6F790FB10B103985B
:10C0E000FFF7CAFF002301A91A46E06CF6F72CFA05
:10C0F00020B94FF4B4710348F6F758FE04B010BDF0
:10C10000B8000020A1D00108F8B5042343700378DB
:10C110000546032B0ABF144B0469DC6BFFF79CFF39
:10C120000646B0B940F277111048F6F73FFE104BC3
:10C13000104A4FF4BC710D480AF0F6FD31466868AC
:10C14000A0473046FFF798FFFA20F5F753F8384636
:10C15000F8BD01272B7807704370002CEED1FFF754
:10C16000B1FF2046F4E700BFB8000020A1D00108CD
:10C1700041D001080AD20108F8B503780646032B1E
:10C1800008BF154B0F460CBFDC6B0469FFF764FF5B
:10C190000546B0B94FF4C8711048F6F707FE104BCA
:10C1A000104A40F291110D480AF0BEFD2946706810
:10C1B000A0472846FFF760FFFA20F5F71BF801209B
:10C1C000F8BD02230370337847604370002CEDD133
:10C1D000FFF778FF2046F3E7B8000020A1D0010860
:10C1E00041D0010826D2010837B5174C10B1002301
:10C1F00084F8083194F8223023B394F8081194F8A5
:10C20000092191421ED994F80A318D1A95FBF3F059
:10C2100003FB1050B0B90D482568A84700F050FF47
:10C2200020B900F05BFF08B900F068FF94F8230024
:10C2300094F8FC3094F8242094F8FD1000902468C1
:10C240000348A04703B030BDB80000203CD401082B
:10C2500092D4010870B5124C054694F82230EBB127
:10C26000037A266843F00103037294F8092194F8D5
:10C27000081194F80A310B48B04794F8081194F863
:10C28000092191420AD92B7A246843F002032B72C8
:10C29000A446BDE8704001230348604770BD00BF5D
:10C2A000B8000020C1D4010801D501082DE9F341EF
:10C2B00005464E4C4E4A4F4823680E4600290CBF97
:10C2C000014611464C48984723684C489847696E88
:10C2D00023684B4898472B784A48072B96BF4A4A11
:10C2E0004A4952F8231027686A78B84723684848B3
:10C2F00098472368697F474898472368297F4648BD
:10C30000984723686989454898472368696844487D
:10C310009847297A0B090193C1F3C0030093002EBB
:10C3200032D0C1F38003C1F34002266801F001015D
:10C330003C48B0472B7A13F0F00F11D023683A48ED
:10C340006FF00B079847DFF8F48005F10C067F1BB0
:10C35000297ABA19B2EB111F236810DB33489847CA
:10C360002368334898472B7F002B3AD12368314804
:10C37000984723682D4802B0BDE8F041184716F8E9
:10C38000011B40469847E3E7C1F38003C1F3400235
:10C39000266801F001012848B0472B7A13F0F00F0E
:10C3A000DED0236820486FF00B079847DFF88C80B9
:10C3B00005F10C067F1B297ABA19B2EB111F23680D
:10C3C000CCDA16F8011B40469847F4E7AB6E4046BE
:10C3D000995DB84701362A7FB3B29A422768F5D8EB
:10C3E000C7E70026DFF85880F5E700BFB800002057
:10C3F0003CD5010843D501084CD5010868D5010892
:10C400007ED501088DD501081CD4010898C9010802
:10C41000A1D50108AED50108C4D50108E3D50108AE
:10C42000FBD5010816D601085BD6010867A40108F0
:10C43000ADD60108BCD601086BD60108C5D60108E7
:10C44000C4D60108064A1378FD2BDFBF00780549E2
:10C45000C8540133DABF012013700020704700BFB9
:10C46000D14B0020D24A002038B10078032803D0F5
:10C47000431F58425841704701207047084B07B589
:10C480001B6808489847052302A800F8013DFFF7FC
:10C49000D9FF0548FFF7D6FF03B05DF804FB00BFE6
:10C4A000B8000020A2DB0108D04A0020037A70B552
:10C4B0001B09D61804460F2E00F10C00154618442F
:10C4C0000E4E0DDC0AF083FD237A0D4805EB1312A6
:10C4D00062F307132372294633689847012070BD21
:10C4E000C3F10F020AF073FD237A064843F0F0030C
:10C4F00023722946336898470020F0E7B8000020EF
:10C500005EDB01087DDB010837B5114C054622785A
:10C5100022B11049FFF7CAFF002323700E4C94F894
:10C5200006213AB1082302A901F8043D0122284658
:10C53000FFF7BCFF94F8073143B140F2011302A9A1
:10C5400021F8043D02222846FFF7B0FF03B030BDBA
:10C55000D14B0020D24A0020B800002038B5074C4B
:10C5600000F00F0523682A4694F80D1104489847F7
:10C57000012384F80D5184F8063138BDB80000203D
:10C5800038DB0108000000002DE9F04F00268FB0D5
:10C59000CDE904019DF860A09F4D08920693564591
:10C5A00080F01082069B9D4813F806B09F190BF18E
:10C5B000FF32D2B21F2A98BF99492B6894BF51F815
:10C5C0002220984A594698470BF1FF331F2B00F25F
:10C5D0007582DFE813F0200073022B00EB013F01AE
:10C5E000FB00A001E601EB01C8017302FA01C100E2
:10C5F000240226027302730273027302730273022F
:10C600007302730273027302730273027302730282
:10C61000730273024802AAEB0603DBB2012B4FF050
:10C62000000427D085F80741022423E00024AAEB68
:10C630000603DBB207938DF82C40079A231D9A421C
:10C6400002DD3B5D032B17D0A4B103230EA800F835
:10C65000083DFFF7F7FE0BA8FFF7F4FE9DF82C103E
:10C660002F6801F001030093C1F38002C1F340037E
:10C670006D48B84734449AE107EB040999F8018002
:10C68000A01C4FEA181138440991FDF74BFA99F8AC
:10C6900004900999C9F302130534062908F00F081C
:10C6A0000290039309F00F09E4B231D90F292B68E6
:10C6B00034D19DF82C3043F002038DF82C3008F172
:10C6C000FF32062A2B682CD9B8F10F0F31D19DF813
:10C6D0002C3043F004038DF82C302B68B9F1000F97
:10C6E00006D04A4695F80B115048984785F80B91AB
:10C6F000039A2B680ABB4E4802999847029800F0AB
:10C70000DFFD9DF82C3043F001038DF82C3094E7C9
:10C7100085F8FC102B6847489847CAE74648984771
:10C72000CDE7424695F8FD104448984785F8FD80CE
:10C73000CDE7414642489847CFE7039A062A06D1FB
:10C740003B484FF6FF7198474FF6FF70D7E7DDE99A
:10C7500002213C48984770E7AAEB0603DBB2052BA1
:10C7600040F2AA813B780D2B40F0A681781CFDF7A2
:10C77000CCF997F905300021002B23DB22A4D4E962
:10C7800000344FF0000995F80D811B184C4118EB4F
:10C7900003031F46089B49EB0404022BA04604D167
:10C7A0007B1C44F100041F46A04604992B683A46BE
:10C7B000096F2548984739464246049BC3E91C1235
:10C7C000062457E712A4D4E90034DAE73B78062BB5
:10C7D00040F072810EA800F80C3DFFF733FE059B78
:10C7E0000EAF03F01F0207F8082D95F80C112C6806
:10C7F0001648A0471648FFF725FE3846FFF722FEE9
:10C80000012437E7AFF300806E3DD5120000000031
:10C810006F3DD51200000000B800002008D80108C4
:10C8200080D7010800D80108F8D801089BD8010872
:10C83000B4D8010829D801084AD8010867D80108E6
:10C8400080D80108CDD801082ED901084CD901089B
:10C85000C4010020AAEB0603DBB2042B40F22C81BA
:10C860003C78052C40F02881D7F801202B680C92E9
:10C8700095F8FE10C2F30212954898479DF83020B3
:10C88000944FC2F3021385F8FE303B7802F00F029A
:10C8900043F00403052A3B702B682DD895F8FF1050
:10C8A0008D4898479DF83030C3F3030385F8FF3077
:10C8B0003B7843F002030DF131003B704FF0640808
:10C8C000FDF728F908FB00F8404605F05BFA2B68F5
:10C8D0008146C0B14246D5F80011804898477D4A4C
:10C8E000C5F80081137843F00103137001227C4BDB
:10C8F0001A70FFF7C3FDBDE611467A4898473B78AA
:10C900006FF34103D7E74146774898473B7869F38F
:10C9100000033B70EAE7AAEB0603DBB2052B40F20B
:10C92000CB803C78072C40F0C7803B4653F8010F82
:10C93000F9781A793B79090241EA0341BB780C90F6
:10C9400019436423787859438DF8342000F03AFC79
:10C950008DF828000EA800F80C4DFFF773FD0AA80B
:10C96000FFF770FD2CE7AAEB0603DBB2042B40F2C5
:10C97000A3803C780A2C40F09F806421D7F8010006
:10C98000030A5943C0B200F065FC8DF82C000EA8D4
:10C9900000F8084DFFF756FD0BA8FFF753FD0524DF
:10C9A00068E6787800F00F00FFF7D8FDB41CE4B219
:10C9B000A64240F08A804D4BAAEB06021B685946FE
:10C9C0004B4898470FB0BDE8F08FAAEB0603DBB2E7
:10C9D000012B71D097F80080B8F10C0F6CD14FF09B
:10C9E00001097C782B68270909FA07F704F00F047E
:10C9F0003A4695F809113F4809FA04F998473E4824
:10CA000085F809712B684A4695F80A1198470EA8CF
:10CA100085F80A9100F8088DFFF714FD04E6F41C70
:10CA2000C5E7AAEB0603DBB2012B45D03C780F2CFF
:10CA300042D1AB687F7898470122304B8DF82C208B
:10CA4000C3E900013B090EA80A3302FA03F307F019
:10CA50000F0700F8084DC5F81831C5F81C71FFF72D
:10CA6000F1FC0BA8D8E7AAEB0603DBB2012B23D01D
:10CA70003B78202B20D17C780CB1022C1CD1204695
:10CA80002F68FEF7A5FD01461D48B84795F833000D
:10CA9000844203D12B681B489847C5E52F68FEF7F1
:10CAA00097FD80462046FEF793FD41460246164814
:10CAB000B84785F83340B7E50024DBE52B68AAEBDF
:10CAC000060259460A48984775E7264667E500BFBB
:10CAD00070D90108D04A00209FD90108EDD901087A
:10CAE000D14A0020CBD901081ADA0108B800002089
:10CAF00000DB010841DA010866DA0108C8010020FC
:10CB00008BDA0108B6DA0108D9DA010830B585B048
:10CB100003910446174B30B91B7803B305B0BDE849
:10CB20003040FFF7ABBC00259DF90E109DF80F209B
:10CB30001D70FFF799FC90B10F48237A90F82250AE
:10CB40002DB113F0010518BF012580F805511B090F
:10CB500007D0009304F10C032046FFF715FD05B044
:10CB600030BD637F002BFAD1237F002BF7D00093D9
:10CB7000A36EF1E7D14A0020B800002010B50446AA
:10CB800078B1836A012B0CD1C36A1BB91021064806
:10CB9000F6F70CF9E36A587802288CBF00200120D0
:10CBA00010BD0020FCE700BF7CDC01082DE9F04F40
:10CBB000054689B018B10378033B012B03D9222124
:10CBC0005548F6F7F3F86B690BB11B781BB12321BD
:10CBD0005148F6F7EBF80026DFF868914F48D9F88E
:10CBE0000030984799F8FF3099F8FD800393D9F801
:10CBF000003199F8FCB0029399F8FEA000F050FAC9
:10CC000000F056FA08AA42F80C6D45494046FDF777
:10CC10001BFA4C46074640B94248D9F800309847BD
:10CC20002846FFF771FA01270AE0059BCBB1FDF713
:10CC3000B1F90599042907D92846FFF79DFA374627
:10CC4000384609B0BDE8F08FD9F80030364898472B
:10CC50000598364B43434FF47A70B3FBF0F0F4F78A
:10CC6000C9FAAB6894F820200133102AAB6035D1A3
:10CC7000012B09D1D4F8F0300133C4F8F0302C4B3B
:10CC80005B699847A4F8E800B4F8E8300133A4F8E9
:10CC9000E83000262368B4F8E8102648984707AB28
:10CCA00094F8FF9084F8FF60019306AB0093394637
:10CCB00041F2707341F2883268690696FEF7C4FF4C
:10CCC0000746C0B923681C4898472846FFF71CFA56
:10CCD000069800F05DFF84F8FF90A4E7112A05D1C3
:10CCE000636916489847A4F8E800D2E750210A483B
:10CCF000F6F75CF8CDE7069A84F8FF90236812B146
:10CD00001278012A20D00E4898472846FFF7FCF9F0
:10CD1000069800F03DFF93E77CDC0108BFDC0108CA
:10CD20007DCB0008DFDC010852CF010840420F0034
:10CD30005CF1010815DD01082ADD01081001002061
:10CD400060DD0108B8000020A548984794F82090BD
:10CD5000B9F1100F40F0E1802368A248984784F8A9
:10CD60005090069B616DDA689F482368626598471A
:10CD7000069B002E00F0E6801122DFF8B4C284F892
:10CD8000502003F1630E03F15302664610685168A8
:10CD9000083203C67245B446F7D1DFF898C203F1F2
:10CDA000230203F1330E664610685168083203C649
:10CDB0007245B446F7D1DFF880C203F1330203F1C4
:10CDC000430E664610685168083203C67245B44681
:10CDD000F7D1DFF84CC203F14302533366461068C3
:10CDE0005168083203C69A42B446F7D1236894F8D2
:10CDF000E72094F8D8107D489847236894F8D72006
:10CE000094F8C8107A489847236894F8C72094F893
:10CE1000B81078489847236894F8B72094F8A81079
:10CE200075489847069BA16B9A687448A26323686B
:10CE30009847069B94F8FF101A7C7148C2F30302CE
:10CE400084F8FF2023689847069B94F8FE101A7C0C
:10CE50006C48C2F3021284F8FE2023689847069BB0
:10CE60000026587CFFF77AFB069BD4F8F0105B7C19
:10CE70006548012B98BF0023C4E93D6698BF84F83C
:10CE80000631C4F8F0602368984723685F489847E4
:10CE900094F83130069813F0FD0F00F1120018BF1E
:10CEA00084F8316084F8326084F8336000F048FA26
:10CEB000236857489847FDF76DF8012384F835300B
:10CEC000FFF7CAF880220646696918300AF07FF831
:10CED0000023069AC6F88030C6F8982094F83520CA
:10CEE0007372327533709DF80C202B78F273737067
:10CEF000029AE36B86F80CB086F80D8086F80EA0D7
:10CF00003261002B67D03146686898476420F4F797
:10CF100071F93046FFF7B0F892E6B9F1110F0CD174
:10CF2000069B93F8226023680EB13A4816E73A4808
:10CF30009847102384F8503013E77D213748F5F7E0
:10CF400035FF0EE71022DFF8E8C084F8502003F127
:10CF5000630E03F15302664610685168083203C637
:10CF60007245B446F7D1DFF8CCC003F1230203F1D8
:10CF7000330E664610685168083203C67245B446DF
:10CF8000F7D1DFF8B4C003F1230203F1330E664694
:10CF900010685168083203C67245B446F7D1204E76
:10CFA00003F123023333B446106851680832ACE809
:10CFB00003009A426646F6D11A4E1B48336896F82B
:10CFC000E72096F8D8109847336896F8D72096F857
:10CFD000C810164825E73046FFF774F830E600BF62
:10CFE00096DD0108BDDD010850DE01087EDE010886
:10CFF000C0DE010802DF010844DF010802E0010889
:10D000002FE001085DE001088EE00108BEE00108A4
:10D01000E7E00108DDDD0108FDDD01087CDC010839
:10D0200060010020B800002086DF0108C4DF01088D
:10D030009001002080010020700100204378827858
:10D040001B02007843EA024303430A20B3FBF0F0DB
:10D050007047000038B5044681B10D7884B1A36AE9
:10D06000012B0DD1E36A1BB95D210648F5F79EFE41
:10D07000E36A5878431B5842584138BDFF25EDE715
:10D080000020FAE778E10108044B93F8252083F8A3
:10D09000FF209A6AC3F80021704700BFB800002043
:10D0A000024B93F8242083F8FD207047B80000203D
:10D0B000024B93F8232083F8FC207047B80000202F
:10D0C000054B93F8242093F8FD1091423ABF0120BC
:10D0D00083F8FD2000207047B8000020064A92F82F
:10D0E000FC3092F8231099423DBF03F1FF33012039
:10D0F00082F8FC3000207047B800002010B5FFF720
:10D10000C3FF0120FDF79CF95023164C0121237029
:10D110000023224614486370FDF70CF918B9322138
:10D120001248F5F743FE50230121114A1148A3701C
:10D13000E170FDF7FFF818B936210C48F5F736FE17
:10D140005023237102230C4A01210C486371FDF71F
:10D15000F1F828B9BDE810403A210448F5F726BE99
:10D1600010BD00BFF8500020043F0D0078E1010819
:10D17000FA500020CC3F0D00FC50002094400D00E0
:10D18000836A10B5012B044608D1C36A1BB94B2131
:10D190000348F5F70BFEE36A587810BD0020FCE762
:10D1A00078E1010807B502A901F8010D0448FCF770
:10D1B0001BFF08B1FDF782F803B05DF804FB00BF68
:10D1C00055D000082DE9F8431746C7F30312052A86
:10D1D000044689464FF000052FD91A4B07F00F017E
:10D1E0001B68194898474FF000084FF47A76B9FB4E
:10D1F000F6F63046FDF716F808B10F2C20D9114B82
:10D2000049461B6811489847002368F3000563F3FB
:10D21000410505F00303032B0CD12046FFF7C2FFA5
:10D220000B4B012103EB4402547003F81470304699
:10D23000FDF780F82846BDE8F8834FF00108D4E7F1
:10D240000123E2E7B800002002E2010822E201081F
:10D25000F85000200F282DE9F04105460F461FD851
:10D26000164B03EB40035C78231A5C425C414FF49D
:10D270007A78B7FBF8F0FCF7D5FF4FF0000360F3C6
:10D28000000364F3410303F00303032B064609D0B4
:10D290004FF0000066F3000064F34100BDE8F08148
:10D2A0000024E4E72846FFF77DFF044A012102EB52
:10D2B000450208FB07F0FDF73DF8E9E7F8500020CC
:10D2C0002DE9F743194D01462B6804461848984745
:10D2D0000023184FDFF86080DFF860908DF807308A
:10D2E0009DF807300F2B02D903B0BDE8F0830DF194
:10D2F00007013846FCF778FE064648B1E2072B687E
:10D300009DF807100BD5484698473046FCF7B4FF08
:10D310009DF80730640801338DF80730E0E7404698
:10D3200098473046FCF786FFF2E700BFB8000020C0
:10D33000BDE1010855D00008EAE10108D3E1010888
:10D3400038B504460320FFF72DFF0420FFF72AFF1E
:10D350000520FFF727FF0620FFF724FF0720FFF730
:10D3600021FF2046FFF76AFE0546FCF75BFF48B148
:10D370005023294A01219371032306325370284612
:10D38000FCF7D8FFE01CFFF759FE0546FCF74AFF03
:10D3900048B15023204A01211372042308325370EC
:10D3A0002846FCF7C7FFA01DFFF748FE0546FCF71F
:10D3B00039FF48B15023184A0121937205230A32DC
:10D3C00053702846FCF7B6FF04F10900FFF736FE5C
:10D3D0000546FCF727FF48B150230F4A012113737C
:10D3E00006230C3253702846FCF7A4FF04F10C000E
:10D3F000FFF724FE0446FCF715FF58B15023064AF8
:10D40000204693730723D3730121BDE838400E32C1
:10D41000FCF790BF38BD00BFF85000200738C0B2FD
:10D4200005289ABF014B185C082070472FE10108BE
:10D4300006289ABF014B185C0020704735E10108AF
:10D44000052804D90628034818BF00207047024861
:10D45000704700BF90D0030048E80100072810B5CE
:10D46000044604D940F243110348F5F79FFC034BEF
:10D4700013F9240010BD00BF78E101083CE1010868
:10D48000142810B5044613DD4FF4A4711148F5F7C4
:10D490008DFC062C14DD082C14DD0A2C14DD0C2C5C
:10D4A00014DD0E2C14DD152CB4BF0020082010BD97
:10D4B000022803DD0428ECDC0620F8E70720F6E765
:10D4C0000520F4E70420F2E70320F0E70220EEE76E
:10D4D0000120ECE778E1010808B50F280DD8DFE856
:10D4E00000F0181818081A1A1A0A0A0C0C0C0C0C5E
:10D4F0000C0A732008BD0020FCE74FF4C1710748F7
:10D50000F5F754FC064B074A40F28311034809F033
:10D510000BFC3320EEE7DE20ECE700BF78E10108EA
:10D52000B6A001085CE101082DE9F04F8DB01E4660
:10D53000169F364B81469F428A46934608D0344B0D
:10D540009F4203D0A6213348F5F730FC002100E0CC
:10D550000121314D0B91EB6A9847EB685046984793
:10D56000B9F1010F4FF000040A95DFF8B8800B996C
:10D5700028D108230A22CDE90132AB693246CDE930
:10D580000644CDE90444039400941D4602204B4612
:10D59000CDE90899A8472146FF2004F001F9D8F801
:10D5A000004053463A4631461C48A047082004F044
:10D5B000EDF8342139200A9B1B6C0A930DB0BDE8AD
:10D5C000F04F18474FF47A634FF00109CDE9074354
:10D5D0000823CDE901930A9B2246DB69CDE9054486
:10D5E000CDE903491D4600960B4602205946A8473F
:10D5F0004946FF2004F0D4F8CDF800B0D8F8004038
:10D6000053463A4631460648A047CFE790D003003C
:10D6100048E801003BE201085CF101087DE20108F5
:10D62000AFE20108B80000202DE9F341044610469E
:10D6300015460E469846FFF703FF07462846FFF7B4
:10D64000F7FEC5B21DB9C5210948F5F7AFFB64B9AE
:10D650004046FFF703FF024600972B46314620461F
:10D66000FFF762FF02B0BDE8F0810022F4E700BFDF
:10D670003BE201080A680368534003604A68436854
:10D68000534043608A68836853408360CA68C368B4
:10D690005340C36070470B6810B514686340036063
:10D6A00054684B686340436094688B686340836050
:10D6B000CB68D2685340C36010BD0000A1F11003D5
:10D6C000DBB2102B2DE9F0470C46154608D84FF079
:10D6D000010909FA03F303F0013323F080732BB936
:10D6E0000023FF2085F8F030BDE8F0870A460146A8
:10D6F000284609F06CFC04F11C0E4FEA8E0E5FFA0E
:10D700008EFE4FEA1E13013B85F8F0302346274971
:10D71000B3FBF4F204FB1232E81812F0FF0210F827
:10D7200004AC10F803CC10F8027C10F8016C32D174
:10D7300011F80C804FEAD91289EA080811F807C0DD
:10D740008F5D11F80A604FEA420A5244C24602EB6A
:10D75000C20282EA49025FFA82F91A1BD2B215F8B4
:10D7600002802A448AEA080A05F803A092F8018098
:10D7700004338CEA080C80F801C092F802C0DBB2D6
:10D7800087EA0C078770D2789E4586EA0206C67043
:10D79000BED80020A8E7182CDFD9102A01BF11F845
:10D7A0000AA011F80CC0CF5D8E5DD6E7ECE401084D
:10D7B0002DE9F04F92F8F030A1B01A911892002B99
:10D7C00000F05D8101461CA8FFF765FF4FF00108DE
:10D7D000AC4CAD4DAD4E189B9DF875E003EB0813B6
:10D7E00019939DF870309DF87AA00093009A9DF8E7
:10D7F0007F90A05C9DF8742014F80A100192019F9C
:10D800009DF87920E75D02920697029F9DF87E20A1
:10D81000E75D03920797A25C9DF8787004920897E1
:10D820009DF873209DF87D70059214F8093014F866
:10D830000EC0A25C09979DF872700A97E75D0B977E
:10D840009DF877700C97E75D0D97089FE75D0E9741
:10D85000099FE75D0F979DF87C7010979DF8717098
:10D8600011979DF876701297E75D13979DF87B707E
:10D870001497E75D1597109FE75D1697119FE75D79
:10D880001797189F97F8F07047453ED88DF87000AD
:10D890009DF818008DF872108DF874009DF82C100A
:10D8A0009DF838008DF87A108DF878009DF81010EA
:10D8B0009DF858008DF876108DF87C009DF84C107E
:10D8C0009DF81C008DF87E108DF875009DF85410A1
:10D8D0009DF83C008DF87F108DF879009DF834108C
:10D8E0009DF85C008DF87B108DF87D008DF8772019
:10D8F0001A98199A1CA98DF871C08DF87330FFF72A
:10D90000CAFE002021B0BDE8F08F81EA03071B9713
:10D91000009F434015F807B01B9F80EA0C008BEA7C
:10D92000070716F80EB081EA0C0187EA0B078DF89D
:10D93000707015F80E707B4016F80A707B408DF8F9
:10D94000713015F80A30584016F809305840009BDD
:10D950008DF8720016F803C0049B8CEA010115F8DB
:10D9600009C0534081EA0C018DF8731001991CA87D
:10D97000695C4B400299715C4B408DF87430069B9A
:10D980005A40029BEB5C5A40039BF35C5A408DF873
:10D990007520DDE906325340039AAA5C5340059A8C
:10D9A000B25C53408DF87630079A049B5340019A3D
:10D9B000B25C5340059AAA5C53408DF877300D9ABB
:10D9C0000B9B5340089AAA5C5340099AB25C53409F
:10D9D0008DF87830DDE90D325340099AAA5C534046
:10D9E0000A9AB25C53408DF87930DDE90E3253402B
:10D9F0000A9AAA5C53400C9AB25C53408DF87A3074
:10DA00000B9B0F9A5340089AB25C53400C9AAA5C45
:10DA100053408DF87B30159A139B5340109AAA5CA3
:10DA20005340119AB25C53408DF87C30DDE91532D9
:10DA30005340119AAA5C5340129AB25C53408DF83D
:10DA40007D30DDE916325340129AAA5C5340149A95
:10DA5000B25C53408DF87E30179A139B5340109A56
:10DA6000B25C5340149AAA5C199953408DF87F30E8
:10DA7000FFF700FE08F101035FFA83F8ABE6FF2031
:10DA800040E700BFECE40108ECE20108ECE3010828
:10DA90000068704782B0034660B16A465968006802
:10DAA000013B03C207221DF8021012F1FF3203F8F6
:10DAB000011FF8D202B070470FB404B070470000E5
:10DAC00030B585B06D4685E80F00104C95E80F0025
:10DAD00084E80F0004F1100208A903C982E80300DA
:10DAE0000BB90B4BE360A3680BB9094BA3606368E8
:10DAF0000BB1236833B9A36806489847064B6360A7
:10DB0000064B23600123237605B030BDD44B0020A3
:10DB1000B9DA000862E60108616F0108516F010877
:10DB20002DE9F041184D80462B7E0E461BB973211E
:10DB30001648F5F73BF9DE2E03D974211348F5F7A3
:10DB400035F92B6880209847044680B18022002157
:10DB500009F061FAB8F1000F12D08EB12B6830468F
:10DB60009847074630B920466B6898473C462046A0
:10DB7000BDE8F0813246414609F029FA2677A766CA
:10DB800000236370F3E700BFD44B002015E60108C3
:10DB900070B50A4C0546237E1BB98F210848F5F75E
:10DBA00005F955B1A86E636810B198470023AB66BC
:10DBB00063682846BDE87040184770BDD44B00200C
:10DBC00015E601082DE9F0479C4B17461A7E92B0E6
:10DBD00005460E4698461AB9A7219948F5F7E6F882
:10DBE000032F01D80024D8E02A786B7843EA421347
:10DBF00033702B78022B02D0042B40F08D80002351
:10DC0000042F8DF82630EDD06B6873706B681B0A9B
:10DC1000B370EB88F370EB7933716B68CDF8223019
:10DC20009DF82630002B40F0C180052FDAD0062465
:10DC30002A7AC2F3400302F001019B0143EAC113B7
:10DC400043EA1213C2F3800243EA4213737195F858
:10DC500008904FEA1919631C9F42C3DD6A89DBB241
:10DC600032556A890234120AF254D8F810301A88F0
:10DC70006B899A4204D040F247117148F5F796F843
:10DC8000D8F81420D8F8103011781B6810290A939E
:10DC90000DD902930DF1220301930123297A0093F8
:10DCA00058320023090905F10C0000F0E5FCB9F138
:10DCB000000F0BD004EB090A574593DB30194A4695
:10DCC00005F10C0109F083F95FFA8AF42B7F002B30
:10DCD00077D0BC4286D26B7F04F1010933556A7F4D
:10DCE0005FFA89F9D8F81430002A68D158330693BE
:10DCF000AB6E06A907932B7F06EB0900ADF8203029
:10DD000000F0ACFB4844C4B2A7425AD240F27511AD
:10DD10004B48F5F74BF865E7032B01D0052B01D1F4
:10DD200001236DE7002B3CD1082F7FF65BAFD8F8BD
:10DD30001440701C224652F8083FC6F80130536860
:10DD40004360FFF7A7FE102F7FF64CAF224652F834
:10DD5000103F06F10900C6F8093053684360FFF729
:10DD600099FE122F7FF63EAFB4F8983006A973746F
:10DD7000B4F8983005A81B0AB37413232834CDE9EE
:10DD80000646ADF8203000F033FB162F7FF62AAFA1
:10DD90001724059BC6F813306B66204612B0BDE809
:10DDA000F087D8F80C30274898471BE740F23D1120
:10DDB0002348F4F7FBFF4FF0000905244BE78833B5
:10DDC00095E7E31C9F427FF70DAFD8F814301A781F
:10DDD000102A0DD1783306A905A8CDE90636ADF88D
:10DDE000204000F06CFA059B33510434E4B2D4E7D0
:10DDF000112A1DD103F1780268330B930DF1220330
:10DE00000F930A9B0BA91093B5F87A3005A8ADF8CB
:10DE1000443095F87C300C928DF8463095F87D3082
:10DE20000D968DF84730ADF8384000F080FADAE70B
:10DE30004FF4CB710248F4F7B9FFAEE7D44B0020A2
:10DE400015E60108ECE501082DE9F04F8F4DA3B070
:10DE50002B7E06460F46904623B940F2A3118C480C
:10DE6000F4F7A4FF022F2CD92B6880209847044692
:10DE700030B9EB6887489847204623B0BDE8F08F5B
:10DE80008022002109F0C7F833785B0923703278CB
:10DE9000072B02F00302627003D1EB687E489847BB
:10DEA0000CE0B8F1000F00F0EF81012B40F0C581CC
:10DEB000AB687A48F3E74246794898476B68204652
:10DEC00098470024D8E701F18802A0E1F3465068A2
:10DED000227A4FEADC1E6EF300024FEA5C1E6EF3FC
:10DEE00082024FEA1C1E6EF3C3026CF30712227209
:10DEF00082B24A454FEA104C84BF0CF1010C1FFA64
:10DF00008CFC09EB0C4906EB0800CDF83090FFF7CC
:10DF1000BFFD0DF1880A68314AF8681D60665146F8
:10DF200007A800F0CCF9079B626E934204D0EE681C
:10DF30005C495D48B047C1E72A6909F10101BBF1BD
:10DF4000000F2CD05160227A04F10C0304931309C2
:10DF50001A4606F108010498059309F038F86A6931
:10DF6000117810290CD90DF12A0101910021CDF869
:10DF7000089000915B46DDE90401583200F07CFB1B
:10DF8000237A1B0903F10C0297422DD903F10D02EC
:10DF9000974206D1002345482377EB686BE79160F1
:10DFA000D1E70933A8EB0300617FC0B220776A692B
:10DFB00061B958321E4408920996ADF828002B68C2
:10DFC0009847A06620B9EB68394868E78832F1E7DE
:10DFD000514600F043FA00283FF74EAFEB68354852
:10DFE00098476B68A06E5AE700232377A36643E740
:10DFF000212F01D101232AE1EB682F484FE79DF83B
:10E000003F30043F09EB0700DB09FFF741FD6E6974
:10E010006066A3B30DF1580A00213022504608F083
:10E02000FAFFFF2332468DF8583052F8083F0DF1C1
:10E030005900CDF8593053683836CDF85D30FFF7C8
:10E0400029FDB6F860303A468DF8613049461B0A22
:10E050000DF163008DF8623008F0B9FFCDE9086A70
:10E0600008F1070808A907A8ADF8288000F0C0F952
:10E07000636E079A9A4223D0EB6810480FE7283660
:10E08000CDE90869A8F10408ECE700BFD44B0020F3
:10E0900015E601088FE60108A7E60108D5E60108A4
:10E0A00024E701089EAF01085FE70108A4E7010823
:10E0B000D8E701080AE8010830E80108A2E80108E9
:10E0C0009DF837609DF83630360446EA03269DF801
:10E0D00035300DF13B001E4366609DF83A709DF8A7
:10E0E00039303F0447EA03279DF838301F43A760C3
:10E0F000FFF7CEFCE0609DF83F20237CD10961F35F
:10E10000C713110961F3061362F3030323749DF827
:10E110004030637494F8213003B322AB33F8472DB9
:10E120009B786282237522AB33F8442D9B78A4F848
:10E130001520E37522AB33F8412D9B782283A3761B
:10E1400022AB33F83E2D9B78A4F81B20637722ABDB
:10E1500033F83B2D9B78E28384F820306D6994F985
:10E16000102005F1280C002AB5F8981004F12300BE
:10E1700004F15303CDF858C016AA12DA05F11807B6
:10E18000ADF868100092083504F1430204F1330140
:10E19000CDE91776199500F0FCF9012384F82230B7
:10E1A0006AE6ADF864101946CDE9176700F0B0F9DA
:10E1B0000023F3E7EB68394871E6701CFFF768FC51
:10E1C000804501466060EB687FF475AE4146344897
:10E1D00098470023052F6377A7F1040807D97379BF
:10E1E00003F00F0308339845C4BFF35C6377F379FA
:10E1F00096F8069096F805C049EA0329637FA4F8CB
:10E200000A906969002B7FF45EAE01F158024FF06D
:10E21000010E0878CDE9082662681028CDF82A207A
:10E22000ADF828808DF82EE02A6902D9002B7FF402
:10E230004DAE90684FF0000B4AE6032BBDD0052B86
:10E24000BBD0012BB6D1112F7FF4D2AE002384F8BE
:10E2500021306B691FFA87F828330893731C0993E0
:10E2600008F1FF33ADF82830337808A90DF13500F7
:10E270008DF8343000F0D4F800280DF134093FF760
:10E28000BEAEEB6807480AE6032B01D0052BD8D1B8
:10E29000701CFFF7FDFB60609BE700BFD7E801083B
:10E2A000F4E601087FE801080022FFF7CDBD0B0A64
:10E2B000017043700B0C090E8370C170704770B50C
:10E2C0001025CEB00C462A4606460021684608F0C6
:10E2D000A2FE49238DF80030A37BD4F80A100DF17B
:10E2E00006008DF80530FFF7E2FF21690DF10A0005
:10E2F000FFF7DDFF238908A88DF80F3000F000FA42
:10E30000216808A800F00CFA2A46694608A800F01F
:10E310000DFA2289616808A800F008FA08A90DEB37
:10E32000050000F06EFA049B33604EB070BD4923C7
:10E3300070B500250C460646CEB08DF800300B8B2C
:10E34000CDE901558DF801301B0A8DF802308B7E26
:10E3500003958DF80330CB7E0DF106008DF8043067
:10E360000B691968FFF7A3FF61690DF10A00FFF758
:10E370009EFFA38908A88DF80F308DF80E5000F08D
:10E38000BFF9216808A800F0CBF9694608A8102257
:10E3900000F0CCF9A289A16808A800F0C7F908A983
:10E3A00004A800F02EFABDF8103008A833808DF8CC
:10E3B00004508DF803508DF802508DF8015000F094
:10E3C0009FF9616808A800F0ABF9694608A8102217
:10E3D00000F0ACF9A289A16808A800F0A7F908A983
:10E3E00004A800F00EFABDF8103073804EB070BD76
:10E3F00030B50C46CBB0054604A800F081F9216881
:10E4000004A800F08DF92289616804A800F08EF953
:10E4100004A9684600F0F5F9009B2B604BB030BDB5
:10E4200070B50C89BEB006460D46A4B114F00F04B9
:10E4300011D101AA10212868FFF740F92889A042CC
:10E4400001DC3EB070BD68683119204401AAFFF7B5
:10E45000AFF91034F2E74FF0FF30F2E72DE9F04367
:10E460000F89C7B081460D46002F4ED001241022DF
:10E470004FEA1718002117F00F0701A818BF08F17D
:10E48000010808F0C8FDAB7BD5F80A100DF10A00B1
:10E490008DF809308DF80440FFF709FF29690DF167
:10E4A0000E00FFF704FF6E68013E444503DD288936
:10E4B00047B0BDE8F08309AA102128688DF8134001
:10E4C000FFF7FCF809AA05A901A8FFF771F944456F
:10E4D00010DB002F14BF3B46102330464A464B4406
:10E4E0000DF1130C934207D80134A4B209F11009BD
:10E4F0001036DAE71023F0E710F801EF1CF8011FDF
:10E5000081EA0E0102F8011BECE74FF0FF30CFE784
:10E5100070B5C2B0144606460D46F122002105A88A
:10E5200008F079FD0023CDE90333636810218DF8ED
:10E5300005301A0A1B0C8DF80730A3688DF80620E9
:10E540008DF808301A0A1B0C8DF80A30A3898DF853
:10E5500009208DF80B301B0A8DF80C30012305AA19
:10E5600020688DF80430FFF7A9F805AA314601A804
:10E57000FFF71EF9022305AA102120688DF8043048
:10E58000FFF79CF805AA294601A8FFF711F942B048
:10E5900070BD2DE9F0431025C3B04A9C80460F465C
:10E5A00016460021F12205A8994608F034FD2A46B6
:10E5B000002101A808F02FFDA26829468DF805204A
:10E5C000130AEA408DF80720E2688DF80630D37907
:10E5D00020688DF8083093798DF8093053798DF8DB
:10E5E0000A3013798DF80B30D3788DF80C3093788E
:10E5F0008DF80D3053788DF80E30137805AA8DF80C
:10E600000F30238A8DF810301B0A8DF8113001234A
:10E610008DF80430FFF752F805AA414601A8FFF72C
:10E62000C7F8022305AA294660688DF80430FFF771
:10E6300045F805AA494601A8FFF7BAF8032305AA39
:10E64000294620688DF80430FFF738F805AA3946C6
:10E6500001A8FFF7ADF8042305AA294620688DF824
:10E660000430FFF72BF805AA314601A8FFF7A0F800
:10E6700043B0BDE8F0830000F0B50F29C7B00446F1
:10E680000D4616461F4604D94FF4A1711B48F4F7F6
:10E690008DFB0123002F019318BF02238DF8083052
:10E6A0009DF830310DF10A0083F001038DF8093037
:10E6B0004D9B1968FFF7FBFD4E990DF10E00FFF71A
:10E6C000F6FD4FF4807309AA1021304605AEADF86F
:10E6D0001230FEF7F3FF09AA314601A8FFF768F8E8
:10E6E0000023601EDAB2954201D847B0F0BD10F8A1
:10E6F000012FF15C01334A400270F3E711E9010890
:10E7000010B5102204460021F13008F084FC0021ED
:10E710002046C4F81411F022BDE8104008F07BBC7C
:10E720000B46024610211846FEF7C8BF2DE9FF47E9
:10E730000446D0F814010E46154604F2011920B320
:10E74000C0F110089045474628BF174648443A464E
:10E7500008F03DFCD4F814313B440F2BC4F81431BD
:10E760001ED9A8451CD204F1F103194613F8012B58
:10E77000D87B4B4582EA000203F8012CF6D12246F1
:10E780000846FFF715F83E44ED1B0DF1100A102D59
:10E7900009D82A463146484608F019FCC4F81451F5
:10E7A00004B0BDE8F08704F1F002731E06F10F001B
:10E7B00013F8017F12F8011F834281EA07011170EB
:10E7C000F6D16A4604F1F103984617469446186854
:10E7D00059680833ACE803004B456246F6D122463F
:10E7E00039463846FEF7E4FF43463A4603CA5245E7
:10E7F00018605960174603F10803F6D11036103D32
:10E80000C5E7F0B50C4689B01022002105466846E0
:10E8100008F001FC224669466846FEF7C9FF9DF9EB
:10E8200000306A46002B0DF10F0140DA137812F820
:10E83000010F5B005BB243EAD013914202F8013C46
:10E84000F4D19DF80F305B0083F087038DF80F3013
:10E85000D4F81431102B39D1002304F201121178AD
:10E860001DF8030001334140102B02F8011BF6D1C3
:10E8700004F1F102134604F2011712F8011BD07BD8
:10E88000974281EA000102F8011CF6D104AA9446DD
:10E89000164618685968083303C6BB423246F7D19A
:10E8A000224629466046FEF783FF09B0F0BD137883
:10E8B00012F8010F5B005BB243EAD0138A4202F800
:10E8C000013CF4D19DF80F305B00BFE79DF90020BB
:10E8D0006846002A28DA027810F8016F520052B216
:10E8E00042EAD612814200F8012CF4D19DF80F20A3
:10E8F000520082F0870280218DF80F20E21882F802
:10E900000111002201330F2B1DD9C4F8143100234B
:10E9100004F2011211781DF8030001334140102B5D
:10E9200002F8011BF6D1A3E7027810F8016F52003C
:10E9300052B242EAD612814200F8012CF4D19DF87D
:10E940000F205200D7E7E11881F80121DAE7000033
:10E95000002103E00A4B5B584350043109480A4B3D
:10E9600042189A42F6D3094A02E0002342F8043BD7
:10E97000074B9A42F9D300F00DF8F1F7E7FF704723
:10E9800044F90108000000207804002078040020E9
:10E99000A0510020314B82B01A6842F480721A6094
:10E9A00099682F4A0A409A601A6822F0885222F029
:10E9B00001121A601A6822F480221A609A6822F4FE
:10E9C0007D029A600022DA6001921B6813F40073E2
:10E9D00018BF01230193019B012B37D14FF48051C4
:10E9E000204B1A68A3F5806322F00102C3F80024CB
:10E9F000D3F8002422F00202C3F80024D3F8002444
:10EA000022F00402C3F800245A6A42F080525A628B
:10EA1000154A11605168C906FCD49A689A609A68D0
:10EA20009A609A689A605A6822F460425A605A68FA
:10EA300042F440425A609A6822F003029A609A684F
:10EA40009A60064A936813F00C0FFBD14FF00062F6
:10EA5000064B9A60064ADA6002B0704700380240FE
:10EA60000CC0FF88003C02400070004000ED00E058
:10EA70000003FA0570B5064688B02E4801F030FC58
:10EA80002D4B1A680092009A91073CD501214FF452
:10EA9000007001F07FFE012001F072FC274A5368EC
:10EAA00043F400335360A2F5374253681B07FCD58B
:10EAB0000024012502A801F04DFC02A91D488DF893
:10EAC0000D4006948DF81C508DF80C4001F01CFC94
:10EAD0002A4606233146174801F05EFC29461548B0
:10EAE00001F044FC0221134801F0E8FC114801F058
:10EAF000D7FC134D01940F4C0221204601F0D8FCA5
:10EB000058B108B070BD1A6842F001021A60009A4C
:10EB10009207BBD41A680092F9E7019B0133019375
:10EB2000019BB3F5805FE7DB38212846F4F73EF917
:10EB3000E2E700BF00240140003802400027014006
:10EB400064E9010808B5002001F01AFC002107481B
:10EB500001F00CFC00214FF4007001F01BFE044A90
:10EB6000136823F00103136008BD00BF00240140B7
:10EB70000038024013B5072301220146114801F075
:10EB80000BFC02210F4801F099FC0E4801F088FCB3
:10EB900000230D4C019302210A4801F089FC28B1A1
:10EBA000084802B0BDE8104001F07FBC019B013372
:10EBB0000193019BB3F5805FEDDB4C212046F4F718
:10EBC000F5F8E8E70024014064E9010870B506465D
:10EBD0000825FFF74FFF00243046FFF7CBFF013D2C
:10EBE0000444F9D1FFF7AEFFC4F3CF0070BD0000BD
:10EBF00008B51120FFF7EAFF07F078FC0146084846
:10EC000007F080FD07F05AF803A3D3E9002307F0CB
:10EC1000ADF807F065FB08BD2FDD24068195F33FB5
:10EC200000F07F450F4A536A43F0805353620E4B06
:10EC30001A465968C906FCD41B68022823F4C0533D
:10EC400006D143F4C05313605368DB06FCD470470D
:10EC5000012802D143F48053F5E70028F3D143F4AF
:10EC60000063F0E7003802400070004010B50C4B24
:10EC70005A68D206FCD41C6814F4C05F0BD114F49B
:10EC800080500AD114F4006404D106482A21F4F714
:10EC90008DF8204610BD0220FCE70120FAE700BFF6
:10ECA00000700040B2E9010838B50546012001F0C6
:10ECB00015FC022D01BF144A136843F001031360D1
:10ECC000124B1A6842F480721A601A689205FCD5D9
:10ECD0005A6822F4604242F440425A6000229A602C
:10ECE0000A4B9C6814F00C04FBD14FF480721A603C
:10ECF000074B084A28461A60FFF794FF2046BDE8F4
:10ED0000384001F0DFBB00BF003C02400038024049
:10ED1000F0010020D0FE3F000C4B5A6B900513D43D
:10ED20005A6A42F080525A62094A116841F480716D
:10ED30001160596B41F480715963596B8905FCD599
:10ED4000136823F480731360704700BF00380240DB
:10ED500000700040054B5A6B910706D45A6B42F085
:10ED600001025A635A6B9207FCD570470038024083
:10ED7000094B5A6A42F020025A629A6942F0200214
:10ED80009A619A6922F020029A610022A3F5093360
:10ED90001A801A855A6270470038024015210238DD
:10EDA000002248430121064B1A85D86299825A6293
:10EDB0001A8219801A8AD207FCD500221A8070475D
:10EDC00000140040002349F6FE7282B00193019BBB
:10EDD000934201DD02B07047019B01330193F6E7D6
:10EDE000002340F6FE7282B00193019B934201DD45
:10EDF00002B07047019B01330193F6E7002382B014
:10EE00000193019BB3F5CC7F01DD02B07047019BFC
:10EE10000133F5E7D0B1012801D1FFF7EFBF0C4B6B
:10EE200000211A684FF47A73B2FBF3F2094B013AEE
:10EE300092B21A8501220138D8629A8259621982E7
:10EE40001A801A8AD207FCD500221A80704700BFA8
:10EE5000F00100200014004000F1774303F578032F
:10EE6000B3F5804F2DE9F04106460C4617462DD2EA
:10EE700002F1F73303F608030344B3F5804F25D2BC
:10EE8000FFF7F4FE804610B10020FFF7CBFE01F043
:10EE90003DFB01252744361BA7420AD101F046FB62
:10EEA000B8F1000F02D04046FFF7BCFE2846BDE88F
:10EEB000F08141F6027001F041FB301914F8011B9A
:10EEC00001F098FB042818BF0025E5E70025EDE7D1
:10EED00010B50C4600F1774101F57801B1F5804F8E
:10EEE0000DD202F1F73303F608030344B3F5804F64
:10EEF00005D20146204608F06AF8012010BD002026
:10EF0000FCE7000008B5114B984215D003F580636B
:10EF1000984213D003F58063984211D003F58063C3
:10EF200098420FD003F5006398420DD0084B094A70
:10EF30001421094807F0F8FE002008BD0120FCE775
:10EF40000220FAE70320F8E70520F6E70000024078
:10EF500049EA010803EA010862EA01080F2808B536
:10EF600005D9094B094A3B21094807F0DDFE012379
:10EF700003FA00F0C043074A51680140516013682A
:10EF80001840106008BD00BFB3EA01080DEA01088F
:10EF900062EA0108000401400F292DE9F84F82467A
:10EFA0000D4693461F4605D95A4B5B4A54215B4890
:10EFB00007F0BAFE4FF0010909FA05F900F0B8F8B8
:10EFC0006FEA0903564E032D7268564C02EA03029B
:10EFD0007260326803EA0203534A3360136A43F0F3
:10EFE000010313622ED80F22A3684FEA850802FAA4
:10EFF00008F223EA0203A3605046FFF783FFA368E9
:10F0000000FA08F01843A0601BF0020F18BFB368A5
:10F01000464A1CBF43EA0903B3601BF0040F1EBF3E
:10F02000F36843EA0903F360336843EA0903336092
:10F030003B01DBB2002D45D182F80633402313603B
:10F04000BDE8F88F072D13D80F22A5F10408E36857
:10F050004FEA880802FA08F223EA0203E360504606
:10F06000FFF750FFE36800FA08F01843E060CBE7D1
:10F070000B2D13D80F22A5F1080823694FEA880841
:10F0800002FA08F223EA020323615046FFF73AFF2F
:10F09000236900FA08F018432061B5E70F22A5F1B3
:10F0A0000C0863694FEA880802FA08F223EA0203AF
:10F0B00063615046FFF726FF636900FA08F01843C2
:10F0C0006061A1E7012D03D182F807338023B6E701
:10F0D000022D04D182F808334FF48073AFE7032D7B
:10F0E00004D182F809334FF40073A8E7042D04D14A
:10F0F00082F80A334FF48063A1E7092D04D882F81F
:10F1000017334FF400039AE782F828334FF48073E3
:10F11000536095E7BFEA010828EA010862EA01089E
:10F1200000040140000001400038024000E100E01E
:10F13000144B984205D1144AD36943F00103D361BB
:10F140007047124B984204D10F4AD36943F002032F
:10F15000F5E70F4B984204D10B4AD36943F00403FF
:10F16000EDE70C4B984204D1074AD36943F00803FA
:10F17000E5E7094B9842E3D1034AD36943F0200302
:10F18000DDE700BF000002400038024000040240FA
:10F1900000080240000C0240001402400323490012
:10F1A00010B584688B4024EA030484600124022A99
:10F1B00004FA01F407D0032A0DD0012A07D183688D
:10F1C0002343836003E083688A401A438260836834
:10F1D0001C43846010BD82681343F2E70F29F8B521
:10F1E00004460F4615461E4603D940211948F3F739
:10F1F000DDFD2046FFF79CFF03237A009340DB43AD
:10F200002168194021600121D4F800C001FA02F000
:10F210004CEA000CB940C4F800C009B266B1A68837
:10F22000314389B2A180E168012D03EA0103E36063
:10F2300006D0022D08D0F8BDA68826EA0101F1E724
:10F24000E3680343E360F6E7E36805FA02F21A4372
:10F25000E260F0E70FEB01080F2970B505460C4698
:10F26000164603D960210E48F3F7A0FD2846FFF7A4
:10F270005FFF032361008B40DB43EA68012E02EA53
:10F280000302EA6005D0022E03D02A6813402B60E7
:10F2900070BDEA6806FA01F11143E960F5E700BFC5
:10F2A0000FEB01080F2910B505D9074B074A762146
:10F2B000074807F039FDFFF73BFF4B0003210268C9
:10F2C00099401143016010BDB3EA0108CBEA01087F
:10F2D0000FEB01080F2938B50446154605D97C21E6
:10F2E0001B4B1C4A1C4807F01FFD0F2A03D91B4B60
:10F2F000184A7D21F6E7FFF71BFF07294FF00F03A0
:10F3000018D8006A8A00934020EA03032362236A24
:10F3100005FA02F21A4322620322236849008A4056
:10F3200023EA020323600223226803FA01F1114356
:10F33000216038BDA1F10802406A9200934020EAA2
:10F3400003036362636A95401D436562E4E700BF9F
:10F35000B3EA0108DEEA01080FEB0108FCEA010844
:10F36000012303FA01F189B201837047012303FAF3
:10F3700001F189B241837047012303FA01F189B297
:10F380000AB10183704741837047008A084100F049
:10F39000010070470F2938B505460C4603D9A9214D
:10F3A0000548F3F703FD28686400E04000F003001F
:10F3B000431E5842584138BD0FEB0108808A08416E
:10F3C000C04300F00100704710B5084C23681BB91A
:10F3D0000120F3F75DF9206023682BB9BDE81040E8
:10F3E00036210348F3F7E2BC10BD00BFF04B00200C
:10F3F0005EEB010810B50B4C22681AB93C210A4893
:10F40000F3F7D4FC206842F21071F3F789FA01286F
:10F410000CBF0124002403D040210348F3F7C6FCAD
:10F42000204610BDF04B00205EEB010810B5074CE4
:10F4300022681AB94D210648F3F7B8FC002320686A
:10F440001A46BDE810401946F3F77EB8F04B00208D
:10F450005EEB010810B50446FFF7B6FFFFF7CAFFE1
:10F4600021461022034801F043FE0446FFF7DEFF69
:10F47000204610BD0054004010B5FFF7A5FFFFF770
:10F48000B9FF01F0EDFD0446FFF7D0FF204610BDA7
:10F4900008B513460A460146034801F05FFA0030FA
:10F4A00018BF012008BD00BF0054004008B5134636
:10F4B0000A460146034801F057FB003018BF0120FF
:10F4C00008BD00BF0054004008B513460A46014677
:10F4D000034801F0DBFB003018BF012008BD00BF6E
:10F4E0000054004008B513460A460146034801F09F
:10F4F0005DFC003018BF012008BD00BF0054004073
:10F5000008B513460A460146034801F0A7FC00303F
:10F5100018BF012008BD00BF005400400123064A67
:10F5200083405169194205D05361044B53F8203090
:10F5300003B11847704700BF00040140F44B00209E
:10F540000F2838B504460D4603D926210348F3F7A2
:10F550002DFC034B43F8245038BD00BFACEB010831
:10F56000F44B00200020FFF7D9BF0120FFF7D6BFE2
:10F570000220FFF7D3BF0320FFF7D0BF0420FFF71F
:10F58000CDBF08B50920FFF7C9FF0820FFF7C6FF68
:10F590000720FFF7C3FF0620FFF7C0FFBDE80840C4
:10F5A0000520FFF7BBBF08B50F20FFF7B7FF0E2000
:10F5B000FFF7B4FF0D20FFF7B1FF0C20FFF7AEFF00
:10F5C0000B20FFF7ABFFBDE808400A20FFF7A6BFFE
:10F5D000FEE7FEE7FEE7FEE7FEE7FEE7FEE7FEE703
:10F5E000FEE7FEE7FEE7FEE7FEE7FEE7FEE7FEE7F3
:10F5F000FEE7FEE7FEE7FEE7FEE7FEE7FEE7FEE7E3
:10F60000FEE7FEE7FEE7FEE7FEE7FEE7FEE7FEE7D2
:10F61000FEE7FEE7FEE7FEE7FEE7FEE7FEE7FEE7C2
:10F620000A23B0FBF3F203FB120040EA0210C0B25F
:10F6300070470000CA22024B5A6253225A62704736
:10F6400000280040014B1860704700BF344C002078
:10F650004FF400320F4B10B50F4C5A61E368DB05D5
:10F6600003D430210D48F3F7A1FBFFF7E3FF4FF47C
:10F670000072A36823F48853A360094BC3F8842065
:10F68000FF236362074B1B6813B1BDE810401847A6
:10F6900010BD00BF0004014000280040FAEB010843
:10F6A00000E100E0344C00202DE9F04F9846374B44
:10F6B00085B01B78824691469DF838709DF83C6075
:10F6C0002BB9334B334A8C21334807F02DFB431EB3
:10F6D0001E2B59D80C2957D8A2F5FA63632B53D89F
:10F6E000B8F1170F50D83B2F4ED83B2E4CD802F113
:10F6F0003000C0B2FFF794FF83460846FFF790FF43
:10F7000004465046FFF78CFF40F400554046FFF793
:10F7100087FF45EA0B4545EA042504463846FFF7CE
:10F720007FFF000240EA04443046FFF779FF2043A0
:10F730001A4CFFF77FFFE36843F08003E360E36860
:10F740005B06FCD565602060E36823F08003E3601E
:10F75000124BDA689206FCD5FF2204A85A6200F820
:10F760000C6D8DF807A08DF80810ADF809908DF894
:10F7700006808DF80570F9F7F0FF094BC3E9000129
:10F78000012005B0BDE8F08F0020FAE7384C0020DA
:10F790007BEC010848EC0108FAEB01080028004066
:10F7A000404C002037B50578C4788378B0F8052040
:10F7B00001790195407800902046FFF775FF03B06E
:10F7C00030BD000038B52B4B04461B781BB9E42133
:10F7D0002948F3F7EBFA294AD36823F02003D360D2
:10F7E000D3689B06FCD513685268C2F30741080929
:10F7F00000EB800001F00F0101EB4001C9B201F5FF
:10F80000FA61A4F80510C2F30721C1F300108500C6
:10F81000284401F00F0101EB4001D2B22171C2F383
:10F82000011101EB810102F00F0202EB4102E270D3
:10F83000C3F30742C2F3011101EB810102F00F0291
:10F8400002EB4102A270C3F30722C2F3021101EBE3
:10F85000810102F00F0202EB4102DBB26270C3F3DE
:10F86000021202EB820203F00F0303EB4203237048
:10F8700038BD00BF384C0020FAEB010800280040DA
:10F880001FB501A8FFF79EFF01A8F9F766FF05B0B5
:10F890005DF804FB08B5FFF73FFA1B4A136843F411
:10F8A00080731360FFF7C6FE184A536B23F440338E
:10F8B00043F482035363164BDA6842F08002DA6045
:10F8C000DA685106FCD5FF221A611A6942F4FE0279
:10F8D0001A619A6822F040029A609A6822F44C52A7
:10F8E0009A60DA6822F08002DA60094BDA689206E0
:10F8F000FCD5FF225A620122064B1A70FFF7C0FFA7
:10F90000054BC3E9000108BD00700040003802400B
:10F9100000280040384C0020404C002008B5094B1E
:10F920001B7823B940F21F110748F3F73FFAFFF79E
:10F9300081FE064B9A6822F480729A60FF225A6216
:10F9400008BD00BF384C0020FAEB01080028004039
:10F9500008B5144B1B7833B9134B144A40F22711E6
:10F96000134807F0E1F9FFF765FE124BDA6822F45D
:10F970008072DA60104A916841F400319160116838
:10F9800041F400311160F0210C4A82F829134FF440
:10F99000007151609A6842F488529A60FF225A625C
:10F9A00008BD00BF384C00207BEC010854EC010876
:10F9B000FAEB0108002800400004014000E100E0EB
:10F9C000F8B51E46194B17461B7833B9184B194A20
:10F9D0004FF4A371184807F0A7F9184CFFF72AFE57
:10F9E000A56825F48075A560E56825F48075E56057
:10F9F000FFF716FE05460846FFF712FE000440EA30
:10FA000005613846FFF70CFE05463046FFF708FE55
:10FA1000084340EA0520E368DB07FCD5FF23E061EB
:10FA20006362BDE8F840FFF793BF00BF384C002089
:10FA30007BEC010869EC0108FAEB010800280040A2
:10FA4000037842788178C078FFF7BABF38B50D46A1
:10FA50000446F2F787FA194A136823F0010313608A
:10FA6000F2F7A0FA25B1164A536843F00603536033
:10FA700072B6BFF34F8FBFF36F8F124A0120136826
:10FA800023F0030343F4007343F00103136000F019
:10FA900031FD0D4B1A6942F004021A6130BF1A6938
:10FAA000022022F004021A61FFF7FEF8034A1368ED
:10FAB00043F00103136004B162B638BD10E000E00A
:10FAC000002004E00070004000ED00E062B67047E6
:10FAD00000220E4B10B51A700D4A0E4C13882046AA
:10FAE00023F040031B041B0C13800D210222FFF79F
:10FAF000B3FB204602220E21FFF7AEFB2046BDE8F5
:10FB0000104002220F21FFF7A7BB00BF484C002086
:10FB10000038004000040240284A38B5136A054600
:10FB200043F480531362052225480C461146FFF723
:10FB3000D1FB052206212248FFF7CCFB0522072135
:10FB40001F48FFF7C7FBC5B1022205211C48FFF77C
:10FB500025FB022206211A48FFF720FB022207217B
:10FB60001748FFF71BFB012C21D144F451740122EB
:10FB7000144B1C80144B1A7038BD2A4605211048BE
:10FB8000FFF70CFB2A4606210D48FFF707FB2A4624
:10FB900007210B48FFF702FB012C05D0022C03D0F4
:10FBA000032C14BF0024032444F45974DFE7022C0F
:10FBB000DBD0032C0CBF03240024D6E7003802401E
:10FBC0000000024000300140494C002000220E4B52
:10FBD00010B51A700D4A0E4C1388204623F04003CE
:10FBE0001B041B0C138005210222FFF735FB204666
:10FBF00002220621FFF730FB2046BDE8104002221A
:10FC00000721FFF729BB00BF494C0020003001400D
:10FC100000000240064B074A988111781A4618895D
:10FC2000C00701D40029FAD19089C0B2704700BF43
:10FC300000300140494C0020054AD36823F4E063BA
:10FC40001B041B0C43F0BF6343F40033D3607047C5
:10FC500000ED00E020220021114B10B5C3F88420F4
:10FC6000104B114C1A6A204642F480421A625A69BB
:10FC700042F480425A615A6922F480425A610B4A26
:10FC800091811A6A092122F480421A620222FFF746
:10FC9000E3FA2046BDE8104002220A21FFF7DCBA51
:10FCA00000E100E00038024000000240003801405E
:10FCB00010B50B4C40F22551204600F028FE48B10B
:10FCC000204600F002FE074BC0B21B6833B1BDE80E
:10FCD00010401847A388044ADBB2137010BD00BF60
:10FCE000003801404C4C00201851002010B504464B
:10FCF0008021084800F005FE0028F9D0214605487B
:10FD000000F0DFFD034C4021204600F0FAFD002802
:10FD1000F9D010BD0038014010B5441E14F8010F91
:10FD200000B910BDFFF7E2FFF8E7000008B5024890
:10FD300000F0CBFDC0B208BD003801402DE9F04312
:10FD40008846012189B08146084614461D4600F0C8
:10FD500015FD01214FF4804000F01CFD4FF4C067F9
:10FD600002230122002602A93F488DF80C308DF8AD
:10FD70000D308DF80F2002978DF80E6000F060FCBA
:10FD800007220921384800F09DFC07220A21364845
:10FD900000F098FCB8F1450FCDF810903CD14FF42D
:10FDA0008063ADF81830072C42D10023ADF8143031
:10FDB000052D4ED14FF48053ADF816300023ADF829
:10FDC0001C300C2304A92948ADF81A3000F01EFDA0
:10FDD000274B1A6802B1012240F22551234800F056
:10FDE00078FD0121214800F061FDFFF79FFF2523E9
:10FDF0008DF804309DF840308DF8053000238DF8E3
:10FE0000063001238DF80730FFF716FF01A800F038
:10FE10004BFA09B0BDE8F083B8F14F0F02D1ADF84D
:10FE20001870C0E7072CADF818600DD1592107E014
:10FE3000082C02D14FF48053B8E7092CB8D15421D3
:10FE40000C48F2F7B3FFB3E7082CAED0092CAFD1C2
:10FE5000F0E70F2D02D14FF44053ADE7022D0CBF58
:10FE60004FF400530023A7E7000002400038014090
:10FE70004C4C002084EC01080E2307B508220093A7
:10FE80004E210123FFF75AFF03B05DF804FB000089
:10FE9000402200210D4B0E48C3F884200D4B5A6AB6
:10FEA00042F400325A629A6942F400329A619A69C5
:10FEB00022F400329A61084A91815A6A032122F49D
:10FEC00000325A620222FFF7C7B900BF00E100E02A
:10FED00000000240003802400044004008B50248DB
:10FEE00000F0F3FCC0B208BD004400402DE9F04F23
:10FEF0004FF000091F46262389B09DF848808A46A6
:10FF000014468DF8043083469DF84C509DF850609F
:10FF10008DF805808DF806908DF80790FFF78CFE20
:10FF200001A800F0C1F90121084600F027FC0121D9
:10FF30004FF4003000F03AFCB5B1082302930223DD
:10FF40008DF80E908DF80C304FF00309012302A9B3
:10FF500056488DF80F308DF80D9000F071FB072298
:10FF60004946524800F0AEFBBEB104230293012380
:10FF70008DF80F3000234FF002098DF80E30032367
:10FF800002A94A488DF80C908DF80D3000F058FB0E
:10FF900007224946454800F095FBBAF1450FCDF8D8
:10FFA00010B043D14FF48063072CADF818304BD11B
:10FFB0000023ADF81430052F57D14FF4805300249F
:10FFC000ADF81630ADF81C40002E59D1ADF81A60CE
:10FFD00075B1BDF81A3043F00403ADF81A30344B54
:10FFE0001A6802B1012240F22551324800F071FC3A
:10FFF00004A9304800F00AFC01212E4800F056FC0C
:020000040801F1
:100000000DB1FFF76BFF26238DF8043000238DF828
:10001000063001238DF805808DF80730FFF70CFEC0
:1000200001A800F041F909B0BDE8F08FBAF14F0F17
:1000300002D14FF4C063B7E70023072CADF81830A6
:100040000ED14FF4827107E0082C02D14FF4805397
:10005000AFE7092CAFD1FF211748F2F7A7FEAAE7B7
:10006000082CA5D0092CA6D1F0E70F2F02D14FF410
:100070004053A4E7022F0CBF4FF4005300239EE728
:100080000823224640F227710A48ADF81A3000F0E2
:1000900020FC40F22661074800F058FC224640F25E
:1000A0002661044800F015FC92E700BF0000024002
:1000B000504C00200044004084EC0108F8B505468F
:1000C0000024134E134F8021134800F01AFC68B12E
:1000D0002946114800F0F5FB00240F4D0C4E0D4F42
:1000E0004021284600F00DFC48B1F8BD0134B4426F
:1000F000E9D94FF4A4713846F2F758FEE3E701342A
:10010000B442EDD940F251113846F2F74FFEE7E71D
:10011000FFFF0F0084EC01080044004008B5064BC7
:100120000246186000B1012240F22551034800F058
:10013000D0FB012008BD00BF504C0020004400400F
:1001400070B5134C40F22551204600F0E0FBC0B1E1
:10015000104B1D6825B1204600F0B7FBC0B2A84780
:1001600040F226610A4800F0D2FB78B140F22661E5
:10017000074800F0EBFB084B1B683BB1BDE8704043
:100180001847A388054ADBB21370E9E770BD00BFCA
:1001900000440040504C0020544C002018510020D6
:1001A000BFF34F8F0449054BCA6802F4E062134362
:1001B000CB60BFF34F8FFEE700ED00E00400FA05CF
:1001C00010B5441EE3B2052B03D90E211148F2F7F6
:1001D000EDFDFEF7BFFD45F255520F4B1A60DA6890
:1001E000D207FCD4052C06D8DFE804F003090B0D78
:1001F0000F1101225A604CF6CC421A6010BD022247
:10020000F8E70322F6E70422F4E70522F2E70622E4
:10021000F0E700BF55ED01080030004010B5194C63
:1002200023683BB95F2000F0D9FA28B1164B236050
:1002300000F0E4FA206810BD5E2000F0CFFA08B1AB
:10024000124BF4E75D2000F0C9FA08B1104BEEE75D
:100250005C2000F0C3FA08B10E4BE8E75B2000F029
:10026000BDFA08B10C4BE2E75A2000F0B7FA08B12A
:100270000A4BDCE7592000F0B1FA08B1084BD6E789
:10028000084BD4E7584C0020D3EC0108E3EC0108FC
:10029000F9EC010814ED010823ED010832ED010825
:1002A0004BED010898C9010830B5012403780A4DC7
:1002B00003F01F029440C278590952B1074A2B44F7
:1002C000D26842781201D2B283F8002345F8214067
:1002D00030BD2031FAE700BF00E100E000ED00E0B2
:1002E00008B5084B98420BD101214FF4007000F083
:1002F00069FABDE8084000214FF4007000F062BACE
:1003000008BD00BF0024014043680A7923F0407310
:1003100023F4807343EA02230A6810B51343436051
:10032000D1E9032313438A6884681343084A2240AF
:1003300013434A7943EA420383600A7D036B013A1F
:1003400023F0F873D2B243EA0253036310BD00BF37
:10035000FDF7FFC000234FF040720360037143714B
:100360008360C0E90323012303757047836819B1D3
:1003700043F001038360704723F00103FAE70000B4
:10038000044B5A6818B142F400025A60704722F4D4
:100390000002FAE7002701401D2970B51BD9072587
:1003A000A1F11E06C46D06EB4606B54024EA05041D
:1003B00003FA06F62643C665062A38D81F24013AF2
:1003C000036C02EB8202944023EA040301FA02F276
:1003D0001A43026470BD13290DD90726A1F1140533
:1003E000C46805EB4505AE4024EA060403FA05F5AA
:1003F0002543C560E0E709290DD90726A1F10A04C4
:10040000056904EB4404A64025EA060503FA04F452
:100410002C430461D0E70726446901EB4105AE4057
:1004200024EA060403FA05F626434661C4E70C2ACB
:100430000CD81F24073AC36B02EB8202944023EAD4
:10044000040301FA02F21A43C263C3E7122A0CD86A
:100450001F240D3A836B02EB8202944023EA0403CB
:1004600001FA02F21A438263B4E7182A0CD81F2457
:10047000133A436B02EB8202944023EA040301FA2D
:1004800002F21A434263A5E71F24193A036B02EBF9
:100490008202944023EA040391401943016399E7DF
:1004A000836843F0804383607047806D80B27047FB
:1004B0000368194214BF012000207047C94301603E
:1004C00070470000044B1A6818B142F002021A602B
:1004D000704722F00202FAE7003C0240044B1A681F
:1004E00018B142F004021A60704722F00402FAE7E1
:1004F000003C0240044B1A6818B142F008021A602E
:10050000704722F00802FAE7003C0240044B5A68A8
:10051000D20741BF034ADA60034ADA60704700BF7E
:10052000003C0240EFCDAB8905040302024A536848
:1005300043F0010353607047003C0240014B986157
:10054000704700BF003C0240084B9A69D10709D4AC
:100550009A69D20508D49B6913F4F05F14BF032095
:10056000042070470120704702207047003C024081
:10057000042313B504468DF80730FFF7E5FF8DF827
:1005800007009DF80730012B0AD11CB905238DF80F
:10059000073007E0FFF7D8FF013C8DF80700F0E7D0
:1005A000002CF3D09DF8070002B010BD10B5044632
:1005B0004FF40040FFF7DCFF042804BF0023236052
:1005C00010BD000038B504464FF400400D46FFF75B
:1005D000CFFF04280BD1064A4FF40040536823F4A0
:1005E000807353602560BDE83840FFF7C1BF38BD58
:1005F000003C024038B504464FF400400D46FFF77A
:10060000B7FF04281BD135B125704FF40040BDE879
:100610003840FFF7ADBFFF2324F0030504F00304C7
:100620002968E40003FA04F421EA04042846FFF7E9
:10063000BDFF21462846BDE83840FFF7C3BF38BD9F
:100640002DE9F0430022012703250E6807FA02F383
:1006500033EA060431D14FEA420C05FA0CF4E443C4
:1006600091F804E0D0F800900EFA0CF804EA0909B9
:100670000EF1FF3E48EA0908BEF1010FC0F8008004
:1006800011D8D0F808E004EA0E0E4C7904FA0CF404
:1006900044EA0E048460848824EA03048B7993403E
:1006A0009BB223438380C36805FA0CF423EA040455
:1006B000CB7903FA0CF32343C3600132102AC5D16E
:1006C000BDE8F08310B50F2401F00703C90800EB63
:1006D0008100016A9B009C4021EA04010162016AD9
:1006E0009A400A43026210BD204B10B59A6802F08E
:1006F0000C020C2A30D8DFE802F02F2F2F2F072F03
:100700002F2F072F2F2F2000194B184A03609368B3
:100710001849C3F30313CC5C0368E3404360946857
:10072000C4F302240C5D23FA04F484609268C2F3DB
:10073000C2228A5CD340C36010BD99680E4CC1F3DD
:1007400083419A68615C9B68094BC2F381524B43B9
:100750000132B3FBF2F3D8E74FF400425B68C3F316
:100760004233013302FA03F3CFE700BF00380240FF
:100770000024F400F401002004020020044BDA6994
:1007800011B11043D861704722EA0000FAE700BFB8
:1007900000380240044B1A6A11B1104318627047C6
:1007A00022EA0000FAE700BF00380240044B5A6A10
:1007B00011B110435862704722EA0000FAE700BF07
:1007C00000380240044B5A6911B110435861704718
:1007D00022EA0000FAE700BF003802404309012B7B
:1007E000054B00F01F000CBF1B685B6B23FA00F089
:1007F00000F00100704700BF00380240024A536B0E
:1008000043F08073536370470038024030B50D46A3
:100810000446028AEB8892B222F440521A43898934
:1008200002828389288923F4B052AB8822F00C021B
:100830000343688985B003431343A381A38A6846B1
:100840009BB223F440730B43A382FFF74DFFDDE916
:100850000231154A944218BF19461923A2894B4305
:10086000296810044CBF49008900B3FBF1F16425ED
:10087000B1FBF5F3A2891801120405FB13130BD584
:10088000DA003232B2FBF5F202F0070242EA00036C
:100890009BB2238105B030BD1B013233B3FBF5F3AE
:1008A00003F00F030343F3E700380140838919B1D4
:1008B00043F400538381704723F400531B041B0C43
:1008C000F8E7C1F30801818070478088C0F3080011
:1008D000704701F01F0310B5C1F342140121012C30
:1008E00001FA03F105D10C3003683AB119430160F4
:1008F00010BD022C0CBF10301430F5E723EA0101C3
:10090000F5E70388194214BF012000207047012336
:10091000C1F3421210B5012A01F01F0403FA04F3D7
:100920000DD182891340028892B26BB10123090A6A
:1009300003FA01F10A4214BF1846002010BD022A32
:100940000CBF028A828AEDE71846F7E70B0A0121FD
:100950009940C94389B20180704700002DE9F341F5
:100960001F46002304460D46019316461AB901207E
:1009700002B0BDE8F08140F6FF7301934FF40031FF
:10098000204600F00EFD002852D10121204600F043
:10099000D8FC4FF2FF71204600F0ECFC012120460C
:1009A00000F0B9FC40F6FF73DFF8B88101934146CF
:1009B000204600F0EBFC002841D0394601222046B9
:1009C00000F0CAFC40F6FF73614F019339462046A0
:1009D00000F0E7FC002838D0012E42D1002120464B
:1009E00000F0AFFCF1F7BEFA31462046238B00F051
:1009F0009DFCF1F7D7FA40F6FF73564E019331464E
:100A0000204600F0CEFC30B3204600F0B0FC287049
:100A100040F6FF73504D01932946204600F0C1FC7B
:100A20000028A4D0019B5A1E0192002BF4D104E0AF
:100A3000019B5A1E0192002BA0D1002098E7019B38
:100A40005A1E0192002BB2D1F7E7019B5A1E019268
:100A5000002BBBD1F1E7019B5A1E0192002BCED196
:100A6000EBE7022E25D1F1F77DFA4FF40061204625
:100A700000F080FC0021204600F063FC238BF1F79E
:100A800091FA40F6FF73354E01933146204600F04F
:100A900088FC40B10121204600F048FC238A2B70DD
:100AA000238A6B70B4E7019B5A1E0192002BECD194
:100AB000C3E740F6FF77033E238BDFF8A0802E4488
:100AC000B54201972CD1254E3146204600F069FCF5
:100AD00090B30021204600F034FCF1F743FA2046A1
:100AE00000F045FC01212870204600F01FFCF1F7C2
:100AF00059FA204600F03BFC40F6FF73184E687030
:100B000001933146204600F041FCD8B1204600F068
:100B10002EFCA8707CE7019B5A1E0192002B8CD002
:100B20004146204600F03DFC0028F4D0204600F06D
:100B30001EFC05F8010BC3E7019B5A1E0192002B16
:100B4000C2D17AE7019B5A1E0192002BD9D174E7DA
:100B500002000010400000101000001004000010FF
:100B600040000300010003002DE9F3411E4600236D
:100B700004460D46019317461AB9012002B0BDE89C
:100B8000F08140F6FF7301934FF40031204600F0EE
:100B900008FC002846D10121204600F0BCFB40F6AD
:100BA000FF73DFF8E48001934146204600F0EEFB3E
:100BB00000283ED031460022204600F0CDFB40F612
:100BC000FF732D4E01933146204600F0DFFB0028D5
:100BD00035D0297820466E1C00F0C7FB3D4440F616
:100BE000FF77DFF89880AE42019733D1234D294635
:100BF000204600F0D6FB002838D02046012100F026
:100C000095FB40F6FF731E4D1E4C0193294620466E
:100C100000F0C7FB0028B0D0019B5A1E0192002BA8
:100C2000F4D104E0019B5A1E0192002BACD10020AC
:100C3000A4E7019B5A1E0192002BB5D1F7E7019B57
:100C40005A1E0192002BBED1F1E7019B5A1E019260
:100C5000002BECD04146204600F0A3FB0028F4D046
:100C600016F8011B204600F080FBBCE7019B5A1ED2
:100C70000192002BBBD1DAE78200070004000010CC
:100C80001000001000540040010003002DE9F34162
:100C90001E46002304460D46019317461AB901204B
:100CA00002B0BDE8F08140F6FF7301934FF40031CC
:100CB000204600F076FB002837D10121204600F0C5
:100CC0002AFB40F6FF73DFF8E0800193414620469F
:100CD00000F05CFB002842D031460022204600F0A4
:100CE0003BFB40F6FF732C4E01933146204600F04B
:100CF0004DFB002839D0297820466E1C00F035FBCA
:100D00003D4440F6FF77DFF89480AE42019737D13B
:100D1000224D2946204600F044FB0028BFD1019B0C
:100D20005A1E0192002BF4D104E0019B5A1E01923D
:100D3000002BBBD12046012100F0F8FA40F6FF73EA
:100D4000174D184C01932946204600F02AFB20B18C
:100D5000019B5A1E0192002BF5D10020A0E7019BB8
:100D60005A1E0192002BB1D1E4E7019B5A1E019259
:100D7000002BBAD1DEE7019B5A1E0192002BD9D07D
:100D80004146204600F00DFB0028F4D016F8011B68
:100D9000204600F0EAFAB8E78200070004000010DD
:100DA00010000010005400400100030000232DE952
:100DB000F3410D464FF4003104461746019300F00D
:100DC000F0FA18B9002002B0BDE8F0810FB9012097
:100DD000F9E7297820466E1C00F0C7FA3D4440F63A
:100DE000FF77DFF86C80AE4201971FD1184D29467E
:100DF000204600F0D6FA28B32046012100F096FAEA
:100E000040F6FF73134D144C01932946204600F021
:100E1000C8FA0028DBD0019B5A1E0192002BF4D1A6
:100E2000D0E7019B5A1E0192002BCBD041462046B1
:100E300000F0B7FA0028F4D016F8011B204600F0A5
:100E400094FAD0E7019B5A1E0192002BCFD1B9E74B
:100E50000400001010000010005400402DE9F34180
:100E60001F46002304460D46019316461AB9012079
:100E700002B0BDE8F0814FF4003100F092FA08B9F9
:100E80000020F5E70121204600F05BFA4FF2FF71E8
:100E9000204600F06FFA0121204600F03CFA40F6AF
:100EA000FF73DFF8B88101934146204600F06EFAE7
:100EB00000283AD039460122204600F04DFA40F68B
:100EC000FF73614F01933946204600F06AFA00280B
:100ED00031D0012E3BD10021204600F032FAF1F74B
:100EE00041F831462046238B00F020FAF1F75AF8FA
:100EF00040F6FF73554E01933146204600F051FAFB
:100F0000F8B1204600F033FA287040F6FF73504DD8
:100F100001932946204600F044FA0028A7D0019BFF
:100F20005A1E0192002BF4D1AAE7019B5A1E01928E
:100F3000002BB9D1A4E7019B5A1E0192002BC2D10C
:100F40009EE7019B5A1E0192002BD5D198E7022EF5
:100F500029D14FF40061204600F00CFAF1F702F8B5
:100F600000212046238B00F0ECF9F1F71BF840F646
:100F7000FF73384E01933146204600F012FA60B1FB
:100F8000F0F7F0FF0121204600F0D0F9238A2B7002
:100F9000238A6B70F1F706F8B7E7019B5A1E01929E
:100FA000002BE8D16CE740F6FF77033E238BDFF898
:100FB000A4802E44B54201972DD1264E31462046BD
:100FC00000F0EFF998B30021204600F0BAF9F0F7ED
:100FD000C9FF204600F0CBF901212870204600F01F
:100FE000A5F9F0F7DFFF204600F0C1F940F6FF73E6
:100FF000194E687001933146204600F0C7F9E0B100
:10100000204600F0B4F9A8707FE7019B5A1E0192B8
:10101000002B3FF435AF4146204600F0C2F90028CE
:10102000F3D0204600F0A3F905F8010BC2E7019BBD
:101030005A1E0192002BC1D122E7019B5A1E019238
:10104000002BD8D11CE700BF0200001040000010A8
:101050001000001004000010400003000100030015
:1010600038B5204B08219A691F4842F400129A6152
:101070009A6922F400129A615A6A22F400125A62A2
:10108000FEF76EF9012308211A461748FEF7A6F865
:10109000092115480122FEF7DFF809211248FEF761
:1010A00074F9D8B1012038BD08212846FEF758F957
:1010B000FDF7A4FE08212846FEF758F9FDF79EFE2D
:1010C000013CF1D109210848FEF75FF920B940F24F
:1010D00063110648F1F76AFE2046E4E73324024D27
:1010E000EEE700BF0038024000040240A8ED01080E
:1010F0002DE9FF41444B054698420E4617467CD1E8
:1011000003F5F2335A6A082142F400125A629A69CE
:101110003E4842F400129A619A6922F400129A61E0
:10112000FEF71EF9012308211A463848FEF756F843
:10113000092136480122FEF78FF809213348FEF7CE
:1011400024F9002855D0012308211A462F48FEF71C
:1011500045F8042208212D48FEF7BCF80123092197
:101160001A462A48FEF73AF8042209212748FEF7D2
:10117000B1F8274B9A6942F400129A619A6922F4F5
:1011800000129A61684600F0ADF8224B694601935F
:101190004FF48063ADF80A304FF480432846ADF831
:1011A0000C30ADF80870009600F038F828460121A0
:1011B00000F0A6F8012019E008214046FEF7D0F81B
:1011C000FDF71CFE08214046FEF7D0F8FDF716FE9D
:1011D000013CF1D109210D48FEF7D7F80028B2D122
:1011E0000D4840F28B11F1F7E1FD204604B0BDE857
:1011F000F0813324DFF81480EAE74FF4CD7106481C
:10120000F1F7D4FDBEE700BF0054004000040240E7
:10121000003802400000FFBFA8ED01087FB504467A
:10122000868868460D46FFF75FFA029A2B4926F03A
:101230003F06B2FBF1F13604360C88B20643A680B5
:101240002388274E23F001031B041B0C23802B68EB
:10125000B3421ED85B00B2FBF3F39BB2042B38BF42
:101260000423013080B22084A3832388AA8843F01A
:10127000010323802388698923F481630A4323F0CF
:101280000203134323802A89AB891343238104B0CB
:1012900070BD4BF6FF70EE8886421BBF192043439A
:1012A00003EB4303B2FBF3F30BBFB2FBF3F39BB2CD
:1012B0009BB243F48043C3F30B020AB943F001032A
:1012C0004FF496724A434FF47A7192FBF1F2013275
:1012D00092B243F400432284C6E700BF40420F00AD
:1012E000A086010041F28832044BC0E900230023AC
:1012F00083604FF480438381704700BF0000FFBFCD
:10130000038819B143F001030380704723F0010300
:101310001B041B0CF8E7038819B143F480730380A6
:10132000704723F480731B041B0CF8E7038819B182
:1013300043F400730380704723F400731B041B0CF9
:10134000F8E7038819B143F480630380704723F4FE
:1013500080631B041B0CF8E722B141F0010189B244
:101360000182704701F0FE01F9E701827047008AAF
:10137000C0B270470388B1F5006F1BBF23F4006350
:101380001B0443F400631B0C03807047838A008BAB
:1013900043EA004321F07F401840431A5842584125
:1013A0007047002382B0009301930B0F01900093CC
:1013B000009B21F07F4153B1019B14330193019BAA
:1013C0001B680B4214BF0120002002B07047019B34
:1013D000090C1833F2E70078013070470FB404B0FD
:1013E000704700002DE9FF470F46002104AC254E51
:1013F00044F8041D80469246306822469946F1F72B
:10140000D1FB0128039B31D13BB14FF080521E4BE1
:101410001A60BFF34F8FBFF36F8FB7F5C87F88BFD8
:101420004FF4C87741463A46184805F0D0FD184DAC
:10143000164B21463068AF802B60A5F806A085F8D2
:101440000890F1F791F9039B3BB14FF080520E4B9E
:101450001A60BFF34F8FBFF36F8F0E4800940023C5
:10146000012204210068F0F779FA039B3BB14FF0A9
:101470008052054B1A60BFF34F8FBFF36F8F04B0DC
:10148000BDE8F087604E002004ED00E0C44C002071
:10149000B84C0020684E002003480023012202219E
:1014A0000068F0F7F1B900BF684E00201FB50023B7
:1014B0000C4904AA42F8043D08700B4800924021F0
:1014C00001220068F0F74AFA039B3BB14FF08052CB
:1014D000064B1A60BFF34F8FBFF36F8F05B05DF8F7
:1014E00004FB00BFA84C0020684E002004ED00E083
:1014F0001FB5002304AA42F8043D0A480092802147
:1015000001220068F0F72AFA039B3BB14FF08052AA
:10151000054B1A60BFF34F8FBFF36F8F05B05DF8B7
:1015200004FB00BF684E002004ED00E01FB5104B27
:101530001C680346A8B1002304AA42F8043D0092A7
:10154000082101222046F0F709FA039B3BB14FF036
:101550008052084B1A60BFF34F8FBFF36F8F04B0F8
:1015600010BD012208212046F0F78EF9F7E700BFF1
:10157000684E002004ED00E01FB5002304AA42F8E5
:10158000043D00920122094811460068F0F7E6F98F
:10159000039B3BB14FF08052054B1A60BFF34F8F56
:1015A000BFF36F8F05B05DF804FB00BF684E0020ED
:1015B00004ED00E01FB5002304AA42F8043D0A48E8
:1015C0000092102101220068F0F7C8F9039B3BB19B
:1015D0004FF08052054B1A60BFF34F8FBFF36F8FF0
:1015E00005B05DF804FB00BF684E002004ED00E08C
:1015F00000487047A04C0020114810B5002303227A
:101600004FF480710068F0F73FF94FF080520D4BB6
:101610001A60BFF34F8FBFF36F8F0B4C2068F1F749
:101620000DFB40B1BDE81040002308481A4619469A
:101630000068F0F789BF0120EFF7DCFDEEE700BF9F
:10164000684E002004ED00E0644E00205C4E002057
:10165000F8B5104B01461868F1F762F90446B8B1C5
:101660004FF080560C4F0D4D002303224FF40071B4
:101670003868F0F709F92E60BFF34F8FBFF36F8F13
:101680003868EFF7DBFB2E60BFF34F8FBFF36F8F30
:101690002046F8BD5C4E0020684E002004ED00E0BE
:1016A000014B1860704700BF544E002070B50446CF
:1016B00078B10378032B0CD1436853B10025054E54
:1016C0001868F26990476068F3690560984765603B
:1016D000257070BD7C4C002010B50D480D4C0023CA
:1016E000052221460068F0F72FFF012805D10A4B9B
:1016F0001B6863B1BDE810401847084B21780848C3
:101700005B6998472046BDE81040FFF7CFBF10BD8A
:10171000584E0020AC4C0020544E00207C4C002041
:10172000F7ED01087FB50024094E002201A93068B9
:10173000F1F764F8651C30B9064BE1B25B69064805
:10174000984704B070BD01A8FFF7B0FF2C46ECE746
:10175000584E00207C4C00201EEE0108014B1868FA
:10176000704700BF584E002010B50446064B010AD2
:10177000A3F84A00202000F09DFBE1B22120BDE843
:10178000104000F097BB00BF1C51002008B5FFF7C8
:10179000EBFF0122014B83F8522008BD1C510020B1
:1017A000002238B50B4B05461D2083F84E100C4621
:1017B00083F84C2000F0D8FB20F0060040EA4401FA
:1017C000C9B21D2000F076FB2946BDE83840232031
:1017D00000F070BB1C51002013B5164C0120A3680B
:1017E0009847002341F6FE720093009B934218DD58
:1017F000A36802209847002341F6FE720193019BE3
:10180000934212DD0C4BB5211C6C4020A047A02157
:101810004120A04700210120234602B0BDE810402E
:101820001847009B01330093DFE7019B01330193CD
:10183000E5E700BF7C4C00205CF10108094B07B5CF
:101840001B6CC2213B209847002341F6FE72019396
:10185000019B934202DD03B05DF804FB019B013361
:101860000193F5E75CF101089048914B2DE9F04FA9
:101870000360904B904F8360904B914C4360914B31
:1018800085B0C360904B914D0361914BDFF874A21A
:101890008361904BDFF87092C3613B68984763693E
:1018A0008D489847002328681A461946F0F74CFEE1
:1018B000DFF858B29AF8040068B94FF0FF331946C0
:1018C00003AAEFF79DFF68B96669EFF775FE014659
:1018D0008248B047EEE741F2883303AA4FF0FF3168
:1018E0000020EEE7039BDE0516D500F0A1FA0020EC
:1018F00000F044FEFB6A9847FFF714FF63697848DD
:1019000098470023D9F800001A461946F0F71CFE44
:101910000020EFF7E7FCCDE7980510D500F088FA36
:10192000FFF78CFFFB6A9847FFF7FCFE63696D4881
:1019300098476421D9F80000F0F7F2FFBAE7D9F828
:101940000000F1F77BF9012803D1636966489847E5
:10195000B0E7DBF8003023B940F23B116348F1F700
:1019600025FA039B190604D50722614B1A70FFF76D
:10197000B3FE039B5A0752D500212868F0F7D0FF29
:1019800001284CD1A3690C209847064688B96369A1
:101990000C21584898473346324631462868F0F7BC
:1019A000D3FD002886D14FF4A8715048F1F7FEF915
:1019B00080E7DFF85C81A369B8F804009847034624
:1019C000A0B9B8F80410019062694B489047E269E9
:1019D00030469047019B28681A461946F0F7B4FD37
:1019E00000287FF467AF4FF4AC71DEE708F1040222
:1019F00003CA33607060B1601846D8F80010B8F8B8
:101A0000042005F0E4FA0322394B1A705E60FFF7F8
:101A100063FE002328681A461946F0F795FD039BDC
:101A2000DB0709D50123324E337000237360EFF7D3
:101A30008FFAB060FFF750FE039BDE0606D5052245
:101A40002B4B1A7000225A60FFF746FE039B1807C3
:101A500006D50422264B1A7000225A60FFF73CFE7E
:101A6000039B990706D50222214B1A7000225A6067
:101A7000FFF732FE039B9A0606D506221C4B1A700E
:101A80001E4A5A60FFF728FE039B5B067FF512AFE4
:101A90001B4B1A78164B32B108221A7000225A607A
:101AA000FFF71AFE06E70922F7E700BF5C4C0020AB
:101AB00079150108E51301085CF101089914010882
:101AC0007C4C00202D150108B5150108604E002042
:101AD000AD140108F114010818F001082EF00108F6
:101AE0004CF0010874F001088BF00108A1F0010826
:101AF000AC4C0020EDF0010823F10108A94C0020B6
:101B0000A84C0020A04C0020644E0020584E00201D
:101B1000B84C0020044B10B55B6998470446FFF7AA
:101B20005BFE204610BD00BF5CF10108F0B56B4CB8
:101B3000064625460F460FCE0FC596E80F0085E8EE
:101B40000F0097E803006369654E013B033388BFCC
:101B5000644B85B088BF6361636886E80300013B1E
:101B6000033307D96048636998474FF423715F488E
:101B7000F1F71CF92368013B033307D95C4863691B
:101B800098474FF424715948F1F710F9A368013BC5
:101B9000033307D95748636998474FF42571534871
:101BA000F1F704F9E368013B033307D9524863694D
:101BB00098474FF426714D48F1F7F8F82369013B37
:101BC000033307D94D48636998474FF42771474855
:101BD000F1F7ECF8E369013B033304D94FF42871C2
:101BE0004248F1F7E3F8A369013B033304D94FF40A
:101BF00029713E48F1F7DAF8414B0FCB8DE80F0021
